:020000040800F2
:1000000000000120C15405085D5505089DBA01088E
:10001000F5B801085D5505085D55050800000000AC
:100020000000000000000000000000005D55050811
:100030005D550508000000005D550508BDAC0108D0
:100040005D5505085D5505085D5505085D550508B4
:100050005D5505085D55050851A4000859A4000820
:1000600061A4000869A4000871A4000849A200085E
:1000700059A200086DA2000881A2000895A20008FC
:10008000A9A20008BDA200085D5505085D55050838
:100090005D5505085D5505085D55050879A40008FE
:1000A00085DF000871DE000895DF000861DE0008CA
:1000B00099DE0008A9DE0008B9DE0008599D000895
:1000C0004D9D00088D9D0008819D00085D55050827
:1000D0005D55050809AC010815AC010821AC010803
:1000E00081A400085D5505085D550508A5DF0008D9
:1000F0005DDF00085D5505084DDF0008D1A200084E
:100100005D55050891D00008C9DE00085D55050859
:100110002DAC010839AC0108D9DE000805CE040871
:10012000E5A20008F9A200080DA3000821A3000819
:1001300035A30008000000000000000000000000DF
:1001400000000000000000000000000089C3040857
:1001500049A300085DA3000871A3000845AC01088D
:10016000C19D0008B59D00085D5505085D55050851
:100170005D5505085D550508000000000000000001
:100180005D5505085D5505085D5505085D55050873
:100190005D5505085D550508000000005D55050822
:1001A0000000000000000000000000005D55050890
:1001B0005D5505085D5505080000000000000000C1
:1001C000000000000000000000000000000000002F
:1001D0000000000000000000000000005D55050860
:108000001B4B1C4A03F5727C016803E063452BD0CF
:1080100053F82C2F9142F9D170B593F804E04279CE
:1080200096450AD0634505D053F82C2F9142F4D0E1
:108030006345F9D14FF0FF3070BD9E468468002241
:10804000DEF80C50A54208D001320EF10C0E032AC6
:10805000E8D0DEF80C50A542F6D1DEF81050C66824
:10806000B542F1D150B270BD4FF0FF30704700BF44
:1080700080700508000001404368426D30B49A6189
:10808000EFF31182502383F312884168D2B2856CDA
:108090000B68046D23EA050323430B6082F3118808
:1080A000436981681A68096822F00102D0E908541E
:1080B0001A60826A1D605C615A60D0E90B429C6064
:1080C000DA600023B0F86C2030BCCA6203777047D6
:1080D00030B5FAB18E464FEA014C034600F1C005B7
:1080E000002419680C3353F8042C43F8084C41EA77
:1080F0000C0142EA0E02AB4243F80C1C43F8042C7C
:10810000EFD1D0F8C03043EA0E03C0E93144C0F8E3
:10811000C03030BD4FEA014E8C46DEE783695969B5
:10812000B3F810C00A6830B49C6822F001022468D9
:108130000A60E26822EA0C02E260027D04681F2AFB
:1081400006D9203A082065689040284242D0FEE7D0
:108150000820256890402842F9D1202000FA02F238
:10816000A260254A1278002A32D01A7F012A36D01E
:10817000D3F800210132C3F80021EFF3118150221E
:1081800082F312885868C9B29D6C0268DC6C22EADE
:1081900005022243026081F311885A699968D3E984
:1081A0000D40096814605061D3E90F40546090603D
:1081B0005C6CB3F8B400D4600124C862106820433A
:1081C00010601A8A1C7783F8FD40CB681343CB609C
:1081D00030BC7047202000FA02F2E260C1E70022C2
:1081E000D3F8040183F8FD2001300A68C3F80401C4
:1081F00022F001020A60EBE78001002010B40C4C71
:108200006368002B11DD002004F1080C0146DCF846
:10821000AC3003F1C00259600C339342FBD1013002
:1082200063680CF5867C8342F1DC5DF8044B704793
:1082300080010020704700BF024B03EB401090F814
:108240005504704780010020704700BF0B4890F82C
:108250006C1589B101EB4101002300F27450490013
:1082600010B41C4650F82320063302B114608B4230
:10827000F8D15DF8044B7047704700BF80010020C3
:108280000B4890F86C1589B101EB4101002300F215
:108290007450490010B41C4650F82320063302B134
:1082A00014609942F8D15DF8044B7047704700BFE5
:1082B0008001002001207047034B00EB400003EBDE
:1082C000C00090F88505704780010020204890F894
:1082D0006C35002B3AD0002200F274534FF02C0C76
:1082E0002DE9F0434FF0500E1A4E1B4D144607E097
:1082F00053F8181B01320C6090F86C15914223DD85
:10830000197C0029F4D05F684FF0FE08B90AA1F586
:1083100080115229294498BF91F8F483EFF3118119
:108320008EF31288D7F824900CFB0868C9B209F1C3
:108330000109C8F82890D7F8148048F00108C7F858
:10834000148081F31188D3E7BDE8F083704700BF44
:1083500080010020101901208070050807EE900AA6
:10836000B8EE670A704700BFBCEEC00A10EE103AC4
:1083700098B27047C84BD3E9A51270B58C0FC2F301
:10838000072C100E83F8C842C1F38364000183F800
:10839000C942C1F3016483F8CA42C1F3074483F8B8
:1083A000CB42C1F30724C9B283F8CC42C2F30354D1
:1083B00083F8CD12A3F8CE02C2F3C030B3F8CE12C8
:1083C00089B22143C2F30344A3F8CE12C2F3403171
:1083D00083F8D042C2F3803483F8D102002083F8BE
:1083E000D24283F8D312C2F3003183F8D41293F847
:1083F000201383F8D502012940F2F380022900F00E
:10840000C580D3F89C122A204FEA4C0C83F8E14235
:10841000C1F3C01201F07F010CF07E0C83F8E2C2C0
:108420004FF0010C93F8E2421443D3F8A02283F8F2
:10843000E242D40F83F8E312910D83F8E442C2F3D1
:10844000417401F00C01C2F3815583F8E542C2F397
:10845000826483F8E64283F8E71293F8E712D3F8D0
:10846000A442294383F8E712C2F3405183F8E8128B
:10847000002183F8E912C2F3004183F8EA12C2F343
:10848000C03183F8EB12C2F3803183F8EC12C2F3EF
:10849000403183F8ED12C2F3003183F8EE12C2F3DB
:1084A000812183F8EF12C2F30121C2F3460283F85F
:1084B000F012C4F3074183F8F122220E090283F877
:1084C000F2C283F8F422C4F30722A3F8F6122406BA
:1084D000B3F8F61289B21143A3F8F612D3F8A81232
:1084E000C3F8F8420C0ED3F8F82242EA0442C3F86B
:1084F000F8220A0AD3F8F84202F47F422243C1F379
:108500000724C9B2C3F8F822D3F8F852D3F8AC2242
:108510002C43C3F8F84283F8FC12110E83F8FD12C5
:10852000110C0906C3F800131102D3F800430A46E0
:1085300001F47F01214392B2D3F8B042C3F8001393
:10854000D3F800130A43C3F80023C4F30352D3F84B
:10855000001341EA1461C3F8001393F804131143A4
:10856000C4F3072283F80413210A01F47061A3F80D
:108570000613B3F8061389B21143C4F34602A3F8F5
:10858000061383F8082383F809C370BD1204D3F8D7
:108590009C1202F47C12C1F3072CC3F8D8220A0EF5
:1085A000D3F8D84244EA0224C1F30742C3F8D842C0
:1085B000D3F8D84222434FF40074C3F8D822D3F83A
:1085C000D822C3F81843013240F10004A40244EA5F
:1085D00092549202C3F81443C1F38034C3F81023B9
:1085E00012E74FEA8C2CD3F89C1292004FF0010E48
:1085F0000CF44064C1F3C26502F47F72C1F3072C2E
:10860000C3F8D842D3F8D8422243CC0BC3F8D822BF
:1086100004F00602D3F8D84244EA9174C3F8D84271
:10862000C1F3026483F8DC5283F8DD42C1F34254A3
:1086300083F8DE42C1F3824483F8DF42C1F3C034E1
:1086400083F8E02293F8E022224383F8E022D3F873
:10865000D84293F8E02293F8D05202320EFA05F590
:108660000EFA02F2C3F81853D617A2FB052E05FB2B
:1086700006EE04FB0EEE0134A2FB0424A644520ACB
:10868000C1F3803442EACE52C3F810234FEA5E228F
:10869000C3F81423B8E600BF10190120B4224FF428
:1086A000A57C4FF4EB71002382801022A0F802C059
:1086B0004FF4E17C02814FF48772C1809621828160
:1086C00044220370A0F80AC0C1814382028270472D
:1086D00070B50E4E0D461446D6F878333BB11A6885
:1086E0009B881269134096F8752352B15BB9FFF766
:1086F00041FED6F810234FF4007300202A60238037
:1087000070BD002BF3D14FF0FF3070BD1019012068
:10871000002070470020704738B5074B14460D46BF
:10872000D3F818341B6A984702464FF400730020B0
:1087300012682A60238038BD1019012008B5074B44
:10874000D3F8183433B15B69984780F00100404298
:1087500040B208BD4FF0FF3008BD00BF1019012026
:10876000002070472DE9F04123B3164688469F1834
:10877000144DD5F81844002341463046A4681A46E3
:10878000A0470028F5D0D5F8183433B15B69984775
:1087900020B9D5F81834002BF8D1FEE7013608F5DA
:1087A0000078B742E5D1D5F81C340020C5F8203454
:1087B000BDE8F081034D0020D5F81C34C5F8203405
:1087C000BDE8F081101901202DE9F0415BB3164698
:1087D0000F4603EB0208184C04E0D4F8181419B142
:1087E0004B699847D4F8181400230D693046394670
:1087F0001A46A8470028F0D1D4F8183433B15B6981
:10880000984720B9D4F81834002BF8D1FEE7013688
:1088100007F50077B045E5D1D4F81C340020C4F842
:108820002034BDE8F081044C0020D4F81C34C4F896
:108830002034BDE8F08100BF1019012000207047EE
:10884000034B93F84803003818BF0120704700BF5E
:10885000101901201C4AD2F878336BB1186892F8CD
:1088600075139B880069034021B12BB1002382F866
:1088700048337047002BF9D092F84833032B0FD8B8
:1088800092F83C330133DBB2072B82F83C33EDD84E
:10889000D2F81C140123C2F8381382F84833704709
:1088A000D2F8243409489908B0EB930F4FF0020333
:1088B00006D249085B0081429BB201D9FF2BF8D94F
:1088C000A2F88033DCE700BF10190120801A0600EF
:1088D000826D136A5B681B78FF2B08D090F8F0302C
:1088E000013BDBB280F8F0301BB101207047002063
:1088F0007047126A0220526813707047836D1B6ABA
:108900005B681B78FF2B0AD190F8F030002B03F145
:10891000FF3280F8F02014BF0120022070470020B1
:10892000704700BF034B93F84803032894BF00200F
:108930000120704710190120004870475C1C01207D
:10894000034B93F84803003818BF0120704700BF5D
:1089500010190120034B93F84803032894BF00200B
:108960000120704710190120004870475C1C01204D
:10897000184B002030B49C7B14B11D688D4205D08B
:10898000013010330B28F6D130BC7047AAB1124B1E
:1089900003EB40218A4201D1022C19D00F4B93F8EE
:1089A000E4278AB10E4B01225A7000F5B170012202
:1089B00003EB00139A7130BC7047094B00F5B1709E
:1089C00003EB00139A71DFE7012283F8E427E9E75C
:1089D000183BEAE7B0430120B02D0120983D01206B
:1089E000982D0120002330B41C4C04F5C36084F89A
:1089F000D03603E0013310300B2B15D005688D42C3
:108A0000F8D190F80EC0BCF1030FF3D1C2B11449F4
:108A100001EB4320824209D1A1F1180203F5B173A1
:108A2000012102EB0313997130BC704794F8E427DD
:108A300012B9012284F8E4270A4A01215170EDE7B6
:108A4000D4F8CC1603F5B173064A0420013102EBC9
:108A50000313C4F8CC169871E6E700BF983D0120D7
:108A6000B02D0120982D0120A0B183681BB10D4BC2
:108A700007229A7070470B4A042110781375032857
:108A80009170C2E903330CBF80234FF48073C2E9B5
:108A900001337047034A012302F58051537081F876
:108AA000E4377047982D01202DE9F041304F07EB56
:108AB000401898F854340BB9BDE8F08100EB8003FE
:108AC0000E460021044607EB4313450193F8362672
:108AD00083F8361688F83A244EF0B2FAB8BB3D4413
:108AE0002448A5F8386400EB44104EF091FA3B7826
:108AF000D5F85024A3B1D5F83C140124D2F8AC30F9
:108B00008C4003F1C001420010F4004F90B202D13A
:108B10005A6822435A600C339942F4D1BDE8F0817F
:108B2000D5F83C140124D2F8AC3001F1100203F165
:108B3000C0019440420010F4004F90B202D15A6834
:108B400022435A600C339942F4D1BDE8F0810A4BBC
:108B500093F8A02402EB420203EBC203234493F8F0
:108B60004D64002EBBD0012388F83A34B7E700BF2C
:108B700080010020B8050020101901202DE9F84FD0
:108B8000374D2B7813B90120BDE8F88F354F05F527
:108B9000876A05F634360024D7F81CB44FF6FE7900
:108BA0004FF6FF7815E0B0F5606F4AD0B081B0EBBA
:108BB00008012D4B4FF05C005A4618BF012100FB05
:108BC000043010F079FF01340AF1200A1436082C21
:108BD00031D0D5F81C2FA2422DDDDAF81800DAF8D2
:108BE0000420D0E93D014EF0EFF9484597F82924DB
:108BF00014D0542A04D1B7F82C240132A7F82C241D
:108C0000D5F83C2B404502F10102C5F83C2BCAD1F6
:108C1000D5F8382B0132C5F8382BC8E7542AD2D101
:108C2000B7F82E2401340AF1200A14360132082C38
:108C3000A7F82E24CDD10123012085F8383CBDE8CA
:108C4000F88F97F8A02402EB420207EBC2022244FD
:108C500092F84D240D2AA9D18022B277A7E700BF50
:108C60008001002010190120BC0D00202DE9F843DF
:108C700012F078F82F4E4FF0000C0746DFF8BC805A
:108C80002D4C716800294ADD00234FF486701D4683
:108C900000FB0362013392F80521994245EA02057F
:108CA000F6D145EA0C0C5FFA8CF9D8F80430C3F31E
:108CB00008038BBBEFF3118373BB4FF0E02CD4F8A8
:108CC0001C34DCF81810D4F81C249342F7D1D4F8E3
:108CD000A4249142F3D8D4F8A8C44FF47A7202FBCA
:108CE0000CF0401AB0FBFCF002FB0300C31BB3F511
:108CF000FA6FCCBF4FF0000C05F0010CBCF1000F77
:108D0000BFD1B9F1000F04D00B4B93F82924542A9A
:108D100008D04846BDE8F88311F0F6FFE6E7E146E3
:108D20000025C2E7B3F8302448460132A3F83024C6
:108D3000BDE8F883800100201019012000ED00E05B
:108D40002DE9F0411C4CD4F87C23136A002BFCD194
:108D500012F008F8DFF864804FF0E02506464FF483
:108D60007A77D8F80430C3F308030BBBEFF3118311
:108D7000F3B9D4F81C04AA69D4F81C349842F8D189
:108D8000D4F8A4349A42F4D8D4F8A81407FB01F319
:108D90009B1AB3FBF1F307FB0030831B092BE0D9CF
:108DA000D4F8843313B11A689B889361BDE8F081CD
:108DB00011F0AAFFF1E700BF1019012000ED00E05B
:108DC00010B504464DF0A2F90146204689B2BDE82F
:108DD000104069E638B50B4D00EB400005F27453C6
:108DE000C40003EBC0032C4493ED027AD3ED037A65
:108DF000E7EE007AB0EE670A4DF088F9D4F87435E2
:108E0000186038BD800100202DE9F0414EF0FCF8DB
:108E100080B31B4F7D68002D12DD3846002410F80A
:108E2000086BA046013416B1037F012B1DD04269A7
:108E3000AC4200F58670136843F001031360F1D172
:108E400011F090FFD7F8204F002C0CDD0D4B03EBF9
:108E5000C4041968083333F8042CC8689C4242EAF9
:108E60000002CA60F5D1BDE8F08180F8FC80FFF710
:108E700003F9DCE747F018F90028CAD1BDE8F08112
:108E800080010020A41000200C4AF8B51368556931
:108E90002B4003EA000555617DB1094F0126B5FA63
:108EA00085F4C4F11F0407EB840306FA04F4D3F835
:108EB000B00403689847A543F1D1F8BD003C0140D8
:108EC000101901200269C3682DE9F04712EA03096D
:108ED0002AD005460E464FF000474FF00008B9FA79
:108EE00089F327FA03F21B3BD24309EA02092A61FC
:108EF000042B16D8DFE803F03B30251A0300B36AD1
:108F0000002B3FD003F1FF3AC6F828801FFA8AFAF7
:108F1000746A34B123682046514698476468002C2F
:108F2000F8D1B9F1000FDAD1BDE8F08770680028F8
:108F3000F7D0696B036889B29847B9F1000FCED1B9
:108F4000F2E7B0680028ECD0A96B036889B29847B3
:108F5000B9F1000FC3D1E7E7F0680028E1D0E96B71
:108F6000036889B29847B9F1000FB8D1DCE73069DE
:108F70000028D6D0296C036889B29847B9F1000F50
:108F8000ADD1D1E7E96A1FFA81FAC1E7836910B56B
:108F90001A4C04EB8303D3F8100540F04DFEB4F8EF
:108FA00030350C2B0ED8DFE803F0070D0D0D220D28
:108FB0000D0D1B0D0D0D1400D4F8F024D36823F40F
:108FC0000073D3600122002384F82D2584F8323504
:108FD00010BDD4F8F024D36823F48053D360F1E7B4
:108FE000D4F8F024D36823F40063D360EAE7D4F81C
:108FF000F024D36823F48063D360E3E710190120E1
:1090000080699C3040F018BE830AA3F58013522B70
:1090100052D8F0B504466A4885B0034493F8F40387
:109020000D2847D8674D860105EB8013D3F83475BA
:10903000A7423FD00139C3F8344589B2C3F840157F
:10904000D5F82414B1FBF2F2013AC3F83825002216
:10905000C3F84425C3F83C25C3F8482593F8712587
:1090600002F0FF014AB358490223AF1901EB801106
:10907000204687F87135043141F048FB012387F819
:109080007135524B9C421BD0B4F1804F18D0A3F5E0
:109090007C439C4275D003F580639C4271D04C4A5E
:1090A00003F57C439C4218BF944249D003F57053AA
:1090B0009C4245D005B0F0BD704783F87015D2E7EB
:1090C00000234FF48051AA19CDE9001392F87015CE
:1090D0000129CDE90233EDD00221D2F83405012473
:1090E00082F871153B4987683940816082F8714583
:1090F00082F870350023AA19CDE90033029392F863
:109100007035012BD6D0D2F8343502212F4882F8A1
:10911000711583425A6899684ED000F58060834289
:109120004AD022F0700221F08001354401205A60BB
:109130009960002385F8710585F8703505B0F0BD9C
:1091400000214FF48053CDE90031AB1993F870251D
:10915000012ACDE90211ADD0D3F83405022283F8FB
:1091600071251C4A87683A4082601B4A83F8701553
:109170000121944283F87115BCD0154B9C4299D1C2
:10918000B8E700224FF48051AB19CDE9001293F8F3
:1091900070150129CDE902228CD00221D3F83405C3
:1091A000012483F871150B4987683940816083F881
:1091B000714583F870259DE722F47002B1E700BF86
:1091C0008070050810190120441E01200000014094
:1091D000000C00408800FEFF0004014010B50E4C5A
:1091E000D4F8F4383BB194F800191A68C9079B8881
:1091F00048BF1B04936145F03DFF02E05B6998475F
:1092000020B9D4F81834002BF8D1FEE7D4F81C3478
:109210000020C4F8203410BD1019012010B58CB006
:10922000114C002301220DF10701844604F55F7003
:10923000049203910D498DF82820069102A902930A
:109240008DF8143009930B9384F814C4CDE90733D7
:1092500010F01CFED4F87C23136A002BFCD19DF87F
:1092600007000CB010BD00BF10190120FD880008D8
:1092700070B5054690B008200C46FFF7CFFFFF28D9
:1092800026D0FE2802D0022010B070BD0023124E5E
:109290000220012201A98DF810308DF824300F939F
:1092A00003948DF83820CDE9073006F55F70CDE9DD
:1092B0000135CDE90533CDE90A33CDE90C3310F0A2
:1092C000E5FDD6F87C33186A0028FCD110B070BDDB
:1092D000012010B070BD00BF1019012030B591B051
:1092E00000231D4DFD200DF1030101228DF8030027
:1092F00005F55F70C5F844338DF810308DF82430D3
:109300000F9303928DF83820CDE9053101A9CDE9FD
:109310000133CDE90732CDE90A33CDE90C3310F042
:10932000B5FDD5F87C331C6A002CFCD10120FFF779
:1093300075FFFF2809D00922D5F81C34204685F88E
:109340004823C5F8383311B030BD0423022085F816
:10935000483311B030BD00BF1019012010B50446CC
:1093600092B0080E4FF0950C8DF8081000238DF880
:109370000500080C01228DF809C08DF80600080AC6
:10938000062144F0400C8DF8070001A805910390D8
:109390000DF10300174904938DF8183007930893D3
:1093A0008DF82C3011938DF804C00A9209908DF835
:1093B0004020CDE90C13CDE90E3345F02BFE80F0B3
:1093C0000103DBB203B18CB90B4C082303A904F5EC
:1093D0005F7084F8143410F059FDD4F87C23136ABC
:1093E000002BFCD19DF8030012B010BDFF2012B07D
:1093F00010BD00BFFD880008101901202DE9F041C3
:109400000546884617461E462A4C94F84803042809
:1094100039D0082807D1D4F84033AB4206D0FFF743
:109420005DFF0228F1D00120BDE8F081FC23D4F8D3
:109430007C2384F80139117B1F4BC3F82C8051B178
:10944000526942B194F80424002A0CBF4FF4807290
:109450004FF4007201E04FF480725A6317491848C4
:1094600010F014FD012206230020C4F82483C4F860
:109470002853C4F83073C4F8346384F82C2384F878
:109480004833BDE8F08194F83E3353B9690218209F
:10949000FFF764FF38B994F84833082BC6D0FE2391
:1094A000C5E72946F3E7FFF74BFCFFF7D3F90320A5
:1094B000BAE700BF101901200000012004000120BC
:1094C0008C1C012070B51C4D06460C4695F848339F
:1094D000042B09D0082B1FD1D5F84033834229D063
:1094E000FFF7FCFE022817D100213720FFF736FFD7
:1094F00021461720FFF732FFB0B995F83E336BB91C
:1095000071021920FFF72AFF70B908230220C5E96C
:10951000D06485F8483370BD012070BD31461920F4
:10952000FFF71CFF0028F0D0FFF70AFCFFF792F9C5
:10953000032070BD022070BD101901202DE9F041FB
:109540001B4C07468846164694F848C31D46BCF196
:10955000040F09D0BCF1080F02D00020BDE8F08153
:10956000FFF7BCFE0228F8D194F83E33B3B1394678
:109570001120FFF7F3FEB8B90522D4F81C340120FE
:10958000C4F82483C4F82873C4F83063C4F834538F
:1095900084F84823C4F83833BDE8F08179021120FB
:1095A000FFF7DCFE0028E7D0FFF7CAFBD5E700BFD6
:1095B000101901202DE9F043804C95B094F87463A4
:1095C000002E00F0B28194F8483304F559775A1E02
:1095D000082A00F29080DFE812F0330055003301D2
:1095E0008E007B009F001A008E00090045F012FDDE
:1095F000002840F0AB82D4F83833D4F81C24FA3376
:10960000934275D2FFF726F994F84833DFE745F027
:1096100001FD0028EFD0D4F844330022012B84F858
:109620003C2340F2B682D4F84023013B0821064691
:109630000132C4F8443384F84813C4F8402370E17D
:1096400000210846FFF78AFE0546FFF779FB012D4A
:109650004ED14FF0000840F2AB11082084F83D8352
:10966000FFF77CFE052800F0DA81012800F09981DF
:10967000FFF766FB94F83D33002B00F07082022365
:1096800084F8483394F83D3300213720022B0CBF77
:109690004FF080450D46FFF761FE29202946FFF770
:1096A0005DFE0546FFF74CFB15BB94F83D33022BDE
:1096B00000F0CD8184F83E5300210920FFF74EFED3
:1096C00000287FD0FFF73CFB94F848335A1E12E085
:1096D0004FF40071D4F82403FFF7CAFD01280546B2
:1096E00000F08181022800F08681002800F09A8134
:1096F00094F848335A1ED2B2022A00F20C81D4F8F0
:109700001C34D4F838239B1AC82B00F23F81002662
:10971000304615B0BDE8F083D4F87C23117B136A82
:10972000002900F008815269002A00F0048194F8B1
:109730000424002A00F0FF80B3FA83F35B09002BB6
:10974000D6D004AA002305A91D4805920222ADF82F
:10975000103007920DF10F0206930B9201228DF843
:10976000203009930A938DF8343013930C928DF8BE
:109770004820CDE90E33CDE9103310F087FBD4F843
:109780007C331D6A002DFCD19DF80F3003F01F03C0
:10979000052B00F0E881FFF75DF8D4F83083B8F1CD
:1097A000000F00F03981D4F834332A46D4F8281356
:1097B0000120C04794F8483309E700BF1019012081
:1097C0008C1C012010213846FFF752FD00287FF441
:1097D00079AF94F87333DB077FF574AF94F86423A3
:1097E000921100F06481012A7FF46CAF94F86B232E
:1097F0001621DFF8C8C302259200D2B2C5F10803D2
:109800008B4228BF0B46C3F108059840C91A42FA9B
:1098100005F24FF0000540EA02001CF8012FEDD1DF
:10982000431C9B02C4F84C33FFF78AFA00210A203C
:10983000FFF794FD002840F03381032384F8483378
:10984000102105A8FFF714FD00287FF451AFBDF8E3
:1098500015209DF81C3052BA9DF81410DDF81D003B
:10986000A4F850239DF8172000BA84F8521303F08F
:109870000F0184F853239DF8182084F85D1384F8B1
:1098800054239DF81920C4F8580384F855239DF8F3
:109890001A2084F856239DF81B2084F857231A09B0
:1098A0009DF8213084F85C231B019DF82220DBB257
:1098B00043EA121302F00F0203F5FA6384F86023FF
:1098C000A4F85E33FFF73CFA94F83E3353B94FF4F3
:1098D00000711020FFF742FD0546FFF731FA002D19
:1098E0007FF490AED4F82434B2499A08B1EB930FC8
:1098F0004FF0020306D252085B008A429BB201D9A4
:10990000FF2BF8D904220021A4F880331346C4F8B1
:10991000441384F84823042B18BF082B0CBF0126DE
:109920000026304615B0BDE8F083304684F8486321
:1099300015B0BDE8F083D4F8243305A994F82C239E
:109940009D4803EB02220023CDE90523CDE909332D
:10995000CDE90B330E9301238DF820308DF8343090
:109960004FF48073079310F091FAD4F87C23136AB4
:10997000002BFCD194F82C230132D2B2A2F10203C5
:1099800084F82C23B3FA83F35B09D8E6FEF762FF71
:1099900094F84863042E18BF082E0CBF0126002639
:1099A000BFE704AB8DF8340005A983480693042370
:1099B000CDF814808DF82080CDF838800793CDE95C
:1099C0000988CDE90B8810F061FAD4F87C23136A7A
:1099D000002BFCD19DF81330AB2B7FF449AE022352
:1099E00084F83D3344E6D4F83833D4F81C24643387
:1099F0009342BFF47DAEFFF7A3F9FEF72BFFD4F837
:109A000030534DB10022D4F83433D4F82813104623
:109A1000A84794F84833DAE594F84833D7E584F852
:109A20003D5325E6FFF78CF90423D4F8307384F80E
:109A30003C5384F84833002F3FF473AFD4F83433E9
:109A40002846D4F82423D4F82813B84750E62946EA
:109A50003A20FFF783FC04AB804605A90693042354
:109A600055480793012305958DF820500E958DF8E4
:109A70003430CDE90955CDE90B5510F007FAD4F88B
:109A80007C23136A002BFCD1B8F1000F08D1FFF73B
:109A900057F9049B1BBAC3F3807384F83E330BE67B
:109AA000FFF74EF9FEF7D6FE94F848338FE594F8A9
:109AB0006933012094F86D53032103F00F03DFF89D
:109AC00000E1AD0198405FFA85FC0625C5F1080369
:109AD0008B4228BF0B46C3F108059A40C91A4CFABD
:109AE00005F51EF801CF42EA05024FF00005EDD161
:109AF0000D4694F86A130232DFF8C88089014FF0EE
:109B00000C0C4FF0060EC9B2CEF108034FF0000E58
:109B1000634528BF6346C3F108099D40BCEB030CB5
:109B200041FA09F145EA010518F8011FECD16B1C57
:109B3000C1179340A3FB000203FB0122400A40EA45
:109B4000C250C4F84C03FFF7FBF86FE60190FFF733
:109B5000F7F80423019884F848330646E1E61E46E8
:109B600084F84833DDE60722D4F81C34D4F8306397
:109B700084F84823C4F83833002E3FF4D2AED4F82A
:109B800034330120D4E9C921B04794F848335A1E30
:109B9000B1E508D0042384F84833FFF7D1F894F8EE
:109BA00048335A1EA7E5FFF799FB02287FF4A0ADC2
:109BB00088E500BF40787D018C1C01207B1C0120C2
:109BC0007D1C01207A1C0120817899B10C48D0F8C5
:109BD0000439102B0FD003EB430201334FF0200C5C
:109BE0000244C0F80439012382F8081982F809C92F
:109BF00082F80A3970470521002011F0F5BB00BF3B
:109C00001019012030B490F8443000F10801484A9E
:109C1000012BC2F838196ED083684649DC68464D7E
:109C200024F46004AB42DC60DC6844F46004DC6073
:109C30009C6B24F440149C639C6B44F480149C63E0
:109C40009C6B24F4F8449C639C6B44F488449C63B0
:109C50009C6824F470249C609C689C609C6824F43C
:109C600040149C609C689C605C6824F480645C6028
:109C70005C6824F480545C605C6901EA0401596109
:109C80005969596147D0DC682A4924F0E064DC60F6
:109C9000DC6844F0E064DC609C6B24F440149C635A
:109CA0009C6B44F480149C639C6B24F478249C6328
:109CB0009C6B44F410249C639C6824F470249C6086
:109CC0009C689C609C6824F440149C609C689C6028
:109CD0005C6824F480645C605C6824F480545C609C
:109CE0009C692140144C9961A3429969996118D0EB
:109CF000002380F844301148114B848DC18D408D74
:109D0000091BC2F84049C2F83C0993FBF1F330BC8F
:109D1000C2F8443970470B4C616841F4000161603E
:109D2000B1E708494B6843F400034B60E0E700BF2C
:109D30001019012000F0FFFF00200140007AF01F01
:109D40008038010000230140704700BF014840F007
:109D500083B900BF6C220120084810B4D0F85C39E8
:109D6000D0F8904999691A682CB1234600F65C1026
:109D70005DF8044B18475DF8044B7047101901203B
:109D8000014840F069B900BFCC220120084810B456
:109D9000D0F8BC39D0F8F04999691A682CB123463B
:109DA00000F6BC105DF8044B18475DF8044B704793
:109DB00010190120014840F04FB900BF2C230120A9
:109DC000084810B4D0F81C3AD0F8504A99691A687B
:109DD0002CB1234600F61C205DF8044B18475DF8B3
:109DE000044B70471019012030B404690023416806
:109DF0004025E46882690C3154624469956053607F
:109E000093631160C2E90333C2E90533C2E9073342
:109E1000C2E90A33C2E90C3384B1C269E0689363D2
:109E200050621160C2E90133C2E90333C2E905336C
:109E3000C2E90733C2E90A33C2E90C3330BC7047C8
:109E4000114A037A0168D35C10B4CC58CA1824F0C4
:109E50000104CC501368DB07FCD4037D1F2B09D908
:109E6000203B20225DF8044B02FA03F343F0180371
:109E7000CB60704720225DF8044B02FA03F343F0F5
:109E800018038B60704700BFB4EC0508F0B5066896
:109E9000356A00295CD12F68AC68D6F818E0002F2D
:109EA0005FD0364B3B40B3F1005F61D007F01F013C
:109EB00004F11F0327F01F02194421F01F01BFF313
:109EC0004F8F00290BDD114402F12003DFF8B0C0F1
:109ED0008B42CCF868221A4603F12003F8D1BFF375
:109EE0004F8FBFF36F8F03684FF48062CEF804701A
:109EF000CEF814205B69CEF8204043B36868F66959
:109F0000002837D01D4B0340B3F1005F1AD000F09A
:109F10001F0220F01F011F32224422F01F02BFF354
:109F20004F8F002A0ADD0A4401F12003144D9A42A2
:109F3000C5F87012194603F12003F8D1BFF34F8F13
:109F4000BFF36F8F4FF48063706073613462F0BD54
:109F5000EC69002CFBD06F691435D6F818E0002F9F
:109F60009FD1084A3346CEF81470CEF80420C1E7DA
:109F70003346B9E7044B70617360E7E70000FFFF09
:109F800000ED00E00000002004000020F8B50768A4
:109F90000646D7E90454002C50D0A0612B7D1F2B1E
:109FA00039D82022286802FA03F343F018038360AB
:109FB000237D1F2B3AD92022203B02FA03F322688B
:109FC00043F01803D3606368002269680A601A606E
:109FD0001A6842F010021A60BA69297A49F0AAF99F
:109FE000FA69217A206849F0A5F92A7A2A492F6866
:109FF00033688D5C5A687B59206843F001037B51BC
:10A00000237AC95C435843F001034350536843F03B
:10A0100003035360F8BD203B2022286802FA03F3B3
:10A0200043F01803C360237D1F2BC4D8202202FAFB
:10A0300003F3226843F018039360C4E72A7D6B683A
:10A040001F2AA8611FD82021286801FA02F242F0D5
:10A05000180282600021BA691960196841F0100184
:10A060001960297A49F066F92A7A0B493368286819
:10A07000895C5A68435843F001034350536843F0E6
:10A0800002035360F8BD203A2021286801FA02F249
:10A0900042F01802C260DDE7B4EC050810B10368B5
:10A0A00082889A61704700BF18B1838802681B04D8
:10A0B0009361704708B51D2010F000FC08B183794A
:10A0C0004BB11E2010F0FAFB08B1837903B108BD33
:10A0D0005523C38008BD5523C380F2E7D3B2012BBB
:10A0E00023D802EB42024FF0000C70B54FEA820E0B
:10A0F0000F4C634622460EF1080504E00133182B8D
:10A1000011D012F81CCF6045F8D192F801C08C45EF
:10A11000F4D15659002EF1D0C3EBC3030EEB8303E9
:10A120000433E01870BD002070BD0020704700BFF0
:10A130004875050810B40C4C002304F6C82C01E047
:10A14000152B0CD003EB430201331CF802108142A3
:10A15000F6D122445DF8044B92F9CA0A70474FF0D9
:10A16000FF305DF8044B704710190120D3B2022B69
:10A1700021D802EB4202002330B54FEA820C0F4D8A
:10A180000F4C2A460CF10C0E04E00133172B10D0B3
:10A1900052F82C4FA042F8D114798C42F5D152F8E4
:10A1A0000E40002CF1D02C2202FB03C30833E81828
:10A1B00030BD002030BD0020704700BF8070050812
:10A1C00000000140002838D0002330B51B4D90F826
:10A1D00004C005F6C82401E0152B2CD003EB430284
:10A1E0000133A15C6145F7D12A44046890F805E089
:10A1F00092F9CA3ADAB2022A1DD803EB4303104897
:10A2000010494FEA830C024600230CF10C0504E0D0
:10A210000133172B0FD052F82C1F8C42F8D1117933
:10A220007145F5D151590029F2D02C2202FB03C30C
:10A230000833184430BD002030BD7047101901208C
:10A2400080700508000001400248436E0BB1543095
:10A2500018477047000001200348D0F888300BB140
:10A2600078301847704700BF000001200348D0F83D
:10A27000AC300BB19C301847704700BF0000012084
:10A280000348D0F8D0300BB1C0301847704700BF3A
:10A29000000001200348D0F8F4300BB1E430184737
:10A2A000704700BF000001200348D0F8183113B1F7
:10A2B00000F5847018477047000001200348D0F86B
:10A2C0003C3113B100F5967018477047000001202B
:10A2D0000348D0F8603113B100F5A87018477047F3
:10A2E000000001200348D0F8843113B100F5BA70A2
:10A2F00018477047000001200348D0F8A83113B177
:10A3000000F5CC7018477047000001200348D0F8D2
:10A31000CC3113B100F5DE70184770470000012002
:10A320000348D0F8F03113B100F5F07018477047CA
:10A33000000001200348D0F8143213B100F5017079
:10A3400018477047000001200348D0F8383213B195
:10A3500000F50A7018477047000001200348D0F844
:10A360005C3213B100F513701847704700000120EC
:10A370000348D0F8803213B100F51C7018477047BD
:10A38000000001200138064B064A00EBC00003EB39
:10A390008000406D90420CBF9520962046F026B973
:10A3A000000001200060024001382DE9E84100EB87
:10A3B000C000124D1E46124B05EB800590460F461D
:10A3C000686D98420CBF9520962046F00FF995F9DC
:10A3D00069004FEA98116F66EE6645F025FF95F922
:10A3E0006930002B07DB03F01F0001225B090549E0
:10A3F000824041F82320BDE8E88100BF0000012031
:10A400000060024000E100E0800AA0F580105228C0
:10A4100008D8054B184490F8F4330D2B02D8034AA2
:10A42000D05670470020704780700508A4EC0508DE
:10A4300058B183884FF00042B3FA83F332FA03F342
:10A4400003D002490A6813430B607047003C014087
:10A450000120FEF719BD00BF0220FEF715BD00BFA9
:10A460000420FEF711BD00BF0820FEF70DBD00BFA0
:10A470001020FEF709BD00BF4FF47870FEF704BD51
:10A480004FF47C40FEF700BD30B1036882881B6941
:10A490001A4214BF01200020704700BF2DE9F04F81
:10A4A000884683B004461746002800F0BC80026846
:10A4B0005E4B13449B0A5E4AC8F3411B134493F856
:10A4C000680746F093F8C8F38103B4F804E008F095
:10A4D0000302256801939EFAAEF0B0FA80F002F113
:10A4E000FF3A3EFA00F35ED00126032103E001307B
:10A4F0003EFA00F357D006FA00F313EA0E03F6D043
:10A50000D5F8009093FAA3F4B4FA84F493FAA3FC78
:10A51000BCFA8CFC6400BAF1010F4FEA4C0C01FA52
:10A5200004F402FA0CFC29EA040444EA0C042C604A
:10A5300049D9D5F80C9093FAA3F4B4FA84F493FAB9
:10A54000A3FCBCFA8CFC6400022A4FEA4C0C01FA12
:10A5500004F40BFA0CFC29EA040444EA0C04EC6051
:10A56000C5D193FAA3FCBCFA8CFC1C0ABCF1070F02
:10A5700041DC2C6A93FAA3FCBCFA8CFC93FAA3F39B
:10A580004FF00F09B3FA83F34FEA8C0C01309B00B4
:10A5900009FA0CFC07FA03F324EA0C0423432B62A8
:10A5A0003EFA00F3A7D1BAF1010F09D86B68C8F3DE
:10A5B000001823EA0E030EFB08FE4EEA03036B604D
:10A5C00003B0BDE8F08FD5F8089093FAA3F4B4FA7D
:10A5D00084F493FAA3FC6400BCFA8CFC01FA04F442
:10A5E0004FEA4C0C29EA0409019C04FA0CFC49EAE4
:10A5F0000C04AC609DE7D5F824C094FAA4F9B9FA2C
:10A6000089F994FAA4F30F24B3FA83F34FEA890982
:10A610009B0004FA09F907FA03F32CEA090C4CEA47
:10A6200003036B6263E74FF0FF3344E70000FEBFB4
:10A630008070050800B131E770472DE9F84FC04F31
:10A640006023064603FB0073D3F84849002C00F052
:10A650006B81D3F850A9BAF1000F04D09AF80630F4
:10A66000002B40F06181602303FB0673D3F854593B
:10A670001DB1AB79002B40F05781731CDBB2BAF1EE
:10A68000000F04D015228AF807308AF8062015B189
:10A690001622EB71AA714FF06009207C45F0A6FFED
:10A6A000294609FB06F9504649F074FB042207EBE2
:10A6B0000908504698F85839002B14BF3E211E2136
:10A6C000FFF7B8FF98F8583928469E4D002B4FF0F9
:10A6D00004024D4414BF3E211E21FFF7ABFF4C2264
:10A6E000002128464CF0FEFAD8F848399FED967ABA
:10A6F000B0EE084A5B68F7EE003AB8F85A994FF0A6
:10A70000000EC8F85C3940F21458904B9FED905AF7
:10A710009A68904BC2F38222134493F87027D7F8BB
:10A720002434D34007EE903AF8EE677AC7EE275A02
:10A7300007EE909A9FED887AF8EEE77AC7EE274AFF
:10A74000DFED867AB0EE007AE5EE877AA5EE875ADD
:10A7500025EE844A37EE856A74EEE72AB9F5C87F9C
:10A760000EF1010CD5BF642332234FF4967078208C
:10A7700007EE90CAD8BF4FF4167A0344C8BF4FF40F
:10A78000827AB8EEE77AD8BF414607EE903AC8BF62
:10A790004FF4FA7127EE257A01EB0A03F8EEE76A27
:10A7A00086EE873A73EE636AFCEEE67A17EE902A3D
:10A7B00007EE90AAB8EEE73A07EE903AF8EEE77A9D
:10A7C00023EE243AC3EE276A36EEC53A72EEE66A05
:10A7D000C3EE077A77EEE37AFCEEE77A17EE901A8B
:10A7E000C6EE877A77EEE37AFCEEE77A17EE903AD8
:10A7F00003F1020A0AEB010BF0EE466A07EE90BA8B
:10A80000F8EE677AE7EE276AF4EEE64AF1EE10FA20
:10A8100000F38E805FFA82FABAF10F0F00F28A809D
:10A82000323807EE900AF8EEE77A77EEC47AC7EE90
:10A83000876AFCEEE67A17EE900A5FFA80FABAF1C0
:10A840000F0F77D81FFA81FABAF1FF0F72D81FFAEB
:10A8500083FABAF1FF0F6DD812054AEA0E7302F0BF
:10A860007F620004134300F47F003D4A034302EA81
:10A8700001210B43602000FB067600272846C6F81E
:10A8800060390123C6F86479C6F86839C6F86C796E
:10A89000C6F87079C6F87879C6F87C7948F0AEFECB
:10A8A00096F89D39202BD9B21AD196F89C39012BF4
:10A8B00016D0242386F89D39D6F85C391A6822F020
:10A8C00001021A601A6822F480521A601A681A602B
:10A8D0001A6842F001021A6086F89D1986F89C7980
:10A8E000002194F9120045F09FFC94F91230A27CEB
:10A8F000002B07DB02F01F0101225B098A40194986
:10A9000041F82320002194F9110045F08DFC94F9C1
:10A910001130627C002B07DB02F01F0101225B0972
:10A920008A40104941F82320BDE8F88FE64615E734
:10A9300001315FE7BCF10F0FF8D100239AE700BFA8
:10A94000101901206C220120286B6E4E0038024045
:10A95000000016438070050800247449000070420E
:10A9600000FFFF0000E100E02DE9F047814DC0EB62
:10A97000001605EBC606D6F8083B002B00F0B880A1
:10A980000446070196F8780B45F030FE96F8783BC0
:10A99000012203F01F015B09013B8A40032B0AD807
:10A9A000DFE813F0DC000400E200D60072494B6AD5
:10A9B00023EA02024A623B1B04F1010905EBC303CF
:10A9C0005FFA89F993F80C0B0FF078FF064618B17F
:10A9D000122380F8079083713B1B05EBC30393F8A8
:10A9E0000D0B0FF06BFF824618B1132380F8079010
:10A9F00083713B1B05EBC30393F80E0B0FF05EFF57
:10AA0000804618B1142380F8079083713C1B504690
:10AA10002E2105EBC40595F8102BFFF70BFE95F8DA
:10AA2000112B0E214046FFF705FE95F80F2B2E2126
:10AA30003046FFF7FFFDD5F8083B50491A688B42B6
:10AA400022F040021A6055D04D4A934269D002F577
:10AA50008062934258D1484A116A41F40041116220
:10AA6000116A21F4004111625A6842F480525A601E
:10AA70001A68520634D443491E68D1F8A842D1F866
:10AA8000B402D1E9A525B0F5005F42EA0502D1F88C
:10AA9000A05242EA0502D1F8A45242EA0502D1F8D6
:10AAA000AC5242EA040242EA0502D1F8B05242EA4C
:10AAB0000502354D42EA000205EA060542EA0502B2
:10AAC0001A60D1F89C225D6842EA14422F4C04EAD5
:10AAD000050442EA04025A6002D1B1F8B8221A61B0
:10AAE000DA6922F40062DA611A6842F040021A6000
:10AAF000BDE8F087204A516A41F480515162516AA1
:10AB000021F480515162AFE7214A934213D11A4A8E
:10AB1000516A41F400515162516A21F4005151626D
:10AB2000A2E7154A116A41F480411162116A21F4C9
:10AB30008041116298E7174A934295D10E4A516AB3
:10AB400041F480115162516A21F4801151628BE706
:10AB500009490B6923EA02020A612CE706494B699D
:10AB600023EA02024A6126E703490B6A23EA02024A
:10AB70000A6220E71019012000380240003001402D
:10AB800000380040000001204000FFFFFBF0FFFF05
:10AB9000003401400050014008B100227EE47047BB
:10ABA000F8B5CB7813B900252846F8BD00F1100799
:10ABB0000C460646897838460EF0ECFF054600281C
:10ABC000F1D0E0780FF07AFEB06123780133DBB288
:10ABD00010B1C371222383710D21FFF7DDFFB0692E
:10ABE000FFF75CFA0D4AD2F81C34632BFBD90C48F2
:10ABF0000EF0BCFF03463846B3823CF0EDF8034646
:10AC000030B9E0781D460FF059FE0FF0B5FECBE7E6
:10AC1000306986F8D83049F0D1F9C5E7101901201C
:10AC200040420F0070B50E4CD4F81C6F002E15DD9D
:10AC300004F58764002503E0B54204F120040DD03B
:10AC4000237F0135002BF7D0E06800220028F3D0E5
:10AC5000217D2034FFF722FCB542F1D1012070BDE7
:10AC600080010020AB4B2DE9F04F91B093F8FA8CA6
:10AC7000A94B0025A94F0093A94BA3F6580ADFF86A
:10AC8000B892DFF8B8B24E46B30AA3F58013522B40
:10AC900055D8534493F8F4330D2B50D8B8F1010F25
:10ACA000FC5640F01E81012C3FD14FF0000949466F
:10ACB000204610F0A5FC10F02BFD90F800C0BCF170
:10ACC000000F18BFBCF1540F14BF4FF0010C4FF030
:10ACD000000C40F0028109F104091FFA89F9B9F169
:10ACE000100FE4D1002D00F0BA808B4A00210DE056
:10ACF000534493F8F4330D2B0FD8FB56A3420FD0D7
:10AD0000013102F58672A94280F2A580906803683D
:10AD10009B0AA3F58013522BEAD90023A342EFD15B
:10AD200043799BF805009842EAD17D4B5B4513D0EF
:10AD30005BF81C6FB30AA3F58013522BA9D9B8F1A5
:10AD4000010FF2D001230024B8F1020FADD1002B86
:10AD5000ABD0734B5B45EBD1009B013503F586739C
:10AD6000042D00938BD1DFF8D8814FF0000B08F54C
:10AD70009E77A8F5876ADAF81C3F5B4568DDD8F84E
:10AD80000C60002E64D098F81030B088D6F800908F
:10AD9000DAF8045063490193B0FA80F34944002D76
:10ADA0000293C3F11F034FEA9121009340F3CD803A
:10ADB000594B002405E0013403F58673AC4200F0E2
:10ADC000C1801A688A42F6D14FF48673524A03FB57
:10ADD0000424009A0BF1010B019B5100C8F80420D8
:10ADE00088F810300323C8F80C6003FA01F5C8F89E
:10ADF0001840B371012386F807B01646A26C03FA17
:10AE000001F12A43A264226D0A4322659AF80020C8
:10AE1000002A6BD003FA06F11A46636D0B4389B220
:10AE20006365C9F81800D4F8AC00FDF751F9204665
:10AE300008F12008FDF720F90123BBF1080F07F105
:10AE4000180708F8043C08F8033C07F8073C92D1BF
:10AE500011B0BDE8F08FBCF1000F7FF466AF58462B
:10AE6000FDF7CEF89BF80540C3B2022B00F24B83EE
:10AE7000431C2D4A5BB203EB430398002B4B03F5B5
:10AE8000727104E0994200F03E8353F82C2FB242D5
:10AE9000F8D11A79A242F5D11A58002AF2D0944674
:10AEA0000023234A51680133614513D0102B02F16E
:10AEB0002402F7D14FF0FF3303EBC3031D4A02EB2B
:10AEC000830393F87030002B7FF42FAF009BC3F8FF
:10AED00008B041E7DBB2013BEEE7002D7FF405AFA0
:10AEE00023E7B4F1080318BF01232DE702990004FA
:10AEF000C1F12F05009903FA01F1AB40656D89B2EC
:10AF00002B436365C9F81800D4F8AC00FDF7E0F8EE
:10AF10008DE700BF1019012088010020A4EC05086E
:10AF2000D87805080000FEBF0000014080700508C9
:10AF3000540001200000012000040140F8770508BA
:10AF4000B8050020032C00F398824FF4867303FBAE
:10AF500005A31869002800F0C08299600131CAB2C7
:10AF600083F811210492542283F810216B1C02688B
:10AF7000CAF8043044790392FDF742F8A04B8646A4
:10AF800093F8113D0593C3B2022B00F2BC8200F18D
:10AF9000010C9C499C4800234FFA8CFC039A0CEB53
:10AFA0004C0C4FEA8C0C05E00133172B00F0AB8200
:10AFB00051F82C0F9042F7D10879A042F4D151F802
:10AFC0000C000028F0D02C210EEB4E0E002401FBCB
:10AFD00003F303EB8E0E8B4B734419694FF48673A6
:10AFE00003FB05A3C3E90701884B9C46DCF804106A
:10AFF000884217D001340CF1240C102CF6D1844B6C
:10B0000093F84C20002A00F06182824B82488349E9
:10B01000834AC3F84804C3F84014C3F8502411B05D
:10B02000BDE8F08F611C7A48C9B2013901EBC1015A
:10B0300000EB810191F8700006900028E5D104989A
:10B040004FF08C0C81F871004FF4867000FB05F412
:10B050002046542481F870400446811071480394BE
:10B06000544400FB01F1C4F800C101FB0CF001EBFA
:10B070004101C4F80C9001EB011C6B4901EB40004D
:10B08000A1F54C7101EB8C01C4F8FC00C4F8B410BC
:10B090003321C4F8B8106549039C0C195849D1F8FC
:10B0A00024940599062900F00D820729604861491A
:10B0B000DFF888E10CBF84468C465F4908BF7146C3
:10B0C00010460593039BB9FBF1F1B9FBFCFC4A1E4A
:10B0D0004FF486790CF1FF3192B209FB05A9A9F86A
:10B0E000BC1003F15801A9F87420504B22660022CD
:10B0F0001944A4F858206266E26547F0B3FFD9F816
:10B10000103018680493026842F0800202605A7995
:10B11000059B0C2A08D8DFE802F06B0707076407D5
:10B1200007075C07070754004FF4867202FB05A26D
:10B1300051694FF0600C02684FF000094FF0020EA9
:10B14000CDF820C04FF4807C22F00102CDF8289089
:10B15000CDF838C04FF0010CCDF83490CDF824C0B4
:10B160004FF00A0CCDF83C900593CDE90BCE026070
:10B1700008AA47F035FE4FF48672049B02FB05A235
:10B1800019685269059B012A5AD0042A58D0102AFE
:10B1900000F0A881402A53D0B2F5807F00F0A5814D
:10B1A000B2F5806F00F0A181B2F5805F00F0A3815D
:10B1B000B2F5803F4FF03C090CBF08224FF400620B
:10B1C0003FE04FF486724FF4805102FB05A25161BB
:10B1D000AFE74FF486724FF4807102FB05A2516114
:10B1E000A7E74FF48672102102FB05A25161A0E788
:10B1F0004FF48672012102FB05A2516199E700BF5D
:10B200001019012080700508000001405400012041
:10B210000000012078120020F57A0108F17A010877
:10B22000FD7A01086B4CA407081A00208801002051
:10B230001055220044950800D0DD060040771B0021
:10B24000082201F1180050F809C042EA0C0240F847
:10B250000920049A1079002840F01B814FF4867170
:10B26000002201FB05A1D1F810C0C869DCF800C0BC
:10B27000DCF8001041F00101CCF8001059680132EF
:10B28000884200F00281102A03F12403F6D14FF026
:10B29000FF339E4A03EBC30302EB8303586D9C4BC1
:10B2A00098420CBF9520962045F0A0F94FF4867384
:10B2B00003FB05A31A6953790C2B00F2E38095492F
:10B2C00001EB4303B3F874C84FF4867310689249D6
:10B2D00003FB05A3A3F818C0002306E0904200F08A
:10B2E00008810133042B00F00B8151F83320002A30
:10B2F000F4D1DAF8202F0132CAF8202F0AEBC3026A
:10B30000DB00C2F8240F1944069823469022B1F8B6
:10B3100004E0DFF818924CEA0E0CA1F804C07F4953
:10B32000FFF742F84FF486734FF4403C402103FB93
:10B3300005A50023E869026842F010020260026875
:10B3400042F014020260C4F8A830C4E91F33C4E913
:10B35000283304232A6AC4F898C04FF4804CC4F8F8
:10B360009C304FF48063A167C4F88430C4F8942003
:10B37000D5F8B820C4F89020C2B220F0FF00103AEF
:10B38000A9FB0231EA68039B1832090922674FF4CE
:10B390008052C4F8882003F17002614B1A44D5F83A
:10B3A000B430C4F88CC0636747F0C4FFE869039BFE
:10B3B0004FF40031D0F800E04FF4006C03F1B80214
:10B3C000574BC4F820E0D0F814E01A440023C4F826
:10B3D00024E0D0F804E0C4F828E0D0F808E0C4F88D
:10B3E0002CE0D0F80CE0C4F8C830C4F830E0C4F861
:10B3F000F030C4E93033C4E93A332B6A03930423B1
:10B40000C4F8E4304FF48063C4F8CC30039BC4E943
:10B410003731D5F80031C4F8D830C3B220F0FF007E
:10B42000103BA9FB0331EB68C4F8D0C01033090905
:10B43000C4F8B830D5F8FC3003934FF48043C4F817
:10B44000D430039BC4F8BC3047F074FFEB69B0887C
:10B450001A68D6F8009062635A69A2635A68E26378
:10B460009A682264DA6862641A6842F010021A600C
:10B470001A6842F014021A60ABE40323294A82F8E6
:10B48000103DC2E54FF0000C1EE7D3B20693013B1E
:10B49000FFE6079305910FF011FA05998146079B86
:10B4A00058B105930221049BDA79FEF7F7FF049B5C
:10B4B0005422A9F806201968059B4A6C42F4004200
:10B4C0004A64CBE6DFF868C01749F9E504995422CD
:10B4D00083F84D1083F84C2097E50223114A82F837
:10B4E000103D92E54FF40062ABE608224FF00409EC
:10B4F000A7E6DB0007E74FF400624FF00409A0E67F
:10B5000000239B88FFDE00235B68FFDE0000012034
:10B510000060024080700508A41000201D81000812
:10B520008801002010190120A0BB0D00ABAAAAAA17
:10B53000882A11002DE9F84F704E0022704B054605
:10B54000D6F8144D5968013224338C4200F0B08093
:10B55000102AF7D100246B4B9D4205D048339D4201
:10B5600002D00020BDE8F88F04F1FF39664F09EBE7
:10B57000C9034FEAC90807EB830393F87020002A38
:10B58000EFD14FF0170BA3F870B0002CE9D0DFF823
:10B5900090A10120DAF8243043F40063CAF8243083
:10B5A0000FF0C6FEDAF82430012023F40063CAF855
:10B5B00024300FF0BDFEA6F866BEDAF8443043F43E
:10B5C0000063CAF84430DAF8303043F48003CAF834
:10B5D0003030DAF8303043F00C03CAF8303096F8E7
:10B5E0001A3D002B66D10C220E214848A6F886BED3
:10B5F000A6F8B6BEFEF752FF0C220E214448FEF715
:10B600004DFF0C220E214348FEF748FF424BDA68FB
:10B61000C6F8145DC2F30222C2F10701131D04290A
:10B6200028BF0421062B4FF0FF338CBF033A0022C2
:10B630008B403A49DB4303F001039340384A1B0136
:10B64000DBB281F831334FF400334B60136B43F4BA
:10B650008003136300232B60324BAB6003F59B33F5
:10B6600003F5EC739D4244D02F4B4FF47412DA6013
:10B67000C8442E4B07EB8807786D98420CBF952085
:10B6800096202B4B2B6007236B6144F0AFFFD6F85D
:10B69000142D1C4B20469A424FF000034FF001023C
:10B6A0000CBF24492449FEF77FFE0120BDE8F88F36
:10B6B000D4B250E70C220E211448A6F86EBEA6F8AC
:10B6C00076BEA6F87EBEA6F886BEA6F8B6BEFEF783
:10B6D000E5FE0C220E211948FEF7E0FE0C220E2199
:10B6E0001748FEF7DBFE0C220E211648FEF7D6FEA9
:10B6F00082E74FF0746243F8502CB9E7101901202B
:10B7000054000120586402400000012070270120ED
:10B7100090270120C027012000ED00E000E100E0BB
:10B7200000380240802C014000640240006002406A
:10B730006054A3084DC2000815C3000878270120F3
:10B740008027012088270120F8B590F8B2311C0924
:10B75000013C052C0FD81B4E054603F00F0306EBEA
:10B760004402B2F8900840FA03F2D20703D595F8E4
:10B77000BD71012F01D00120F8BD07FA03F3344455
:10B78000013B184049F0C8FC94F89C2813180E4A55
:10B7900002EBC30152F833208B8810691840EBD0BC
:10B7A000002395F8B3210846022185F8BD31FEF744
:10B7B00075FED5F820213846136843F0080313605E
:10B7C000F8BD00BF807005083026012070B50379F0
:10B7D0008AB0344C002B14BF0122002284F8742359
:10B7E00003D184F848330AB070BD04F55F7605468E
:10B7F00090F9001030460EF0CDF9AD78002D44D10F
:10B8000001232949294A84F88833D4F82434C4F818
:10B810001024B1EB930FC4F884534FEA93024FF016
:10B82000020306D252085B008A429BB201D9FF2B69
:10B83000F8D94FF47A70A4F880330FF079FDD4F87A
:10B84000843313B11A689B889361194DEC460FCD70
:10B85000ACE80F000FCDACE80F0095E803008CE8D2
:10B860000300694630460EF011FBD4F87C23136ABE
:10B87000002BFCD1D4F81C14012284F83C33C4F80A
:10B88000381384F848230AB070BD28460FF016F824
:10B8900005460028B4D01E2300220D21C380FEF7E8
:10B8A000FDFDADE710190120801A0600341C0120AF
:10B8B000247905082DE9F04F00228DB02F21804614
:10B8C0000FF07EFFC8B1974E05464379D0F800903F
:10B8D000A6F83035FEF776FC78B144686CB1924F2B
:10B8E00000233A465168013324328C4210D0102B89
:10B8F000F8D18E4B93F84C201AB100200DB0BDE862
:10B90000F08F2F21104683F84D2083F84C10F5E777
:10B91000DBB2864A013B03EBC30302EB830393F8DC
:10B9200070A0BAF1000FE8D18268C6F8F0940192D5
:10B930002F22A3F87020D6F824347D4A934280F059
:10B94000D38052461B0A7B49C6F8F4240020A1FB91
:10B950000331794BDFF808B20A09C6F80005090976
:10B96000C6F8F804A3FB0232C6F8FC1452082BF800
:10B97000D62C52002BF8D82C96F82D2502F0FF017A
:10B98000002A00F0BD80022248466C4986F82D2529
:10B990003EF0BCFE0122404686F82D250EF08EFFBB
:10B9A0004BF8D40C28B12F21C1804E21EA79FEF743
:10B9B00075FD634A0021019B4FF4806C4BF8C41C59
:10B9C0004BF8B41C4BF8AC1C4BE934434BE9291140
:10B9D000106B40F400101063106B00F40010039023
:10B9E0000398106B40F480001063126B02F4800225
:10B9F0000492049A40224BF8C82C4FF480524BE931
:10BA000030C24FF480424BF8B82C4FF400324BF860
:10BA1000B02C03224BF8A82C96F830250C2A72D8AB
:10BA2000484901EB4202B2F8CC88C14608F1080847
:10BA3000454A464906EB88034BF8981CC3F8F024A6
:10BA40003B4600225968013224338C4261D0102ACF
:10BA5000F8D14FF0FF3202EBC202344B03EB820B02
:10BA60003B4BDBF8540098420CBF9520962044F0E5
:10BA7000BDFD00237A6801332437944246D0102B51
:10BA8000F8D106EB880850464B4660223149FEF754
:10BA90008BFCD8F8F0043DF0E9FF00287FF42DAFCF
:10BAA00060210A90AB79059159000B90DB0006905C
:10BAB00001F00201099003F00803B6F8302523488D
:10BAC000CDE9071305A944F06DF900287FF415AFFF
:10BAD000AB79B6F830159B071C481DD53EF0A2FE89
:10BAE000B0FA80F0400909E71B4A1C491A44A1FB3F
:10BAF0000212920D013A92B2511CB3FBF1F321E70D
:10BB000086F82C153FE7894688468FE75FFA83FA67
:10BB1000B7E7D2B2013A9EE73EF0C8FDB0FA80F036
:10BB20004009EBE61019012054000120000001201B
:10BB3000006CDC02598B4F01ABAAAAAA041E01209B
:10BB4000003802408070050838290120001E0120BD
:10BB5000006002408D8F000800366E01819F5E16E6
:10BB6000082A0120014B43F820107047502800405C
:10BB70001D4B1E48196C1E4A41F0805130B41964A7
:10BB800082B0196CFF2401F0805101910199016884
:10BB900041F480710160CA20196C41F4806119641C
:10BBA000196C01F4806100915321009D5462506230
:10BBB00051625B6FDB000DD40E4B00210E4A43F83F
:10BBC000041B9342FBD10D4B0D4AC3F8502802B021
:10BBD00030BC7047094A0A4BD2F850289A42EBD140
:10BBE00002B030BC704700BF003802400070004017
:10BBF00000280040542800406C28004000200040ED
:10BC0000316665422DE9F0470646086888B00C4663
:10BC10004FEA902CBDF84080ACF5801C9DF8449014
:10BC2000BCF1520F64D8374FBC449CF8F4530D2D2F
:10BC30005ED81946FDF7E8F9334A2368617902EBCB
:10BC4000851A94F806E0B9F1000F54D1F4469B0A26
:10BC5000A3F58013522B23D83B4493F8F4030D280B
:10BC60001ED84FEA4C034FF480774FEACC0CCDF846
:10BC7000088003F0020302EB80100A4601A9039337
:10BC80000CF008030493602301934FF40073CDE993
:10BC900006730023059344F085F8617994F806E073
:10BCA0001EF0020F504629D03EF0BCFD174BA801F4
:10BCB000022203EB8515D5F8341585F87125144A51
:10BCC0008D682A40062A06D0B2F5803F03D00A6864
:10BCD00042F001020A600344012283F871252168C1
:10BCE000637901F1340271600021D0183060D150C5
:10BCF00008B0BDE8F0878EF0010CA8E73EF0D6FC56
:10BD0000D4E700BF80700508441E012010190120EF
:10BD100007000100F0B50446D0F89400434B83B00F
:10BD2000A16804F1640204F118070E68C1B220F0A2
:10BD3000FF0001921039A3FB0131090947F044FBD0
:10BD4000616D0023019A012984F8583018D0042924
:10BD500016D0102955D0402912D0B1F5807F53D08C
:10BD6000B1F5806F50D0B1F5805F55D0B1F5803F0F
:10BD70004FF03C030CBF6FF0080C6FF4006C01E057
:10BD80006FF0080C06F118053046E95801EA0C017D
:10BD9000E950616D47F024F8636D012B16D0042B38
:10BDA00014D0102B0FD0402B10D0B3F5807F2FD0A4
:10BDB000B3F5806F2CD0B3F5805F31D0B3F5803F01
:10BDC00006F1540502D04FF4006100E008212B6811
:10BDD0003A46D4F894000B4340212B602162C1B253
:10BDE000124B20F0FF001039A3FB0131090947F085
:10BDF000A1FAD4F89420136843F01003136003B041
:10BE0000F0BD6FF4006CBDE76FF0080C0423B9E7D8
:10BE100006F11C050821DAE76FF4006C0423B1E792
:10BE200006F11C054FF40061D1E700BFABAAAAAA36
:10BE30002DE9F04FDFF85CB29BF800402DED028B4E
:10BE400087B034B90124204607B0BDEC028BBDE8B1
:10BE5000F08F8B4BDFF840A2D3F81C3408EE103A79
:10BE60000EF080FF9AF8243C0390002B00F0018133
:10BE70000BF234670BF634330BF63C4400263D4698
:10BE800001930597DAF81C34039AD31A03D4EA6DA8
:10BE90009A4200F3D08006EB86030BEB431393F832
:10BEA0008C3603F0FF020292002B00F08D80D5F853
:10BEB0009410AB6873481A68CBB221F0FF01103BB5
:10BEC000A0FB030370481B09C35C19444B68A98994
:10BED0001FFA83FCD368CCF1160C23EA0103BCF1F2
:10BEE000070FD36070D9DBF83C3B002201210133FE
:10BEF00096468946CBF83C3BD5F89C301F460493C8
:10BF000057F8048B40461CE0D7F80080BEF1140FB0
:10BF1000A8EB000340461CDC13F1080848BF03F1FE
:10BF200017084FEA28130EEB281E03F1FF380131E2
:10BF300002FA03F3043709FA08F28C4542EA0302D5
:10BF400007D38C45E0D8CEF1150338684FF0150EB5
:10BF5000EBE7BEF1150F65D14C49C2F38423C2F360
:10BF6000441001EB830301EB8000D3F8E838D0F8EC
:10BF7000E8081B0243EA001302F01F00C2F3C432B8
:10BF800001EB800001EB8202D0F8E818D2F8E82833
:10BF90000B4343EA023383EA132282EA121202F0CD
:10BFA0000F020F2A3ED1C3F30F134FF6FF729342D5
:10BFB00038D0B3F5606F45D0019A9381029918EE9D
:10BFC000102A20460DF078FD019B284601365C348E
:10BFD0001433A0350193FFF79DFE9AF8243CB34239
:10BFE0003FF750AF0122059F8BF8382C0022CAF88A
:10BFF0001C24002B3FF426AF03EB830307EB431312
:10C000003A7CA03757F84C0C12F0020F57F8982CD6
:10C0100011680A6A14BF42EA80020243BB420A6204
:10C02000EED10FE7DBF8383B0133CBF8383BCEB12C
:10C0300000230293C2E70024204607B0BDEC028B28
:10C04000BDE8F08F0E4991F8A02402EB420201EB0B
:10C05000C202324492F84D240D2AADD18023019AB8
:10C060009377ABE70499582209484AF0C7FD029636
:10C07000A4E70122CAF81C348BF8382CE3E600BF91
:10C0800010190120ABAAAAAAB4EC05088070050813
:10C09000600D002080010020781200204A1C4FF41F
:10C0A000003310B408BF4FF0800C4C4C18BF4FF059
:10C0B000450C00E0FBB1626B013B12EA0C0FF9D0BA
:10C0C000002923DD626B52071CD403291ED0434A8A
:10C0D000536B13F0010320D1022908D01369DBB29E
:10C0E00083421ED1012953692BD006291BD0002081
:10C0F0005DF8044B7047002904DD636B5C0701D4D5
:10C100000329E4D103205DF8044B7047002B5DF850
:10C11000044B14BF00200320704701205DF8044B3E
:10C1200070471020EFE713F4604F02D12C4A42F819
:10C13000703C990431D45A04F3D41B04D7D50F2092
:10C14000E1E7284818400028DDD0002B29DB5C00FF
:10C1500025D4980029D4D90025D41A0129D45C010A
:10C1600025D4D8012FD41902E9D45A02D9D49C027B
:10C1700027D4D8022FD419030FD45A0329D49C03EF
:10C1800025D4D80321D4190419D45A0415D49C04F5
:10C1900011D41807ABD51A20B5E71320B3E709204F
:10C1A000B1E71C20AFE70B20ADE70A20ABE70D207D
:10C1B000A9E70C20A7E71920A5E71820A3E7172077
:10C1C000A1E711209FE70E209DE716209BE7152091
:10C1D00099E7142097E7122095E700BF002C014053
:10C1E000082A012008E0FFFDF8B5164DD5F8BC324D
:10C1F000A3B1D5F8C4120446012915D0124B40F260
:10C20000FF500021DA6A22F00802DA629863C5F86A
:10C21000BC12236823F001032360F8BD0A4AD36BE4
:10C2200043F48073D363F8BD074E40F2FF570023F9
:10C230000C20B763B36040F24C43F360FFF72EFF6E
:10C24000B763DBE710190120002C01402F4B1A685F
:10C25000910102D59A6D52074BD42C4B1A685002AB
:10C2600002D5DA6E11063CD4284B1A68D20102D5E9
:10C270009A6D90072DD4254B1A68510102D59A6DFD
:10C28000120717D4214B1A68120112D59A6DD006E5
:10C290000FD59A6D510334D49A6DD20503D49A6D9B
:10C2A00022F010029A65194B4FF0006218489A600C
:10C2B0009AE770479A6D500307D49A6DD10503D45D
:10C2C0009A6D22F008029A65104B4FF080629A60D6
:10C2D000D8E79A6D4FF0807122F002029A6599605A
:10C2E000C9E7DA6E4FF4800122F08002DA669960C5
:10C2F000BAE79A6D4FF0007122F004029A659960D6
:10C30000ABE74FF000629A60704700BF00640240E4
:10C3100058640240384B5A68110303D5D3F8A02063
:10C3200052075BD4344B5A68D00303D5D3F8B420FA
:10C33000110649D4304B5A68520303D5D3F8A020D4
:10C34000900737D42C4B5A68D10203D5D3F8A020DC
:10C3500012071CD4284B5A68920217D5D3F8A02094
:10C36000D00613D5D3F8A020510341D4D3F8A02090
:10C37000D20505D4D3F8A02022F01002C3F8A020E3
:10C380001D4B4FF400121D48DA602DE77047D3F8BB
:10C39000A02050030AD4D3F8A020D10505D4D3F8A7
:10C3A000A02022F00802C3F8A020134B4FF4801203
:10C3B000DA60CFE7D3F8A0204FF4802122F0020208
:10C3C000C3F8A020D960BDE7D3F8B4204FF4803182
:10C3D00022F08002C3F8B420D960ABE7D3F8A020E4
:10C3E0004FF4002122F00402C3F8A020D96099E79D
:10C3F0004FF40012DA60704700640240A06402400B
:10C40000554B93F82033022B00F295802DE9F04133
:10C41000524D82B06B6913F0007303D00E2002B04E
:10C42000BDE8F081CDE9003340F2FF564FF48A6356
:10C4300008270446AE630121AF601020EB60FFF7D0
:10C440002DFEAE630028EAD1DFF81C8140F277436D
:10C45000AE63012158F8702C3720AA60EB60FFF71B
:10C460001DFEAE630028DAD13D4A40F2734301213C
:10C470006A62AF62EA6A42F03302EA62AE63A860BF
:10C480003320EB60FFF70AFEAE630028C7D1694690
:10C4900040F22A4201E09F0251D46B6B13426B6B56
:10C4A000F9D01E0750D46B6B98074FD46B6B99066D
:10C4B0004ED46B6B9B024DD4B4F5006F009B08BF4C
:10C4C0004FF480221BBA18BF4FF480321A4234D086
:10C4D000224D40F2FF5658F8702C40F27743AE637D
:10C4E0000121AA603720EB60FFF7D8FDAE6300287A
:10C4F00095D1B4F5006F40F24643AE634FF00101B1
:10C5000008BF0220A8600620EB60FFF7C7FDAE63FE
:10C51000002884D16B6803F400639C423FF47FAF32
:10C52000104A6B68134023436B606B6803F400632D
:10C53000A342F6D173E72820704726206FE7D5F88D
:10C54000803041F8043BA8E7042068E7022066E752
:10C55000062064E7222062E710190120002C014028
:10C5600000E1F5050081FFFF082A01200E4A0121A4
:10C570000D2052F8702C38B50C4C40F2FF5540F2AB
:10C580004D43A563A260E360FFF788FDA56340B952
:10C590006069C0F34320A0F10400B0FA80F04009C4
:10C5A00038BD002038BD00BF082A0120002C014002
:10C5B000A34A0220A34B516C41F400612DE9F043E2
:10C5C000516483B0526C03259F4C02F400620192C7
:10C5D000019A6268134043F076036360636823F452
:10C5E0008073636025600EF0A3FE636840F2FF5025
:10C5F000002143F480734FF4806263604FF4003392
:10C60000A063A160E26001E0002B60D0626B013B9F
:10C610001706F9D5002B5AD040F2FF554FF4D572CA
:10C620004FF489630721A5630820A563A260E36036
:10C63000FFF734FDA563002842D04FF00009824F78
:10C6400040F2774340F2FF58002201213720C7F81B
:10C650003880BA60FB60FFF721FDC7F838800346D9
:10C6600050BB7A4D0446064649EA050510E0C7F876
:10C670003880BD60FA60FFF711FD4FF6FE72034689
:10C68000C7F83880C0B97B69002B29DB944227D8D2
:10C6900040F27743C7F838800121BE603720FB6045
:10C6A000FFF7FCFC034640F26942032129200134D4
:10C6B000C7F83880002BDAD0184603B0BDE8F08305
:10C6C000634B01224FF0804983F82023B7E703230F
:10C6D0005D4A40F2FF511846916303B0BDE8F08314
:10C6E0004FF6FF72944200F0A4805E002DD4564BAA
:10C6F0001B68980731D0564C94F82003042831D198
:10C70000FBF738FE03460028D6D1524A40F2474391
:10C710004D4D40F2FF5652F8702C0121AE630720B8
:10C72000AA60EB60FFF7BAFCAE63464A6B681A403A
:10C7300003466A600028BFD194F81A3D0BB14FF44C
:10C74000006003B0BDE8F0435AE6414C02203E4B86
:10C7500084F820031B689D0704D12623184603B0E4
:10C76000BDE8F083384940F2FF5200238A6340F26B
:10C77000C2428B604FF40033CA6000E023B14A6BC1
:10C78000013B12F0450FF9D02F4A536B5B0752D48F
:10C79000536BD90748D440F2FF5301289363536980
:10C7A000C4F8A4329369C4F8A832D369C4F8AC328F
:10C7B000136AC4F8B03201D9062832D1224D40F2B2
:10C7C000434340F2FF56002206210320AE63AA60D5
:10C7D000EB60FFF763FCAE63034600287FF46CAFA9
:10C7E0001C4A40F2C943184D40F2FF5652F8702CD3
:10C7F0000221AE630920AA60EB60FFF74FFCAE6335
:10C80000034600287FF458AF6B69C4F89432AB69D3
:10C81000C4F89832EB69C4F89C322B6AC4F8A03291
:10C820006EE70228CAD0DBE740F2FF510123916393
:10C8300042E71B2340E740F2FF51032391633BE7AC
:10C84000003802400081FFFF002C014000001080F2
:10C8500010190120082A012038B52E4C14F86B0C51
:10C860000EF02CF828B11F210022C1802021FDF7F5
:10C8700015FE294DD5F8F4383BB195F800191A6822
:10C88000C9079B8848BF1B04936195F91B2DD3B240
:10C89000012B17D8214B4FF00C0C082003F5217108
:10C8A0001CFB020C99420DD013F81C2F032AF9D15E
:10C8B0005A78002AF6D153F80C000028F2D0FEF77F
:10C8C00039FE08B9012038BDD5F8783343B11A686C
:10C8D0009B881269134095F8752372B9002BF1D02B
:10C8E00014F8673C63B10E4B93F8BC020028E9D101
:10C8F000D5F81C34C5F8203438BD002BE2D1EFE761
:10C90000012304F8673CFFF753FE054B83F8BC0294
:10C91000ECE700BF082A012010190120487505081E
:10C920000000012008B51A4B13F8672C82B1194B8F
:10C9300093F8BC0258B1184A92F83C330133DBB289
:10C94000072B82F83C330CD9002382F8483308BD0A
:10C95000012203F8672CFFF72BFE0E4B83F8BC0275
:10C96000E8E7D2F8783343B1186892F875139B88DA
:10C970000069034049B1002BE6D1D2F81C14012311
:10C98000C2F8381382F8483308BD002BDCD0F4E736
:10C99000082A0120000001201019012010B5037998
:10C9A0003F4C002B14BF0123002384F8743303D1C0
:10C9B000002384F8483310BD94F91B2DD3B2012B0A
:10C9C000F6D8384B4FF00C0C082003F521711CFBF6
:10C9D000020C9942ECD013F81C2F032AF9D15A7893
:10C9E000002AF6D153F80C000028F2D02E49134645
:10C9F0004A682431904208D00133102BF8D100232B
:10CA000084F8153484F8483310BD94F8192D013397
:10CA1000003A84F8153418BF012284F81624FEF772
:10CA200089FDD4F8783393B1196894F875239B88FD
:10CA300009690B40E2B9003B18BF01233BB994F8E8
:10CA40003C2384F84833531C84F83C3310BD174B07
:10CA500013F8672C82B1164B93F8BC02A8B194F876
:10CA60003C330022013384F8482384F83C3310BD62
:10CA7000B3FA83F35B09E1E7012203F8672CFFF7C0
:10CA800097FD0B4B83F8BC02E8E7D4F81C24012384
:10CA900084F83C03C4F8382384F8483310BD00BF41
:10CAA000101901204875050854000120082A0120AA
:10CAB00000000120184A01210D2052F8702C38B5D1
:10CAC000164C40F2FF5540F24D43A563A260E3606F
:10CAD000FFF7E4FAA56320B96369C3F34323042B8A
:10CAE00002D04FF0FF3038BD0D4BD3F8780300284B
:10CAF000F9D001688288096993F875330A402BB12F
:10CB0000002A0CBF00204FF0FF3038BD002A14BFB0
:10CB100000204FF0FF3038BD082A0120002C0140D2
:10CB200010190120F8B51B4E1046D6F878433CB1D9
:10CB30002568A2882C69224096F875432CB332BB35
:10CB40000A46002143F072F808BBD6F8BC32002B2D
:10CB5000FBD1114F40F2FF55104C57F8702C40F2AA
:10CB60004D43A5630121A2600D20E360FFF796FA13
:10CB7000A5630028F1D16369C3F34323042BECD1EF
:10CB8000D6F81C34C6F82034F8BD002AD8D14FF0AE
:10CB9000FF30F8BD10190120082A0120002C0140A7
:10CBA000F8B51B4E1046D6F878433CB12568A288EC
:10CBB0002C69224096F875432CB332BB0A460021FB
:10CBC00042F0CEFF08BBD6F8C032002BFBD1114F8C
:10CBD00040F2FF55104C57F8702C40F24D43A563BE
:10CBE0000121A2600D20E360FFF758FAA563002839
:10CBF000F1D16369C3F34323042BECD1D6F81C3481
:10CC0000C6F82034F8BD002AD8D14FF0FF30F8BD67
:10CC100010190120082A0120002C014070B5174D81
:10CC2000002295F81634C5F8442313BB144B53F86F
:10CC3000702C40F2FF56134C40F24D4301210D2061
:10CC4000A663A260E360FFF729FAA66320B96369CF
:10CC5000C3F34323042B08D00922D5F81C34002049
:10CC600085F84823C5F8383370BD022085F848336D
:10CC700070BD034B43F8642CD9E700BF10190120A5
:10CC8000082A0120002C0140F8B58F4C94F8745309
:10CC9000002D00F0FD8094F848230226531E082B37
:10CCA0003DD8DFE803F03335A23C684B163C050065
:10CCB000FFF75CFC002840F0FC80D4F83833D4F84F
:10CCC0001C24FA33934227D2FFF72CFE94F8482312
:10CCD000E4E7FFF74BFC0028EFD0D4F84433002200
:10CCE000012B84F83C2340F2E880D4F84013013B48
:10CCF0000131C4E9D01394F8163413B1734B43F8DF
:10CD0000642C0823054684F8483315E084F848630A
:10CD1000FFF72CFC002849D194F84823531EDBB2BE
:10CD2000022B00F2AD80D4F81C34D4F838239B1ABF
:10CD3000C82B00F2B18000252846F8BDD4F8C032D7
:10CD4000002BF8D10722D4F81C34D4F8305384F8DF
:10CD50004823C4F83833002DEED0D4F83433012002
:10CD6000D4E9C921A847D7E7D4F83833D4F81C242C
:10CD700064339342DFD2D4F8BC72002FF4D1FFF7B2
:10CD8000F5FB0028A2D00423D4F8305384F83C7378
:10CD900084F84833002D00F08A80D4F834333846C4
:10CDA000D4F82423D4F82813A847B5E7FBF7E2FA10
:10CDB0000028B1D194F82033002BA3F10203B3FA79
:10CDC00083F314BF022201225B0984F83D2384F817
:10CDD0003E33FBF7CFFA00287FF476AFD4F8102368
:10CDE0000323C4F84C2384F84833FBF7C3FA002824
:10CDF00092D194F8F4520422B4F8F612D4F8F8322E
:10CE0000C4F84403A4F85013180ED4F8F812D4F858
:10CE1000F832090C84F853031B0A84F8525384F83F
:10CE2000541384F85533D4F8F81294F8FC0294F8AB
:10CE3000FD3284F85613D34094F8FD1284F857035A
:10CE400084F85C3301F00F01D4F80033B4F8060322
:10CE5000C4F85833B4F8063384F85D13C3F30B13E6
:10CE6000B4F8061384F8482343EA102301F00F01B5
:10CE700003F00F0384F8601303F5FA63A4F85E333C
:10CE8000082A18BF042A0CBF012500252846F8BD32
:10CE9000284684F84853F8BDFFF744FD94F84853FA
:10CEA000082D18BF042D0CBF0125002544E70546B9
:10CEB00042E7042384F848333EE7FAD1FFF7AEFE99
:10CEC00094F84823531E2AE710190120082A01204C
:10CED0002DE9F047054682B00E4690461F463A4C73
:10CEE00094F8480304280DD0082807D1D4F840331B
:10CEF000AB4207D0FFF792FE0228F1D0012002B02A
:10CF0000BDE8F087DFF8C89059F8643CC3F34F21BF
:10CF10005A0A0F29C4E9C9652DD8D4F844A3BAF137
:10CF2000000F28D094F8160428B3B3F5005F42D060
:10CF3000264831464FF400720193184449F05EFED2
:10CF4000019B03F50073C3F34F215A0A49F8643C6F
:10CF5000102930D0BAF1010F2DD0D4F840230AF1B6
:10CF6000FF33042102200132C4F8443384F848130B
:10CF7000C4F84023C3E70123062128460125324691
:10CF800084F848130021C4F83083C4F8347384F85B
:10CF90002C5342F0E5FD0028B1D0FFF7C3FCD4F8D4
:10CFA000306376B12846D4F834330022D4F82813FD
:10CFB000B0470320A3E792B20B46044E013AAD1AE4
:10CFC000DAE703209BE700BF10190120EC450120A0
:10CFD000082A012070B50E4D04460E4695F84833D8
:10CFE000042B0BD0082B07D1D5F8403383420CD04B
:10CFF000FFF714FE022801D0012070BD0823022093
:10D00000C5E9D04685F8483370BD022070BD00BF29
:10D01000101901202DE9F0411C4C054688461746A1
:10D0200094F848031E46042808D0082802D000209F
:10D03000BDE8F081FFF7F2FD0228F8D10123424656
:10D040002846002142F0F2FD68B1FFF76BFCD4F8EE
:10D050003053002DEBD00022D4F83433D4F8281309
:10D060001046A847E3E70522D4F81C340120C4F891
:10D070002483C4F82853C4F83073C4F8346384F8A4
:10D080004823C4F83833BDE8F08100BF10190120EF
:10D0900070B52F4C636BD9051DD54FF4807240F2EB
:10D0A000FF562C4BA263A663E26B2B4D1340E36348
:10D0B000D5F8C4329A0721D401220023C5F8B4223E
:10D0C000C5F8B832224B40F2FF51224A9963D96B1E
:10D0D0000A40DA6370BD636B980704D51E4B0222C9
:10D0E000C3F8B822EEE7636B190723D4636B9A0683
:10D0F00025D5194B0622C3F8B822E3E7D5F8142D3D
:10D10000136823F0010313600022E36A23F008038D
:10D11000E362C5F8C022D5F8C432DB07CCD540F2B3
:10D120004C43A6630121A2600C20E360FEF7B6FF2A
:10D13000A663C1E7084B0422C3F8B822C2E7636BB9
:10D14000DB06BFD5044B0522C3F8B822BAE700BFFF
:10D15000002C0140C53EFFFF10190120D0F820111E
:10D16000242200232DE9F041C0F8942104460A68E6
:10D17000806804F5907522F001020A600B604B6034
:10D180008B6094F805C0C4F89C314FEA8C22C4F837
:10D19000943184F8903102F48052C4F89831C4F884
:10D1A0003831C4F828214FEA0C32C4F8403102F477
:10D1B0000052C4F834312379C4F82C214FEA0C22F0
:10D1C000C4F8240113F0010002F48062C4F8302195
:10D1D00002D00422C4F8342113F0020305D0D4F89D
:10D1E000342142F00802C4F834211CF0010F0DD0A4
:10D1F00048B1D4F8442142F00202C4F844214FF46B
:10D200008032C4F84C21002B40F0FF80A84B03F182
:10D21000200053F8042F944200F0BD809842F8D1CA
:10D220001CF0080F40F0CD80D4F89431002B00F0B2
:10D23000168124232846C4F894310B6823F0010397
:10D240000B603DF013FB012815D0D4F84431002BBE
:10D2500040F01881D4F8203128465A6822F49042D0
:10D260005A609A6822F02A029A601A6842F0010213
:10D270001A6046F097F92379DA0761D5D4F8FC20D3
:10D28000002A00F0D9800023D4F8041104F13C06F0
:10D29000E263A3644FF480623046E264C4E9101391
:10D2A000C4E91433C4E91833C4E91A334FF48033A2
:10D2B000E3654FF48073A36546F0EEF930463CF029
:10D2C000D5FBD4F89881C4F88C61B8F1200F65675C
:10D2D00031D1E368626999B26AB3B1FA81F77F0923
:10D2E00049B394F89001012825D030460126C4F8AE
:10D2F0009C710B4684F890612226A4F87811C4F83A
:10D3000098616C4ED4F82011A6676B4E2431C4F896
:10D310007421E667694EC4F88C70C4F888603CF0EC
:10D3200043FC002800F0B280102384F89071C4F808
:10D330009C31C4F89481E26B23795268C4F81421BB
:10D340009B0777D5D4F80021002A69D00023D4F8B0
:10D35000081104F19C06C4F89C20C4F8A8304022AF
:10D36000C4F8B8303046C4E92C33C4E93033C4E9DA
:10D3700032334FF48033C4F8BC304FF48063C4E9D7
:10D380002812C4F8AC3046F087F930463CF06EFB0A
:10D39000002867D0FEE7002C3FF442AF94F8BC3180
:10D3A000002B3FF43DAFD4F844311CF0080F43F09C
:10D3B0000803C4F844314FF40043C4F854313FF437
:10D3C00033AFD4F89431002B55D024232846C4F829
:10D3D00094310B6823F001030B603DF047FA0128FC
:10D3E0003FF449AFD4F84431002B47D1D4F8203171
:10D3F00028465A6822F490425A609A6822F0220223
:10D400009A609A6842F008022EE7D4F8443143F05B
:10D410000103C4F844314FF40033C4F84831F5E651
:10D42000D4F8A0311A6842F080021A601A6842F0FB
:10D4300040021A60BDE8F081D4F8A021116841F4DF
:10D4400080711160916841F001019160116841F0B3
:10D4500020011160116841F01001116070E784F83B
:10D460009031E6E6D4F89C30C4F88861C4F8D45012
:10D470005860BDE8F08184F89031A6E728463DF079
:10D48000AFFBB3E728463DF0ABFBE3E6D4F8203131
:10D4900084F890011A6842F480721A609A6842F027
:10D4A00001029A609A6842F040029A6043E700BF26
:10D4B000A01E0020F95B0408295C04082D5C040808
:10D4C000F8B5EFF31185502383F31288D0F80031BB
:10D4D0001B6813F0010303D0EDB285F31188F8BD8A
:10D4E000D0F894210446D0F898110A4302F02102A2
:10D4F000212AF1D0D0E90901884253D043D82269CA
:10D500001846531A9BB2D4F894710022A062202FBF
:10D5100084F8A421E0D1A2695118DDD0B3FA83F6D2
:10D520007609002BD8D094F89021012AD4D001227A
:10D53000D4F88801A4F8723184F890212122C4F82B
:10D540009C61C4F86C11A4F87031C4F89421E8B15E
:10D55000DFF858C0D4F82021C0F83CC0DFF850C034
:10D5600028320665C0F840C0DFF848C0C0F84CC09B
:10D570003CF01AFB50B1102384F89061C4F89C3140
:10D58000C4F89471A8E7431A9BB2BCE7D4F82031E1
:10D5900000224021196284F890219A6842F08002AA
:10D5A0009A6099E7012384F8A43195E7D15B0408D8
:10D5B000F55B04082D5C040870B5D0F820410546E1
:10D5C000E369990614D5606AEB6AC0B2002B74D087
:10D5D000296B9847D5F82041236823F48073236092
:10D5E000A36823F00103A360A36943F00803A361C8
:10D5F000E369DA0701D501232362E3699B0701D5BB
:10D6000002232362E3695E0701D504232362E369F1
:10D61000180701D508232362E369590614D540236E
:10D62000236295F8BD61002E31D0D5F80031CBB121
:10D630002846FFF745FF95F8A4311BB195F8BD6169
:10D64000002E4BD0D5F82041D5F8003163B1E36905
:10D65000DB0606D56B6B13B19847D5F82041102334
:10D66000236270BDD5F82041E3691A06EFD5D5E9EC
:10D67000092393422DD0AA69D25C0133D2B2A262AF
:10D680002A69B3FBF2F102FB1133AB62DFE795F8D5
:10D69000B2010DF013F9236823F00803236001237E
:10D6A00085F8BD310028C0D032462021FCF7F6FEB7
:10D6B000D5F80031002BBBD1D4E7EB696A69D054AF
:10D6C000EB69EA680133B3FBF2F102FB1133EB6162
:10D6D00080E7236823F080032360B8E795F8B20160
:10D6E0000DF0ECF8D5F820410122236823F008035F
:10D6F000236085F8BD210028A6D032462021FCF702
:10D70000CDFE9FE72DE9F04FAE4C83B004EB8004D3
:10D71000D4F82C4C002C6BD0D4F8AC511F46DFF859
:10D72000C0B290466B680646A74AC4F8A0316B6B3E
:10D73000DFF8B09263612B6BA160A3616B8FE36034
:10D740002B8FC4F8A82123610BF6681323602A7875
:10D7500009EB420313F9600C53000193C3B2012B90
:10D7600040F28680D4F8003183B1984900209C466D
:10D770004B68013024319C4500F0F6801028F7D129
:10D78000934B93F84C10002900F05081D4F8FC0022
:10D79000002840F0C2806B68C4F8203195F828005A
:10D7A000002840F0D28094F8B2010DF087F80221F1
:10D7B0003A07034694F8B09184F8BD111CD558B3CC
:10D7C00017F0510F4FF00B0206F1010614BF0A21AA
:10D7D0001A2117F0410FC671827114BF4023202314
:10D7E00094F8B3211943FCF759FED4F8FC3043B345
:10D7F000204603B0BDE8F08F18F0020F0CD058B1EE
:10D800000B223B06827106F10102C27100F1158103
:10D8100094F8B321FCF742FE48460DF04FF800287B
:10D82000E3D018F0010FE0D00C2201360221C671BE
:10D83000827194F8B121FCF731FED4F8FC30002B52
:10D84000D6D195F82C1095F92A00890942F0ECFC04
:10D8500095F92A3095F82A20002BC9DB02F01F0227
:10D8600001215B095B4801FA02F240F82320BFE77F
:10D8700008234FF00C0A0BF5996C1AFB003A0023B1
:10D88000E64619460131182962D01EF81C3F042BC8
:10D89000F8D19EF801309342F4D15EF80A30002BA3
:10D8A000F0D08E460199C4F800318944CEEBCE0108
:10D8B00019F95FEC890000EB4009BEF1FF3F01EB75
:10D8C00089015944D1F8D414C4F808113FF44DAF7C
:10D8D0000021013118293FF447AF1CF81CEFBEF1BD
:10D8E000050FF6D19CF801E09645F2D15CF80AE00C
:10D8F000BEF1000FEDD0C1EBC101C4F8FCE000EBBC
:10D900004000890001EB80008344DBF8D414C4F8A4
:10D910000411002B7FF429AF70462C4A0023516874
:10D920000133243281425FD0102BF8D1284B93F879
:10D930004C20002A7FF42FAF2A78013283F84D2043
:10D940000C2283F84C206B6826E742F04FFE2AE752
:10D95000019B9944D4F8003119F95F1C0131B7D10A
:10D96000002B7FF402AF11E75FFA80F9184B013208
:10D9700009F1FF31D2B201EBC10103EB810393F84E
:10D98000701000297FF402AF83F8712012485A6D9D
:10D9900082420CBF952096200B2283F8702042F023
:10D9A00025FE2346484695F82B200C49FCF7FCFC45
:10D9B0006B68D4F8FC002833C4F8183100283FF411
:10D9C000EAAEAAE77812002049B700085400012007
:10D9D0000000012000E100E000600240019000082A
:10D9E00080700508082A0120DBB2174A013B03EBCF
:10D9F000C30302EB83032A7893F870100132D2B28A
:10DA000000297FF4C8AE586D83F871200F4A904208
:10DA10000CBF952096200C2283F8702042F0E6FD82
:10DA20006B6803F12402C4F81C21B5E6013283F8C7
:10DA30004D200B2283F84C20A8E60123204684F8D1
:10DA4000BD31FDF781FEE7E60000012000600240E5
:10DA5000BFF34F8F0549064BCA6802F4E0621343D7
:10DA6000CB60BFF34F8F00BFFDE700BF00ED00E0CC
:10DA70000400FA0508B572B6FFF7EAFF30B583B0C7
:10DA8000FEF776F8334BDB68012B4BD0324C002588
:10DA9000324A0523C4F89850C4F89C50C4F8A0201A
:10DAA000C4F89430BFF34F8FBFF36F8F4FF6FF0171
:10DAB000E2682B4B0A4013432A4AE360536F3CF061
:10DAC0005BFB294B2949A3FB0023D4F8FC209B0CCA
:10DAD00042F08072C4F8FC20C1F8A834D1F8243494
:10DAE0002349244AA1FB031323499B09C2F8B01F11
:10DAF0005560013B1168B3F1807F41F00101116075
:10DB000008D24FF0E022F0215361072384F823105C
:10DB1000956113614FF0E022136943F00403136130
:10DB200003B030BD02210320FEF71CF80D4B134853
:10DB30005A6C134942F480425A645B6C03F480438C
:10DB40000193019A02680B68026083F308884B68AE
:10DB50009847FEE75028004000ED00E01B0000065B
:10DB60000005FA050038024083DE1B43101901202E
:10DB7000D34D6210001000E055CEACC50038014016
:10DB80000000F01F800AA0F5801052281CD80F4B0F
:10DB9000184490F8F4330D2B16D8013910B40C4CFE
:10DBA00004EB831CD4F824448BB2DCF834050CF568
:10DBB000A761CCF84035B4FBF2F2013A5DF8044BB2
:10DBC000CCF838253CF0A2BD704700BF8070050836
:10DBD0001019012070B504460068830AA3F580136C
:10DBE000522B05D82E4E334493F8F4530D2D00D903
:10DBF00070BDFBF709FA2B4BA801022203EB851538
:10DC0000D5F8341585F87125274A8D682A40062AEB
:10DC100006D0B2F5803F03D00A6842F001020A60E4
:10DC2000034401202168214A83F87105002320481C
:10DC300001E050F8332091420AD001330E2BF8D185
:10DC40000121002042F0F0FA1A4B01221A6070BD47
:10DC500006EBC303012193F99D4993F89D69204682
:10DC600042F0E2FA002CC3DB06F01F030121640935
:10DC7000104D01FA03F31B2E45F8243008D02E2E48
:10DC8000B6D12C2042F0D0FA4FF480536B6070BDB7
:10DC9000192042F0C9FA4FF000732B6070BD00BF2D
:10DCA00080700508101901200700010000000140E4
:10DCB000187A050800E100E003689B0AA3F58013C9
:10DCC000522B56D870B53B4C234493F8F4C3BCF1A7
:10DCD0000D0F4DD84079850800294ED00CEB8C03F0
:10DCE0004FF0020E840834480CEB43030EFA04F4A0
:10DCF0002B4400EB8C15D5F8345500EB830EEE6801
:10DD0000CEF804103443CEF81420EC604FEA8C14A3
:10DD1000EFF3118E502383F312882C2303FB0CF3B3
:10DD2000C258C11832B3131D4A622C22234D02FB84
:10DD30000CF215441432024452F8041B19B1196054
:10DD400052F8043C04339542F6D100225FFA8EFE6D
:10DD50001A608EF311882C2303FB0C0C2044DCF892
:10DD60002430D0F8342503B3D36843F00103D360E3
:10DD700070BD704724330344D7E70CEB8C030E4887
:10DD80002C460CEB43032B4400EB8C15D5F8346583
:10DD90000225A540F46824EA0504F46000EB83043E
:10DDA000616062614FEA8C14B2E7D36823F001032B
:10DDB000D36070BD8070050810190120341901204E
:10DDC00003689B0AA3F58013522B00D97047144AAD
:10DDD000134493F8F4330D2BF8D810B4114C79B9DF
:10DDE0004179022204EB83105DF8044B21FA02F31F
:10DDF000D0F834159A40CB6823EA0203CB60704711
:10DE00004179022204EB83105DF8044B21FA02F3FE
:10DE1000D0F8341502FA03F3CA681343CB60704795
:10DE2000807005081019012003689B0AA3F5801370
:10DE3000522B10D8084A134493F8F4230D2A0AD819
:10DE4000407902230549D84001EB82128340D2F881
:10DE50003425DB43136170478070050810190120D9
:10DE600001490248FBF72EB81019012000000140BB
:10DE700010B5064C06482146FBF724F804F5C67198
:10DE80000448BDE81040FBF71DB800BF1019012081
:10DE9000000001400044014002494FF08040FBF780
:10DEA00011B800BF3C19012001490248FBF70AB82C
:10DEB000681901200004004001490248FBF702B83C
:10DEC000941901200008004001490248FAF7FABFFE
:10DED000C0190120000C00402DE9F843194E3569A6
:10DEE000F3681D4010D04FF00047DFF85C80B5FAB2
:10DEF00085F227FA02F31F2A6FEA030305EA0305F6
:10DF0000336103D0002DF2D1BDE8F883D8F8043195
:10DF1000A3B103F1FF3900231FFA89F9C8F80431CE
:10DF2000D8F80041002CEDD0236820464946984798
:10DF30006468002CF8D1002DD9D1E5E7F16A1FFA09
:10DF400081F9EDE700100040101901200149024855
:10DF5000FAF7B8BF441A01200004014010B5064C7E
:10DF6000064804F59A71FAF7ADFF04F50471044808
:10DF7000BDE81040FAF7A6BF1019012000040140C7
:10DF8000001C004001490248FAF79CBF701A0120AA
:10DF90000040014001490248FAF794BFC81A012025
:10DFA0000048014001490248FAF78CBFF41A0120E9
:10DFB000001800402DE9F0414FF425728EB0002189
:10DFC000664848F08FFE664B664E4FF080415A6CB3
:10DFD00006F68805374642F00102DFF89081A6F187
:10DFE0008C045A645A6C02F001020092009A1A6C76
:10DFF00042F001021A641A6C02F001020192019AC5
:10E000001A6C42F002021A641A6C02F002020292C6
:10E01000029A1A6C42F004021A641A6C02F00402AA
:10E020000392039A1A6C42F008021A641A6C02F006
:10E0300008020492049A1A6C42F010021A641A6CD4
:10E0400002F010020592059A1A6C42F020021A643E
:10E050001A6C02F020020692069A5A6C42F00202F2
:10E060005A645A6C02F002020792079A5A6C42F400
:10E0700080325A645A6C02F480320892089A5A6CC0
:10E0800042F400325A645A6C02F400320992099A3E
:10E090005A6C42F480225A645A6C02F480220A922A
:10E0A0000A9A1A6C42F040021A641A6C02F040029A
:10E0B0000B920B9A1A6C42F080021A641A6C02F0EE
:10E0C00080020C920C9A1A6C42F480721A641B6CD7
:10E0D00003F480730D930D9B4246002301E054F836
:10E0E000332091420BD001330E2BF8D11C37002086
:10E0F00042F07CFAAF420CD057F81C1CECE71A4AED
:10E100001C3702EBC30393F89C0942F06FFAAF424D
:10E11000F2D14FF08041154F154C3A46002301E0F3
:10E1200054F8332091420BD001330E2BF8D11C361A
:10E13000002042F05BFAAE420CD056F81C1CECE713
:10E14000094A1C3602EBC30393F89C0942F04EFACD
:10E15000AE42F2D10EB0BDE8F08100BF101901202F
:10E1600000380240A47A05088070050800000140CC
:10E17000187A0508800AA0F5801052280ED8084B9E
:10E18000184490F8F4230D2A08D8064B03EB8213A9
:10E19000D3F83425136843F001031360704700BFC0
:10E1A000807005081019012038B5254C14F8483C3A
:10E1B000012B12D1042894BF002301236BB904EB77
:10E1C00040000D4614F8301C44F81C3C34F82E2C4A
:10E1D00030F8263C34F82A0C01B138BD07EE902AFD
:10E1E00064229FED180AB8EEE77ADFED177A02FB9A
:10E1F00003F327EE277A54ED0E7AF8EE676A07EEFE
:10E20000903A02FB0033B8EEE76A07EE903A66EE0A
:10E21000806AF8EEE77A27EE067A87EE270A20EE84
:10E22000260A47F073FF54F8402C084B106034F86E
:10E230002C1CD3F81C341944294444F8181C38BD4C
:10E24000082A0120CA269B3E0AD7233C1019012028
:10E25000F0B5A44CA5B0E368022B00F04082A248C0
:10E26000A24AA349121A48F0C9FCA248A24AA349EB
:10E27000121A48F0C3FCA368012B00F2C48003EB20
:10E2800043039F4A9F4D02EB430032F8132041881D
:10E290008388C5E9B021C5F8C8329B4C9B4E9C4B86
:10E2A000B2FBF1F29B4901FB02F20021C6F82424E3
:10E2B000D4F8882042F47002C4F888201A6842F02A
:10E2C00001021A609960944A1868024093481A60E3
:10E2D000C0F30807924A5A601A6822F480221A6032
:10E2E000D96007B1FEE78F49A0604FF6FF000A68CA
:10E2F0008D4B42F400720A60E26802401343E3600F
:10E3000043F0CAFABFF34F8FBFF36F8FC4F8507258
:10E31000BFF34F8FBFF36F8F636943F400336361C3
:10E32000BFF34F8FBFF36F8FC4F88470BFF34F8F6D
:10E33000D4F8803043F6E07CC3F3C90EC3F34E3308
:10E34000580100EA0C01734641EA8372013B5F1CED
:10E35000C4F86022F8D1203810F1200FF1D1BFF3BA
:10E360004F8F636943F480336361BFF34F8FBFF313
:10E370006F8F6C49664B0A6842F480720A60196CB0
:10E380006A4A41F080511964196C01F08051029180
:10E390000299116841F4404111601268D5F8C00239
:10E3A00002F44042D5F8C412D5F8C8720192019A1D
:10E3B0009A6802F00C02042A00F090809A6802F039
:10E3C0000C02082A00F08680514A594C136843F425
:10E3D0008033136054F814CC05E054F8143CA3EBDC
:10E3E0000C03642B75D813689B03F6D5484A9368D1
:10E3F00003F00C03082B6CD0136823F080731360B8
:10E4000054F814CC09E03F4DD5E9B02145E754F864
:10E41000143CA3EB0C03022B5BD813689B01F6D4CE
:10E4200049083B06013943EA801343EA0143414965
:10E4300019435160136843F080731360344B54F8F0
:10E44000141C04E054F8142C521A022A41D81A68F9
:10E450009701F7D51A6C42F080521A641B6C334A4C
:10E4600003F080530393039B136843F480331360DA
:10E4700054F8141C06E054F8143C5B1AB3F57A7F88
:10E4800000F2CE805368D803F5D51368274943F4CA
:10E490000033136054F8142C06E054F8143C9B1A13
:10E4A000B3F57A7F00F2BC804B689B03F5D54FF43F
:10E4B00000134FF4C07E04A804934FF0006321932F
:10E4C0000723CDE908E303230A933BF089FE98B3C1
:10E4D000FEE7FEE75B685A027FF576AF0C4B144C03
:10E4E0001B6883E75028004000000000283E000021
:10E4F000347A06080000002080010020A1DC060814
:10E50000108305080000012000ED00E01019012033
:10E510000038024040420F00FFFFF6FE00000008F6
:10E5200010300024003C02400003FA050070004057
:10E53000082A0120080040206C4A136803F00F03EA
:10E54000062B0AD8136823F00F0343F00703136068
:10E55000136803F00F03072B63D1654B9A6842F4ED
:10E56000E0529A609A6842F460429A609A6822F097
:10E57000F0029A601A68900153D59A6841F2883087
:10E5800022F0030242F002029A6054F8141C04E0E4
:10E5900054F8142C521A824243D89A6802F00C02A2
:10E5A000082AF5D1514A136819070AD5136823F0D0
:10E5B0000F0343F007031360136803F00F03072BE7
:10E5C0002FD14B4C4B4FA36823F4E05343F4A0539B
:10E5D000A360A36823F4604343F40043A3603BF0CB
:10E5E000CBFDA368C3F303133B4493F8A431D84095
:10E5F000C6F8240443F050F9002304A8CDE91333EE
:10E60000CDE91533CDE91733CDE91933CDE91B3306
:10E61000CDE91D33384B04933BF0E2FD10B1FEE72A
:10E62000FEE7FEE702234FF0007204A8CDE90633AF
:10E63000D823CDE9042301230B933BF0D1FD00B196
:10E64000FEE7D4F88C3023F08073C4F88C30D4F813
:10E650008C3043F08073C4F88C30A36803F00C0353
:10E66000042B36D0082B18D0244BC6F82434204A6B
:10E67000D5E9B031B3FBF1F39168D6F82424C1F3A6
:10E6800003110F4497F8A411CA401D4901FB03F37D
:10E69000C6F82424934220D0FEE76368626813F42E
:10E6A000800F636802F03F0218BF1649C3F3881356
:10E6B00008BF1249B1FBF2F202FB03F30C4A5268A5
:10E6C000C2F3014201325200B3FBF2F3C6F8243424
:10E6D000CDE70C4BC6F82434C9E725B0F0BD0021C6
:10E6E0000320FDF73FFAFFF7B3F900BF003C0240FB
:10E6F0000038024078810508C0FF03000024F400C0
:10E7000040420F0000127A000A4B93F8CC0218B96D
:10E71000094B13F8100C7047084AD1680329F7D148
:10E7200005494FF0010C01F810CC0021D16083F8AD
:10E73000CC12704700000120082A01205028004018
:10E740000021032008B5FDF70DFA72B6FFF780F936
:10E750002C4C54F80C2C14F8060C08B552B1116866
:10E76000938809690B40002845D1003B18BF01235D
:10E77000002BF3D1142000250CF0DAFD224900BF54
:10E7800054F80C3C63B1186814F8062C9B88006997
:10E79000034062BB003B18BF01230BB1FFF7D0FF62
:10E7A000D1F81C24D1F82034D31A322B11D854F8C4
:10E7B000043C9342E3D2D1F8F43833B118689B8813
:10E7C0004669334218BF1B048361323244F8042C7B
:10E7D000D5E7D1F8F4383BB191F800091A68C007C1
:10E7E0009B8848BF1B04936144F8045CC7E7B3FAF5
:10E7F00083F35B09D1E7B3FA83F35B09002BADD157
:10E80000B8E700BF082A01201019012070B51C20AC
:10E810000CF054F804461121FCF7BEF9002C56D038
:10E82000A388C82022681B0493610CF081FD204658
:10E83000FBF734FC1B200CF041F808B12923C380FE
:10E840002923E3802B4CD4F88C3213B10023C4F875
:10E850008C320023284E01252370C4F8886284F886
:10E86000745243F06BF894F8B13206F11C02022B9B
:10E87000C4F88C2201D0284670BD14F8683CAB4225
:10E8800033D0022BF7D15436C4F8A462D4F8A802CE
:10E8900090F8BC33012B14D00168D1F8043823F070
:10E8A0000203C1F8043854F8142C54F8143C9B1A91
:10E8B000032BFAD98B68002243F001038B6080F8A8
:10E8C000BC2300230D4A184682F8233070BDC820AF
:10E8D0000CF02EFD2046FBF7E1FB1B200BF0EEFFBA
:10E8E0000028AFD02923C380ACE77436C4F8A462F3
:10E8F000CCE700BF082A0120D002012000ED00E093
:10E900000A4AD2F8783373B11968988892F8753347
:10E910000A6910401BB1B0FA80F040097047003816
:10E9200018BF012070470120704700BF1019012057
:10E93000024BD3F818341B6A184700BF1019012086
:10E94000034BD3F8180408B183691847704700BF18
:10E95000101901200378022B12D00F494368026975
:10E96000D1F84808023A184010B4400AD1F840489B
:10E97000D1F83C1804FB02005DF8044B08447047D2
:10E98000054B4268D3F83418D3F8300800EB410047
:10E9900000EB5220704700BF983D01202DE9F04F59
:10E9A00083B002F0020E019310B9BEF1000F50D1F6
:10E9B0008D4DD5F83878B7BB4FF0FF3C8B4C002617
:10E9C0008B4FE146E046E2462368984200F0CF8054
:10E9D00094F80EB0BBF1000F4BD0BBF1010F15D175
:10E9E00006F5B17B07EB0B1B9BF807B01BF0010F83
:10E9F0000CD11BF07E0F09D15FEADB1340F0C5801C
:10EA0000D4F808B0D34501D2DA46B1460136103405
:10EA10000B2ED9D1BCF1FF3F36D1B8F1FF3F2ED03C
:10EA2000C446734C31E0D5F84068D5F83C4806FB45
:10EA30000744A042C0D395F8E43713B9012385F801
:10EA4000E43700266A4B012230465A7003B0BDE815
:10EA5000F08F654D95F8E437A5F5805413B901237F
:10EA600085F8E437012302266370304603B0BDE821
:10EA7000F08FB446013610340B2EA5D1CAE7B9F198
:10EA8000FF3F00F08980CC46594CD5F8C86604EBAE
:10EA90000C1841F218690CF5B177013648F80900F5
:10EAA00041F21C69C5F8C86648F809604FEA0718C2
:10EAB00044F8086004EB07164FF00008C6F804801D
:10EAC00004EB0716B679042E00F28780DFE806F023
:10EAD000031B641B330012F001086DD104EB071017
:10EAE000019B4FEAE20990F807A0032B69F3C71ACC
:10EAF00080F807A05ED94FF6FF70834228BF034617
:10EB000004EB07108380042E15D0BEF1000F12D045
:10EB1000D5F8C836D5F8CC0601330130C5F8C8366B
:10EB2000C5F8CC0604EB0C1041F21C65435104EB14
:10EB3000071304209871500705D504EB0710C3791B
:10EB400043F00103C371D30608D504EB0714E3793E
:10EB5000C3F34502013262F34603E3710126254BFC
:10EB6000304603EB4C230B6003B0BDE8F08F06F595
:10EB7000B1771F4C04EB071C4FEA07189CF806C03E
:10EB8000BCF1000F0DD1B4467FE7B046013610341A
:10EB90000B2E7FF419AF3DE70026304603B0BDE8E9
:10EBA000F08FB446D5F8C866013644F80860C5F859
:10EBB000C86685E74346A3E70F4B0E49D3F81834E0
:10EBC00001EB4C210D4A9D680023A8470028E3D0A3
:10EBD00004EB07140223A37147E795F8E437002BF1
:10EBE0003FF43DAF3EE700BF983D0120B043012018
:10EBF000982D0120B02D01201019012071890008E5
:10EC000070B5114E82B00D463378022B16D1020A30
:10EC1000C4B20E4B01A9D3F83008002310440322DC
:10EC2000FFF7BCFE012807D13378022B019B0CBFF4
:10EC300023F8145043F8245002B070BDC0F3D4122E
:10EC400000F07F04E5E700BF982D0120983D0120EA
:10EC50002DE9F04FDFF82081012885B00C4698F8A7
:10EC600000608CBF002301231546032E01930B681F
:10EC70003DD0022E63D14FEA13294FF4807ADFB2E0
:10EC80000138012820D84FF0010B9D4217D9394E89
:10EC9000D6F8A8271AB1D6F8C417994252D0D6F898
:10ECA00030080023092203A94844FFF777FE012812
:10ECB00026D0022817D020B123689D42E8D803202F
:10ECC000256005B0BDE8F08FC7B12A4B93F8E42763
:10ECD00012B9012283F8E4270123022088F80130C9
:10ECE00005B0BDE8F08F022005B0BDE8F08F4FF011
:10ECF000800AC3F3D41903F07F07C1E7D346C4E702
:10ED000098F800200399DDF804C0022A14D0032AE1
:10ED1000E9D151F8273023F07043B3FA83F35F440D
:10ED20005B096345236821D05B4457452360ECD3DE
:10ED300009F101090027C0E731F81730EDE74FF47A
:10ED4000807AD6E7D6F84018013A02EB4122490210
:10ED5000B2FBF1F21344B3FBFBF20BFB12320AB12C
:10ED60005B449B1A9D42236092D8A8E7AB42A8D38C
:10ED7000A5E700BF983D0120982D01202DE9F04F17
:10ED8000DFF860B18946174683B09BF80010D9F8C8
:10ED90000020022940F088800BF58053D6B2D3F8CA
:10EDA0003058A6EB02084FF4807305EB1225B844E7
:10EDB0009844BA4208F1FF38B8FBF3F847D200F0A4
:10EDC000010AA844032907EB0604A8EB0503A4EBFA
:10EDD00002040CBF80224FF48072944228BF144674
:10EDE0000EB9944237D20B2201A92846FFF7D6FD6F
:10EDF000012802D003B0BDE8F08F9BF80010D9F8CD
:10EE00000020022902F1010327D0B44210D96FF08B
:10EE100040420198324400EB8202043800EB840047
:10EE200042F8043F824203F10103F9D1D9F80020EE
:10EE3000A61B32449742C9F8002002D1BAF1000F54
:10EE400044D1974205F101054FF00006BAD80120E0
:10EE500003B0BDE8F08F0A22C6E7B44210D96FF0C4
:10EE6000004CDDF804E0B4440EEB4C0CAEF1020EA5
:10EE70000EEB440E2CF8023FE64503F10103F9D1F5
:10EE8000921B22449742C9F80020DAD1BAF1000F50
:10EE9000D7D06FF00043019A4FF6FF71234422F858
:10EEA000131003B0BDE8F08F02F07F060BF580531E
:10EEB0000329C2F3D415D3F83038A6EB02081D4459
:10EEC000B84414BF4FF48073802371E76FF0404360
:10EED000019A4FF0FF30234442F82300D9F8002074
:10EEE000AFE700BF982D012030B50446C06983B05C
:10EEF00010B9012003B030BD0D460023032201A943
:10EF0000FFF74CFD0128F5D1B4F92030002B0ADAC7
:10EF1000144B93F8E4270AB983F8E407124B012253
:10EF200002205A70E6E7019A012D4FEA431102EBE5
:10EF3000431303D0022D11D1E5255554A268DA619F
:10EF40002278032A04D100221A775A779A77DA773F
:10EF5000626A110C5A83998203B030BDE268DA61AB
:10EF6000EEE700BF983D0120982D01202DE9F041EA
:10EF7000002990F83C3082B0044614BF02210021E1
:10EF8000042B76D8DFE803F0030C3D486400FFF75C
:10EF9000ABFF01286BD1626B002A70D184F83C0072
:10EFA0003D4E4FF6F777DFF8F88006F5805516E00E
:10EFB000BA424AD83FF0FEFF01284FF000011DD1B0
:10EFC000206BFFF71DFE012818D1019AD5F84438AF
:10EFD000511E22638B4228BF0B46C5F84438327855
:10EFE00001A9236B032A18469AB2E1D143452CD8D4
:10EFF0003FF0E0FF01284FF00001E1D002B0BDE892
:10F00000F081426B04F130010020FFF7B7FE0128C8
:10F010002DD1032384F83C302048E26AD0F8C4376D
:10F0200000F5F460D0F8A0109B1A4262C26801FBA0
:10F0300003F3816801EB4325002102EB4323856044
:10F04000C360FFF751FF012811D1042384F83C303D
:10F0500094F82830042B02D1002384F82830A36BC5
:10F060008BB120469847012002B0BDE8F08102280C
:10F07000C4D194F82830042B09D00220BEE7022323
:10F0800084F83C30BEE7012002B0BDE8F0810023E7
:10F09000022084F82830B1E7982D0120983D012006
:10F0A000F7FFFF0F38B590F834300446052B40D8F1
:10F0B000DFE803F01E03390F1863006B4FF0FF31D8
:10F0C000FFF79EFD012834D1E06AA0BB032384F83A
:10F0D000343000212046FFF707FF012829D10423FF
:10F0E00084F8343094F82830082B28D0012038BD1B
:10F0F000234D00F130010120D5F838280232FFF706
:10F10000A7FD012828D00238C0B2012811D8052354
:10F1100084F8343094F82830082B15D001230220CD
:10F1200085F8E53738BDC06A216BFFF769FD012816
:10F13000CCD0002038BD022384F83430F4E700231B
:10F14000012084F8283038BD0023022084F82830BC
:10F15000012385F8E537E5E7D5F84028E368206B1B
:10F1600003EB4223E26AC5F84408C4E9033002B95C
:10F170006062012384F83430A0E7014DCAE700BF84
:10F18000983D012010B590F838300446032B59D82B
:10F19000DFE803F0022F38432B4BC0681A7803F5E1
:10F1A0008053032AD3F84018D3F8C4270CBF4FF07C
:10F1B000800C4FF4807C226101FB0CF100EB4120BC
:10F1C000E060D3F8A807A0EB4120C3F8A807D3F864
:10F1D000AC07A0EB4121E06AC3F8AC1702EB0C01CD
:10F1E000C3F8C417C4E90C2140BB6262012384F850
:10F1F000383000211548FFF777FE012811D102238E
:10F2000084F83830626B04F130010120FFF7B6FD5D
:10F21000012806D1032384F8383000212046FFF767
:10F2200063FE431EDBB2012B00D910BD94F82830D9
:10F23000062BFAD1002384F8283010BDA2EB0C0273
:10F240002263D3E70220ECE7982D01203845012006
:10F250004368C3F308020A44B2F5007F2DE9F04386
:10F26000044683B00D4605D22B440120636003B0F1
:10F27000BDE8F08390F91A20501C0AD0434902F5EA
:10F28000B17201EB0212D1796FF30001D171FF224B
:10F29000A27694F91B20511C0FD03C4902F5B172A3
:10F2A000FF2601EB0212D179C1F34500013820EAB3
:10F2B000E07060F34601D171E67694F800C0BCF1CD
:10F2C000020FD1D0DFF8CC80D8F84028B5EB422F20
:10F2D0004FEA42290DDCD8F848781F407A42AA420A
:10F2E00007DCEA194A4508D2206900283DD10120EF
:10F2F000BDE7002003B0BDE8F083227E206912F054
:10F30000080627D0D8F8C427411C8A4214D300D15C
:10F3100000214B44A5EB0905BCF1020F6061A3EB92
:10F3200007033D44084621616360DED1D8F85028C8
:10F33000B3EB422F98D3DAE798F8E42722B90123F8
:10F3400088F8E43763682069104A0126567094F8FB
:10F3500000C0DEE701A93FF02DFE0128C9D10199C7
:10F36000636894F800C02069D3E7084A1278032A3A
:10F3700006D080B24FF6F77290427FF675AFB6E7CF
:10F38000034A90427FF670AFB1E700BF982D01208D
:10F39000F7FFFF0F983D01202DE9F04790F8384026
:10F3A00082B00546032C00F2A680DFE804F00218C4
:10F3B0006E0BFFF777FE01280FD0022809D1032337
:10F3C00085F8383000202B6C022485F8280003B122
:10F3D0009847204602B0BDE8F08785F838002B78C2
:10F3E000022B5ED0454A6B68D2F8482803EA02092E
:10F3F000C9F34F29DFF804812846FFF7ABFA064628
:10F40000A9EB0009A8F5805A01A902223046002381
:10F41000FFF7C4FA09EB060701284FF40072BFB2E8
:10F420004FF00001044606F10106D2D1019847F0E1
:10F4300059FCEB694FF4007128460BB16B68B3B30C
:10F44000D8F84038013B9F420CD2FFF701FF01235F
:10F450000028D9D198F8E4270AB988F8E4378AF85F
:10F460000130D1E7C3EBC35328465902FFF7F0FE42
:10F4700040B998F8E43713B9012388F8E437204BF2
:10F4800001225A70022385F8383000222B6C85F84F
:10F49000282053B1012428469847204602B0BDE8F1
:10F4A000F0876B68C3F34F29A4E7012491E7019B20
:10F4B0004FF020324FF0100C4FF02E0E1A605A60B1
:10F4C00083F800E0C3F807206C6A1A625A6283F876
:10F4D0000BC0C3F8272083F820E083F821E0EA6B13
:10F4E0005C8324FA0CF45A8722FA0CF29C8283F88B
:10F4F0002BC09A86A4E700246BE700BF983D01204B
:10F50000982D0120B1F904300F2B2DE9F0410E4662
:10F5100082B00446174637D02046FFF71BFA94F90D
:10F520001B80B8F1FF3F40D05E4B41F2186203EB05
:10F5300008118A58904212D1183303EB4825B3883A
:10F54000204601331BB205EB4315B3803D60FFF746
:10F5500001FA01233060184602B0BDE8F08103F5DE
:10F56000805292F8E41700296AD001225A7022785A
:10F57000022A69D02369002B50D1012300221846AA
:10F580003A6002B0BDE8F0814FF40071FFF760FE11
:10F59000002850D04FF6FF732046B380FFF7DAF90A
:10F5A00094F91B80B8F1FF3FBED12278022A53D0D4
:10F5B0002369002BDCD03B490978032969D09BB231
:10F5C0004FF6F7718B4294BF00230123002BCFD15C
:10F5D00038B9354A92F8E437002B4ED0314B01222E
:10F5E0005A700023112201A9FFF7D8F9012842D14E
:10F5F000019D2E4BEB1A48BF03F2FF13B3F5B05F2A
:10F600004FEA632230D3284A92F8E43713B9012332
:10F6100082F8E437234B01225A7027E0214A1278FE
:10F62000032A2ED09BB24FF6F772934294BF002369
:10F630000123002BA1D10023184602B0BDE8F081C0
:10F64000012182F8E41790E7174A6368D2F850283E
:10F65000B3EB422F91D2EEE7134A6368D2F8501809
:10F66000B3EB412FB4D3F1E74FFA82F884F81B8053
:10F67000002D7FF464AF22787AE7012382F8E43723
:10F68000ACE70B4A934294BF00230123002BD2D056
:10F6900073E707498B4294BF00230123002B97D0C7
:10F6A00066E700BF982D0120983D0120B02D012074
:10F6B000F7FFFF0F2DE9F04790F8303088B004468F
:10F6C000042B4AD8DFE803F0030C4CD04500C548B2
:10F6D00042F08CFB4FF6FF720123228484F8303015
:10F6E00004F11C0801AEBF4D04F131093246414618
:10F6F0002846FFF707FF012800F0DB8002282CD105
:10F70000B94901F5805595F90228531C0AD002F534
:10F71000B17201EB0212D3796FF30003D371FF23AF
:10F7200085F8023895F903385F1C0FD003F5B173E3
:10F7300001EB0313DA79C2F34501013921EAE171E2
:10F7400061F34602FF21DA7185F80318042384F877
:10F7500030300020E36A2070984708B0BDE8F08799
:10F76000A24D95F81038002BF7D104F11C0901AE19
:10F770009C4F4FF00908324649463846FFF7C2FE13
:10F78000012840F0E8800198002800F0C28003784A
:10F79000E52B01D0002BEED1954A821A48BF02F228
:10F7A000FF12B2F5B05F4FEA622380F00E811B01B9
:10F7B0008D49904A13449A7B042A0CD0D5F8C82668
:10F7C0000132C5F8C8265A6004229A73D5F8CC369F
:10F7D0000133C5F8CC3695F902385E1C0AD003F522
:10F7E000B173FF2201EB031385F80228DA796FF376
:10F7F0000002DA7195F903385A1C0FD003F5B17382
:10F8000001EB0313FF21DA7985F80318C2F34501F0
:10F81000013921EAE17161F34602DA712022002107
:10F8200047F060FAD4F83110D4F8352005A8019BD0
:10F8300019605A6094F83B20B4F839109A72198113
:10F84000019B627EDA7202F0D1F8BDF81430002B11
:10F8500040F0068144F28171019A03201182D38124
:10F860001183D38284F83000237E980608D50023C4
:10F87000112205A9E069FFF791F801287FF46DAF27
:10F88000204642F0B3FA2369002B68D0237E03F0B0
:10F89000F70213F0040322766ED1122A00F083805F
:10F8A0000022E36A204684F82820984708B0BDE883
:10F8B000F087019F002F00F09F803B78002B00F025
:10F8C0009B8097F80BA01AF0080F7FF40FAF0B2264
:10F8D0004946384647F033FB00287FF407AF637E84
:10F8E0008AEA0303DB0640F1FC803F4901F58055BD
:10F8F00095F902385E1C3FF415AF03F5B173FF2292
:10F9000001EB031385F80228DA7960F30002DA715B
:10F9100008E795F8E837022B3FF418AF95F8103850
:10F92000002B7FF413AF85F820383846C5F824380B
:10F93000C5F8283885F81C38D5F8FC3785F81088C4
:10F94000C5F81438D5F84438C5F81838FFF724FD41
:10F9500001283FF410AF02283FF4F8AEFDE6237E05
:10F9600019079DD5214B93F8C827002A7FF4F5AEDF
:10F97000072283F8C82793E7A56800232046E66A94
:10F98000294684F82830FFF763FC002840F0A38064
:10F9900094F82830002B7FF4E0AE0223C4E90B6515
:10F9A00084F82830D9E6E06A0421626AA063204620
:10F9B00084F83C3084F8281063636362C4E90B2246
:10F9C000C4E9023342F012FAC7E695F8E43713B9F6
:10F9D000012385F8E437012303494B706FF00F03CF
:10F9E000E7E600BF80450120982D0120983D0120C9
:10F9F000B02D0120B0430120584901F5805595F9FB
:10FA000002385E1C0AD003F5B17301EB0313DA79F7
:10FA10006FF30002DA71FF2385F8023895F9033895
:10FA2000581C0FD003F5B17301EB0313DA79C2F35D
:10FA30004501013921EAE17161F34602FF21DA71E2
:10FA400085F80318237EDA067FF580AE444842F03D
:10FA5000CDF94FF6FF720223228484F8303080E61D
:10FA6000404B05A8B3F9B48201F0E8FE4FF47A7276
:10FA7000002306460F4645F0E7FA3C230546394683
:10FA800030464FF47A7208FB0355002345F0DCFA48
:10FA90004FF47A7192B2002302A8C5FB012301F052
:10FAA00003FF9DF80A209DF80B109DF80C3041EAE9
:10FAB0004211BDF80820DB02A2F2BC7241EA4221E9
:10FAC0009DF80D2043EA42139DF80E2089B243EAC7
:10FAD00052039BB2C0E6002E3FF43FAE2046B04733
:10FAE0003BE6BA8A7B8B204D43EA0243D5F8402897
:10FAF00063625202FB69B3FBF2F102FB1131A360B6
:10FB000009B113445B1AE36084F819A095F902382F
:10FB10001249581C0AD003F5B17301EB0313DA79CB
:10FB20006FF30002DA71FF2385F8023895F9033884
:10FB30005A1C0FD003F5B17301EB0313DA79C2F34A
:10FB40004501013921EAE17161F34602FF21DA71D1
:10FB500085F80318032384F8303085E6982D0120BA
:10FB600080450120082A0120983D012010B5037826
:10FB7000044690F818C0023B012B02D91CF0060F76
:10FB80005DD11CF0200F3CD194F91A30591C0AD0D9
:10FB9000314A03F5B173FF2102EB0313DA796FF3F6
:10FBA0000002DA71A17694F91B305A1C0FD02A4A50
:10FBB00003F5B17302EB0313DA79C2F3450101399E
:10FBC00021EAE17161F34602FF21DA71E1761CF06E
:10FBD000080F0DD0214B93F8C827072A05D093F8BA
:10FBE000E427A2B31C4A01215170002283F8C827E0
:10FBF0000023E26A237084F82830FAB1BDE810408F
:10FC0000104700231649E0691A018A58904206D02D
:10FC100001330B2BB8D01A018A589042F8D10E4A02
:10FC200003F5B17302EB0313DA79C2F3450101392D
:10FC300021EAE17161F34602DA71A5E710BD012105
:10FC4000FFF752F90128F9D194F818C099E7012279
:10FC500083F8E427C6E700BF982D0120983D0120D6
:10FC6000B04301204FF0FF3C344A002334482DE9D3
:10FC7000F041644603E0013310320B2B15D01178AC
:10FC80000429F8D103F5B17100EB0111C979CE0750
:10FC9000F1D4651C52F80A1C01D06145EBD21C4618
:10FCA00001338C4610320B2BE9D1631C02D10120A9
:10FCB000BDE8F081224D04F5B1772601DFF88C8094
:10FCC00005EB0713998879BBD8F81824AB191D4E9A
:10FCD000D2F8108041F2186206EB442198580023B4
:10FCE000194AC04788B1022802D00020BDE8F0813F
:10FCF00006F6E87605EB071501220020D6F8CC368B
:10FD0000AA71013BC6F8CC36D2E706F6E87605EBD9
:10FD1000071503210122D6F8CC36A971013B86F8DC
:10FD2000D026C6F8CC36C3E705EB041341F21862BF
:10FD30009858D8F81834DB689847C5E7BE430120C7
:10FD4000982D0120B02D0120E5890008101901200F
:10FD50002DE9F04F90F8283083B00446013B082B82
:10FD60000BD8DFE803F0383C1F2305290A2E3300A7
:10FD70000121FFF7FBF8012802D003B0BDE8F08FA6
:10FD80000022237884F82820002BF6D0226C03214F
:10FD9000D4E9010384F828108342E26238BF0346A5
:10FDA0002046A36003B0BDE8F04FDFE6002103B0BA
:10FDB000BDE8F04FFFF7DAB803B0BDE8F04FFFF74A
:10FDC000E1B903B0BDE8F04FFFF76CB903B0BDE88F
:10FDD000F04FFFF7E1BA03B0BDE8F04F6AE4544FCB
:10FDE0004368D7F84858016B9C461D40D7F8402817
:10FDF00068185602B0EB422FC0F0978094F800E0EC
:10FE0000A7F5805A4FF6F778DFF82891BEF1020F78
:10FE100014D02069002856D1D4F804C0A36800216A
:10FE2000E26A634584F8281038BF6346A360002A5D
:10FE3000A3D0204603B0BDE8F04F1047D4F804C06B
:10FE4000D7F85028BCEB422FE8D22069227E120757
:10FE50002BD5D7F8C42700F1010C624521D297F8C1
:10FE6000E42722B9012387F8E4376368216B012274
:10FE70008AF8012094F800E0891B334429445B1B75
:10FE800000258E4263602163C4E904C09C46BDD94D
:10FE9000BEF1020F3DD020690028BFD0DFF898B036
:10FEA0001FE0E9D14FF0000CE6E701A93FF082F82E
:10FEB00001287FF462AF2069DDF804C094F800E007
:10FEC0006368216BD8E79AF80020D346032A19D03B
:10FED00082B2424594BF00220122002AB6D0D4F853
:10FEE00004C09BF80030032B19D080B24FF6F77393
:10FEF000984294BF0020012000288FD18C44C4F880
:10FF000004C08BE7484594BF00220122002A9DD0FF
:10FF1000E5E7D7F85028B3EB422FEFD37EE7054B48
:10FF2000984294BF00200120E6E794F800E0AFE794
:10FF3000983D0120F7FFFF0F982D012043F2012289
:10FF40000121002343F2010C028043F201120172ED
:10FF50004FF601718280FF22A0F802C043818381A5
:10FF6000C381018282747047FF22174B4FF0FF3C20
:10FF7000C270027102724272427382738274C274DE
:10FF80000022F0B503F10C076646172516244FF042
:10FF9000150E02EB8202BB4200EB020100F802E008
:10FFA0004C708D70CE7081F804C00BD093F9062090
:10FFB000063393F801E09C78DD7893F9046093F9B7
:10FFC00005C0E6E7F0BD00BF788305084FF0000CE0
:10FFD00001210222032380F805C08171C2710372DE
:10FFE000704700BF00230222037043708370C37008
:10FFF000027170474FF0010C2C210222002380F87F
:020000040801F1
:1000000000C041708270C370704700BF4FF4F07140
:1000100040F22E4C0022072301804FF47A71A0F8A1
:100020001EC04FF4FA6C41844FF4F5618271A0F860
:1000300020C040F2012C428242F22462818442F2CA
:100040001F31A0F814C040F2034C018142F2275145
:10005000428142F220128370A0F816C040F2056C73
:1000600081810E21C281012283760223A0F818C06B
:1000700080F826104271437400B540F2262EA0F895
:100080001CE05DF804FB00BF8388C3F30B039342BD
:10009000A8BF134670B51D460C461A460646806832
:1000A00046F0ACFD6219084B9442B56908D0074888
:1000B00014F8011B00FB03F3A24283EA0103F7D10A
:1000C00001202B6070BD00BFC59D1C819301000104
:1000D0000023037043708370C37070470023037064
:1000E00043708370C3707047002201234FF0390CB6
:1000F0008121427080F800C08270C270017143712A
:100100008371C371704700BFFF23002243700270E8
:100110008370C370704700BF002306214FF47A72CA
:1001200001700373C0E90123704700BF00234FF043
:10013000030C422101224370C37080F800C081701B
:10014000027170470023FF22411C10B500F81320F4
:1001500001F8132001330B2BF8D10B4B4FF0FF317B
:10016000002203F10F048C4605E093F904C093F9D3
:10017000051013F8032F00EB420E9C4200F812C04A
:100180008EF80110F1D110BD8C8305084FF01F0CC3
:1001900001220023022180F800C04FF0230C42709E
:1001A00080F803C04FF0240C027180F806C04FF0B5
:1001B000260CC27180F809C04FF0270C827242737E
:1001C00080F80CC04FF0250C0274202280F80FC07C
:1001D0004FF0210C8274382280F815C04FF0130CB8
:1001E0000276032280F81BC04FF0FF0C027710222A
:1001F000837043710372C37283734374C174037554
:100200008175C37541768376C17780F81DC082778A
:1002100080F82030704700BF03230370704700BF91
:100220000A4491421AD001F1FF3C41F2210100B58C
:1002300002F1FF3E1CF8012F082380EA022010F48F
:10024000004F4FEA400281EA40000CBF90B280B2FA
:10025000013BF4D1E645EDD15DF804FB704700BFEA
:10026000704700BF2DE9F047089F002B0E4605465A
:100270003C4614BF4FF030094FF0200914F8011B21
:1002800041B3002A2CDD234600E0B2B113F8010B84
:100290009046013A0028F8D1A8F102086AB1C24696
:1002A00049462846B04753460AF1FF3A002BF7DC8F
:1002B00028EAE8723978013249B1D71B2846B0479D
:1002C000E01914F8011B0029F8D1BDE8F0871046A9
:1002D000BDE8F087002A02F1FF38E0DC0846F4E7C9
:1002E0000022EAE703685A1C02601970704700BFD9
:1002F000024B186803681B68184700BFF0650120AF
:100300000378092B01D0202B05D110F8013F202BB9
:10031000FBD0092BF9D02D2B63D02B2BB7EE000A85
:1003200008BF01300278A2F13003D9B2092961D89F
:10033000F2EE046ADFED4D7A07EE103A10F8012F65
:10034000B8EEC77AA2F13003D9B2A7EEA67A09298E
:10035000F0EE477AF0D92E2A50D0037803F0DF036D
:10036000452B3BD110B442782D2A73D02B2A62D072
:10037000A2F130030130092B63D80024002303EBE2
:10038000830302EB430310F8012FA2F13001303B4D
:100390000929F4D9B3F59A7F1A46B7EE007A28BF37
:1003A0004FF49A72072B09D91346DFED316A083BE7
:1003B00027EE267A072BFAD802F007022AB1F2EECE
:1003C000046A013A27EE267AFBD1002C3BD0C7EE17
:1003D000877A5DF8044B20EE270A704720EE270A43
:1003E000704742780130BFEE000AA2F13003D9B263
:1003F00009299DD92E2ADFED1D7AAED1437801302F
:10040000A3F13002D1B20929A8D8B2EE047AF0EEF5
:10041000475A06EE902A10F8013FB8EEE66AA3F1BB
:100420003002D1B2C6EE076A092927EE257A77EEA7
:10043000A67AEED992E782780230A2F13003092B36
:100440009BD9B7EE007A67EE877A5DF8044B20EE11
:10045000270A704782780230A2F13003092B01D8B5
:1004600001248BE7B7EE007AB1E700BF000000007F
:1004700020BCBE4CF8B5164D6B78BE2B25D1AC1CFC
:10048000144F022229464FF6FF70FFF7C9FE22885B
:100490004AB1A618BE4218D2052A16D921463446BA
:1004A000FFF7BEFEF3E721460222FFF7B9FE022264
:1004B000A1180634FFF7B4FE074B641B9C8041F67D
:1004C0000F53C31A58425841F8BD0020FCE700BF43
:1004D0000040000800800008F0650120F0B50679B2
:1004E00006F0E003402B03D145794FF0FF3406E0DE
:1004F000602B4FF00105F8D1447905FA04F400238C
:10050000012006F00706AB4200D1F0BD052E0FD842
:10051000DFE806F00308101D242448B1C85CD75C4E
:1005200078400FE020B1C856D756C71B78427841B3
:100530000133E8E70028FBD031F8130032F81370DC
:10054000784080B220420CBF01200020F0E7002854
:10055000EED031F9130032F91370E6E70028E7D046
:1005600051F8230052F82370DAE7037903F01803F7
:10057000102B1DD004D82BB1082B06D000207047BB
:10058000182BFBD1B0F80B007047114BB0F80B00E3
:1005900093F90030591C09D10E4B1B7A03EB8302EF
:1005A00003EBC20300EB830080B27047DBB2F5E7D8
:1005B000074BB0F80B0093F901305A1C06D1054BDC
:1005C0005B7AC3EB031300EB4300EDE7DBB2F8E724
:1005D000AC030120F0650120114A00234FF0280CE4
:1005E0000360838030B54FF448744FF0290E02F158
:1005F0000C0503EB4303AA4200EB430100F813C0D0
:1006000081F801E0D3788C808B7008D092F90630A5
:10061000063292F801C092F802E09488E9E730BD12
:10062000A0830508092917D0B1FA81F35B0999B1B4
:10063000013903604B0001F0030103F00802C1EB34
:1006400001119300C1EB0111A3EB92038900C3EBED
:10065000031381809B004380704700BF00B587B0C3
:1006600000224FF4E16C40F68C2E02A90346ADF84F
:100670000820ADF80AC0ADF80CE04FF4007E03C9C5
:100680000092ADF804206A46ADF81410ADF802C02F
:100690009860BDF814C092E8030040F20122A3F86C
:1006A0000CC0ADF8141042F20121DA8140F233524D
:1006B00043F6017C59809A8240F63401BDF814203B
:1006C000A3F800E0A3F810C0D980C3F816005A833D
:1006D00007B05DF804FB00BF144B1522144910B598
:1006E000044618681B79206204F1250084F8243040
:1006F00046F039FC0F4B4FF0010E1A7E84F83AE0B9
:1007000012B984F83B2010BD03F11C0CBCE80F00AB
:1007100020606160A260E360BCE80F0084F83BE009
:1007200020616161A261E36110BD00BFC0EC0508FA
:10073000C8EC0508F06501202DE9F84338220021B6
:10074000064646F0CFFA01230922174C4525B3731C
:10075000412186F8213041F61E63DFF86090671E64
:10076000F384124B09F108083272B362104B114A3C
:10077000336103F1C87303F2B63373610E4BC6E9FC
:100780000623484646F0B5FB631E294628B1DA1B0E
:100790004045A0EB090338BFF25415B114F8015FCE
:1007A000EFE7BDE8F88300BFD9EC05081E7D010125
:1007B0006400DC050019750343080E0028320608A2
:1007C000202108B546F095FB034618B11A78013090
:1007D000202AF9D0184608BDB5EEC00ADFED357AFB
:1007E0000023F1EE10FA70B5C8BF30EE270A86B0CC
:1007F000D8BF30EE670ADFED307A054603A90293D1
:100800006E4620EE270ACDE90033FDEEC07A17EEE2
:10081000904A84EAE470A0EBE4703DF0E3FC002C25
:1008200003A8ACBF20232D238DF8003043F048FFF0
:10083000012829D0022833D003281DD003A930462F
:1008400046F048FB304643F03BFF0446314628461D
:10085000033CE4B2224646F0D1F9002328462B554A
:1008600043F02EFF2E22431C31192A54E81846F07B
:100870004DFB284606B070BD302303A930468DF8E5
:10088000013046F027FBDDE7302303A930468DF821
:1008900001308DF802308DF8033046F01BFBD1E7B4
:1008A000302303A930468DF801308DF8023046F030
:1008B00011FBC7E76F12033A00007A4409F036B91A
:1008C00013B568B14C1E14F8011F21B902B0BDE880
:1008D000104009F03FB9019009F028F90198F2E7BA
:1008E00002B010BD10B50C4628B1C943013801F063
:1008F00001010AF0E9F8E30701D4FDF7BBF810BDE8
:100900002DE9F3410023124D044600EB8106114FFF
:1009100005F83C3FB44203D10F4802B0BDE8F08176
:10092000394628464FF0000846F0D4FA214668467A
:1009300046F0ECFA2021684646F0DBFA28B9694611
:100940002846043446F0C6FAE4E780F80080F1E770
:10095000F0650120474106082C660120014B186E06
:1009600031F088BFF065012010B5184C44220021F9
:10097000174846F0B7F9237804F580540321022B79
:100980004FF6FF70D4F84C284FF0100C18BF0B46F0
:10099000A4F8020884F8001804F5FD600021C4F8EA
:1009A000F82784F801C884F8E837C4F80C28FEF763
:1009B0004FFC48B994F8103833B90222C4F81438FF
:1009C000C4F8183884F81028012010BD982D012093
:1009D00080450120084B024608498B420AD218463E
:1009E00002E01C30884205D20388C3F30B039A420D
:1009F000F7D170470020704764B8060878C1060830
:100A000070B50546B0F80900FFF7E4FF064B044651
:100A1000284693F86460FFF7A8FD16B1E368184410
:100A200070BDA368FBE700BFF065012038B505463F
:100A30000C46FFF7E5FF2B7903F0E00203F0070314
:100A4000602A2AD1052B0CD8DFE803F0030B0F0B2B
:100A50001B1B6A79012393400278DBB214B1134364
:100A6000037038BD22EA0303FAE76A790123934051
:100A700002889BB214B113430380F2E722EA030316
:100A8000FAE701236A7903FA02F2036814B1134307
:100A90000360E6E723EA0203FAE7052BE1D8DFE883
:100AA00003F00303050507070470DAE70480D8E7BD
:100AB0000460D6E770B585880B4604460021C5F36F
:100AC0000B0518462A4646F00DF96169084A0346A7
:100AD000914202D3074A914205D319B11846BDE8A5
:100AE0007040084770BD2A46BDE8704046F086B8A1
:100AF00078C1060891C3060838B5064C064DAC42CD
:100B000006D2A16820461C34FFF7D4FFAC42F8D3CC
:100B100038BD00BF64B8060878C1060808234840FD
:100B200010F0800F4FEA400182EA40000CBFC8B2CB
:100B3000C0B2013BF4D1704730B505688D421AD977
:100B400001F1FF3E6C1E00231EF801CF082183EA4D
:100B50000C0313F0800F4FEA430C82EA43030CBFEF
:100B60005FFA8CF3DBB20139F3D17445ECD16A1C26
:100B700002602B7030BD00236A1C02602B7030BDF8
:100B80009FED067AF7EE007A60EE870A20EE800A83
:100B900070EE277A80EE270A704700BFDB0FC9404E
:100BA000B0EEC07AF0EEE06A86FE876AB5EE406A83
:100BB000F1EE10FA3DD0C6FEC75AC5EE867ADFEDDB
:100BC0001E2ADFED1E3ADFED1E4A9FED1E5A9FEDF5
:100BD0001E3AB7EE006A9FED1D4ADFED1D5AE7EEA3
:100BE000E23AA7EE834AE7EEA34AA7EE846AA7EEAD
:100BF000A45AE7EE855AC5EE867AF4EEC76AF1EE9E
:100C000010FA03D59FED137A77EE677AF5EEC00AF6
:100C1000F1EE10FA03D59FED107A77EE677AB5EE14
:100C2000C00AF1EE10FA48BFF1EE677AB0EE670A3B
:100C30007047DFED077AE0E739094E3DE3B59E3EA8
:100C400088FA163E45FE7F3F99FB243F69A2163E77
:100C5000A7DFA834DB0FC93FDB0F494091ED056AE0
:100C6000D0ED017AD1ED036A91ED047A67EEA66AC0
:100C7000D0ED005A27EE877AD1ED014A67EE867AE9
:100C800091ED025A91ED004AA4EEA57A90ED026A28
:100C9000E5EE257AD1ED064AE4EE256A91ED075A94
:100CA000D1ED085AA5EE067AE5EE867AE4EE866A7C
:100CB00080ED017AC0ED027AC0ED006A704700BF96
:100CC000DFED277AB4EEE70AF1EE10FA0CDDDFED86
:100CD000256A9FED257AF0EE407A30EE660AF4EE52
:100CE000C77AF1EE10FAF6DCDFED207AB4EEE70A0F
:100CF000F1EE10FA0CD5DFED1B6A9FED1D7AF0EED8
:100D0000407A30EE260AF4EEC77AF1EE10FAF6D405
:100D1000DFED187AB4EEE70AF1EE10FA14DDDFED3C
:100D2000107A37EEC00A60EE006A9FED136A9FEDFD
:100D3000137ADFED137AA6EE867A20EE266AE6EEC7
:100D4000877AA6EE270A7047DFED0E7AB4EEE70A3F
:100D5000F1EE10FAE7D5DFED057A37EEC00AE2E7EB
:100D6000DB0F4940DB0FC940E4CB1641DB0F49C024
:100D7000E4CB16C1DB0FC93F92E741B99730083C7D
:100D800015A82ABEDB0FC9BFFDEEC07A17EE903A58
:100D90002033402B00D893E79FED010A704700BF36
:100DA00000000000D0ED005A9FED2B4A08B535EE4B
:100DB000840AFFF7E9FFB0EE405AB0EE650AFFF78C
:100DC000E3FFD0ED014AF0EE405A34EE840AFFF71B
:100DD000DBFFF0EE403AB0EE640AFFF7D5FF90ED8E
:100DE000023AF0EE404A33EE040AFFF7CDFFB0EED0
:100DF000404AB0EE430AFFF7C7FF25EE236A65EECF
:100E0000046AC1ED024A25EE847A25EE005A81ED8E
:100E1000086A23EE844A23EEE53AB0EE666A65EE90
:100E2000805A81ED004AB0EE454A81ED053A60EE08
:100E3000637AA4EEE56AA4EE874AE4EEE65AC1EDD1
:100E4000017AA4EE857A81ED046A81ED034AC1ED51
:100E5000065A81ED077A08BDDB0FC93FB7EE001ACD
:100E60000022DFED050A10B546F0FAF80023836191
:100E700043610362C36110BDF304353F2DE9F04FB8
:100E80001F461346894689B013F8011B002900F05C
:100E90002B8215468046002609E0404601361D4655
:100EA000C8472B4613F8011B002900F08C80252928
:100EB000F3D16978302900F0DD8002350023A1F1FB
:100EC000300C5FFA8CF2092A4FF000025ED96C29CF
:100ED0007DD07829E5D8572967D9A1F15800202875
:100EE000DFD801A454F820F069110108A30E01080D
:100EF000A30E0108A30E0108A30E0108A30E01080A
:100F0000A30E0108A30E0108A30E0108A30E0108F9
:100F1000A30E0108A7100108B5100108A30E0108CF
:100F2000A30E0108A30E0108A30E0108A30E0108D9
:100F3000A30E0108A30E0108A30E0108A30E0108C9
:100F40009F100108A30E0108A30E0108A30E0108BB
:100F5000A30E01088B100108A30E01080F11010850
:100F6000A30E0108A30E010869110108BEF1050FC7
:100F700018D9BAF1050FAAD80A2CA8D102EB82021F
:100F800015F8011B04EB4202A1F1300C5FFA8CF062
:100F9000A1F1610EA1F1410AA1F137040928E5D8B8
:100FA0006446EBE7A1F15704E6E761B125297FF438
:100FB00078AF25214046C8472B46013613F8011B60
:100FC00000297FF474AF304609B0BDE8F08F15F802
:100FD00001CBBCF1780F3FF664AFBCF1570F4DD990
:100FE000ACF1580120293FF65CAF01A050F821F088
:100FF000CB110108A30E0108A30E0108A30E0108DE
:10100000A30E0108A30E0108A30E0108A30E0108F8
:10101000A30E0108A30E0108A30E0108A7100108E2
:101020007D120108A30E0108A30E0108A30E0108FA
:10103000A30E0108A30E0108A30E0108A30E0108C8
:10104000A30E0108A30E01089F100108A30E0108BA
:10105000A30E0108A30E0108A30E01088B100108BE
:10106000A30E01082B120108A30E0108A30E01080C
:10107000CB110108A9780123033520E7BCF1000F4B
:10108000A1D0BCF1250F94D00BE757F8040B002337
:10109000494600904046FFF7E5F8064401E757F857
:1010A000043B1E60FDE657F8041B40460136C9B2FA
:1010B000C847F6E6D7F800C0BCF1000FC0F2AC801C
:1010C00005ACA246BCF1090FE6464FF0010108DD70
:1010D00001EB81014900BCFBF1F00928F8D8002997
:1010E0003DD08948BEFBF1FBBBF10A0FA0FB01C05C
:1010F00001FB1BEE34BF4FF0300C4FF0570CC00813
:101100000929DC4401460AF801CBEAD827E038680F
:101110000121092809D901EB81014900B0FBF1F453
:10112000092CF8D8002900F0E68005AC0393A2460C
:10113000754BB0FBF1FBBBF10A0FA3FB013C01FBBC
:101140001B00B4BF4FF0300E4FF0570E4FEADC0CCF
:101150000929DE4461460AF801EBE9D8039B04370C
:1011600000218AF8001029E057F804AB0120BAF1F9
:101170000F0F40F2C6800001BAFBF0FCBCF10F0F6C
:10118000F9D8002800F0BA8005ACA34601E0BAFB0C
:10119000F0FCBCF1090F4FF0300E05DD58290CBFF3
:1011A0004FF0370E4FF0570EE64400FB1CAA000923
:1011B0000BF801EBEBD100218BF8001049464046BB
:1011C0000094FFF74FF806446BE657F804BB012183
:1011D000BBF10F0F40F28D800901BBFBF1F00F282E
:1011E000FAD8002900F0828005ACA24601E0BBFBE2
:1011F000F1F009284FF0300E06DDBCF1580F0CBF9E
:101200004FF0370E4FF0570E864401FB10BB090913
:101210000AF801EBEBD1A3E72D21CCF1000C0DF185
:10122000150A05AC8DF814104CE757F8040B012192
:10123000092808D901EB81014900B0FBF1F4092C20
:10124000F8D8002952D005AC0393A2462E4BB0FB30
:10125000F1FBBBF10A0FA3FB013C01FB1B00B4BF78
:101260004FF0300E4FF0570E4FEADC0C0929DE44E8
:1012700061460AF801EBE9D8039B71E757F8040BC4
:10128000002829DB05ACA24609284FF001010AD944
:1012900001EB81014900B0FBF1FCBCF1090FF7D86B
:1012A00000293FF45DAF0393174BB0FBF1FBBBF19B
:1012B0000A0FA3FB013C01FB1B0034BF4FF0300EB3
:1012C0004FF0570E4FEADC0C0929DE4461460AF85C
:1012D00001EBE9D8039B43E72D2140420DF1150AAC
:1012E00005AC8DF81410CFE70E466CE605ACA246AF
:1012F00036E7584678E705ACA24630E705ACA3468A
:1013000059E7D44640E700BFCDCCCCCC73B5114CE7
:1013100006460D460192A06EA0B10F49FFF7D0FA24
:101320003146A06EFFF7CCFA0C49A06EFFF7C8FA61
:101330000B49019B2A46A06EFFF7A0FD0949A06E4C
:10134000FFF7BEFA94F86C3013B1012384F86D30C6
:1013500002B070BDF06501203D3206082736060850
:10136000BD0801084A3206080EB400B584B0084929
:1013700005AB019001A853F8042B0393FFF77EFD02
:10138000019B00221A7004B05DF804EB03B07047B3
:10139000E502010800232DE9F0411C4682B0074612
:1013A00003802146013438462BF046FC082CF8D146
:1013B000002307F1FC06DFF8608087F8EA301D465D
:1013C000C7F8EC30C7F8F030C7F8F430C7F8F83099
:1013D0001F462A46414601A83446FFF7C5FF0322AF
:1013E00001A911F8013B5BB1013A04F8013BF8D1C6
:1013F000013504362770082DEBD102B0BDE8F0812D
:10140000013520462021144445F06CFC082D06F1DE
:1014100004062770DDD1F0E7E4EC0508F7B5114EBE
:10142000074600230C46304615460F496E3600F835
:101430006E3F04EB45050D4B002F08BF19460C4FBE
:1014400045F048FDAC4202D10A4803B0F0BD394630
:1014500034F8022B6846FFF787FF6946304645F0AF
:1014600039FDEFE7F06501204E32060857320608D5
:10147000603206085E660120F7B500230B4E044675
:1014800000EB41050A4F06F89F3FAC4202D10948E4
:1014900003B0F0BD394634F8022B6846FFF764FF0D
:1014A0006946304645F016FDEFE700BFF0650120C4
:1014B000863306088F660120F8B54E1E054601F1F9
:1014C0001F04054F16F8012F284639460235FFF74D
:1014D0004BFFA642F6D1F8BD6532060803685A1CD8
:1014E00002601970090A03685A1C0260197070477B
:1014F00002681146531C0360D31C11F802CB016033
:101500005178036093781B0443EA0123111D43EAD9
:101510000C030160D07843EA00607047A0F130030B
:10152000092B07D920F02000413819288CBF002052
:101530000120704701207047303809288CBF0020F7
:1015400001207047413819288CBF002001207047C6
:10155000613819288CBF00200120704720280BD04B
:10156000092809D00A2807D00D2805D00B380128F2
:101570008CBF00200120704701207047A0F141037B
:10158000192B98BF20307047A0F16103192B98BF29
:101590002038704710B56FF000440246044404E060
:1015A000B3EB0E0015D1A24214D012F8013BA3F107
:1015B0004100192811F8010BA0F1410C98BF20330C
:1015C00000F1200EBCF1190FEAD91B1A04D1002832
:1015D000E9D110BD002010BD184610BD02B38446ED
:1015E00010B5841804E0B3EB0E0014D1A44513D059
:1015F0001CF8013B11F8010BA3F1410200F1200E90
:10160000192AA0F1410298BF2033192AEBD91B1ADD
:1016100004D10028EAD110BD002010BD184610BD2D
:101620001046704770B5044608460D4643F048F82A
:10163000064602E014F8013F43B1204632462946EF
:10164000FFF7CCFF0028F5D1204670BD1C46204690
:1016500070BD38B507490546FFF7E4FF041E06498B
:10166000284618BF0124FFF7DDFF08B144F002044B
:10167000204638BD6A320608324806082DE9F04196
:10168000064686469EF800C070460EF1010EBCF17B
:10169000200FF7D0BCF1090FF4D0BCF10A0FACF168
:1016A0000B05EFD0ACF10D04B4FA84F46409002CFE
:1016B000E8D1012DE6D9BCF12B0F3DD0BCF12D0FA7
:1016C00039D0102A86463DD04FF0FF359046B5FB05
:1016D000F2F502FB05F7FF43FFB20EF1010E002009
:1016E00010E0ACF1300C5FFA8CFC944512DA8542C4
:1016F000764602D334D1674532D21C404FF0FF30DA
:101700001EF801CBBCF1390FEBD94CF0200CBCF129
:10171000600F0BD801B10E602CB3B0F1004F2BD984
:10172000DB0729D54FF00040BDE8F081ACF1570C44
:101730005FFA8CFCD9E70124102A00F1010E90F821
:1017400001C0C1D1BCF1300F19D04FF0FF354FF0BF
:101750001008B5FBF2F502FB05F7FF43FFB2BCE74B
:1017600008FB00C0CCE70028DEDA13F0010F18BF39
:101770006FF00040BDE8F0814042BDE8F0819EF886
:1017800001C00EF10106ACF141056046192D01D8EA
:101790000CF1200078280BD04FF0FF354FF01008E7
:1017A000B646B5FBF2F502FB05F7FF43FFB294E73F
:1017B00010229EF802C06FF070450EF1020E0F2746
:1017C00090468AE701230A22002157E770B50D46AB
:1017D0001446FEF7F5FF0646A0B1FFF7F3FF40F60B
:1017E00034039842A8BF1846B0F5617FB8BF4FF4E4
:1017F0006170A0F561731920B3FBF0F32B702378AF
:10180000013323703046FEF7DBFF0646A0B1FFF739
:10181000D9FF40F634039842A8BF1846B0F5617F5F
:10182000B8BF4FF46170A0F561731920B3FBF0F3FA
:101830006B70237801332370304670BD028840F20C
:10184000B55CA2F5FA6210B54FEA920E817802F00B
:101850000302C3780139124C02EB4202013B01EB57
:1018600082020CFB0E33017904EB42028479928FE1
:1018700013444279008903EB430301EBC3030021C6
:10188000C3EB031302EB8303064AC3EB03132244A7
:1018900002EB83024FF47A73C2FB030110BD00BF59
:1018A0007883050880436D382DE9F04117461E46C0
:1018B00005464FF47A72002338463146454C43F0D2
:1018C000C3FB4549454A0144454882FB01C34FEAF1
:1018D000E17C0B44CCEB631382FB03C24FEAE37C55
:1018E0001A44CCEB621284FB02C44FEAE27CCCEBDC
:1018F000A40C80FB0C404FEAEC74C4EBE010C3EB8B
:101900000314A1EB8401A971C2EB0211A3EB8103C3
:101910006B710CEB4C03A2EBC30240F2B55303FB1B
:1019200010CC80002A71BCF5896F44DA40F2DA23CA
:101930009C4547DCBCF5B77F2A4BB4BF002201228F
:1019400002EB42014FEA420803EBC10391B2B3F844
:10195000523008EB020E244C04EBCE044FF00B0E79
:10196000163401E034F8023D63451FDDBEF1010E7F
:10197000F8D11C4B42444FF0010E03EBC202938F8F
:1019800000F5FA600CF1010C4FF47A7285F802E070
:101990000844ACEB030C314600232880384685F818
:1019A00003C043F051FB2A81BDE8F0810EF1010E26
:1019B0005FFA8EFEE4E7032140F296534FF00608EB
:1019C0000A46C6E7022140F229434FF004080A46BE
:1019D000BFE700BFABAAAA2A80BC92C789888888C3
:1019E00073B06D1678830508B483050808B50D4BF0
:1019F000D3E9322352EA030C0AD10146002340F214
:101A0000011218460B804A808B808B710B8108BDB8
:101A1000054909688A1843F10003FFF745FF0120D3
:101A200008BD00BFF06501202C1D012090420B462F
:101A30002DE9F041B0FBF2F60446154608D2124AF1
:101A400005FB16441846135D00F8013BBDE8F08124
:101A50009642B6FBF2F706D20B4A05FB1767D15D3B
:101A600003F8011BECE7BA42B7FBF2F807D905FB14
:101A70001878054A12F8081003F8011BEDE74046F4
:101A8000FFF7D4FF0346F2E7ECEC050830B5684CED
:101A900083B0B4F8DC33B3F57A7F03D94FF47A73AB
:101AA000A4F8DC33B4F8DE33B3F57A7F03D94FF40E
:101AB0007A73A4F8DE33B4F8E003B0F57A7F04D982
:101AC0004FF47A731846A4F8E033B4F8E213B1F592
:101AD0007A7F03D900231946A4F8E233B4F8E4234B
:101AE000B2F57A7F04D94FF47A731A46A4F8E43336
:101AF000B4F8E633B3F57A7F02D90023A4F8E633CD
:101B0000884202D80021A4F8E013934202D30023B4
:101B1000A4F8E433B4F8F223B4F8F4339A4202D9C7
:101B20000023A4F8F233434B1B8803B3424DAA7839
:101B3000062A43D8414901EB820191ED270A297910
:101B4000002940D194F8FC1307EE903AAB7907EEE8
:101B5000101AF8EEE77AF8EEC76A86EEA77A0BB1AC
:101B600030EE000AB4EEC70AF1EE10FA30DC637A08
:101B7000032B14D8C3EB0313314A02EB4302237A3D
:101B8000032BC4F8042412D803EB83012D4A03EB82
:101B9000C10302EB8303C4F8083403B030BD002353
:101BA000274A6372237AC4F80424032BECD9002259
:101BB000244B2272C4F8083403B030BD29799FED5C
:101BC000220A0029BED0042A21D8002ACFD021E041
:101BD00067EE807ABCEEE77A8DED017A9DF80420FD
:101BE00007EE102AB8EEC77AF4EEC77AF1EE10FAD3
:101BF00001DD0132D2B2CAB1102AA8BF1022D2B27E
:101C00008A42134638BF0B4684F8FC33AFE7053AE7
:101C1000032AACD9F7EE007A87EE800A44F076FA10
:101C20002B88984228BF18462880A0E70122E6E7C3
:101C3000F0650120C41E0020F825012078830508E6
:101C4000C0660120386701206F1203382DE9F04F7C
:101C5000AD4E85B096F80C3400AFA3F11702022AFE
:101C600000F2C682A94BBB60DFF8C0924FF00008BB
:101C700096F81C1409F16C0A4C46DFF8B4B2A44D76
:101C800034E010F0010C4ED1142A00F0AD8243086C
:101C9000820803F0773302F033321344C208C31AC8
:101CA00002F011329B1A03EB131303F00F33ABFB5B
:101CB00003E2D209C2EB02229A1A830302D5012A57
:101CC00000F09282012A0ED9082A00F28D82BCF11E
:101CD000000F01D0284206D1F96041F0F7FDF96804
:101CE000002800F081820C34544521D094F904205E
:101CF0002068A2F11E03DBB2012BC2D8A37920F029
:101D000041004FF0000C022B2060A8BF0223A371FA
:101D1000E379022BA8BF0223E371237A022BA8BF29
:101D200002232372B3E708F101085FFA88F8AEE7EF
:101D300008F1FF38B8F1020F00F2568200240220A9
:101D400086F8BC440CF0E0FD96F8C034022B00F09D
:101D5000FB82002800F068836E4B4FF47A7E96F881
:101D60008D854FF0000C03F5247B5A88B2F57A7FFD
:101D7000B3F8462088BFA3F802E0B2F57A7F9A88CC
:101D800088BFA3F846E0B2F57A7FDA8888BFA3F867
:101D900004E0B2F57A7F02D90022A3F806C0998840
:101DA0009142B3F85A10B3F85C2098BFA3F804C06E
:101DB000914293F86B2002F1FF3288BFA3F85AC01A
:101DC000632A03D94FF0640283F86B2093F86C20E8
:101DD00003F1660019460132D2B2092A4FF000021F
:101DE00088BF83F86CC08D7A013210F8014B063140
:101DF000A54238BF00F801CC032AF4D1B8F1010F95
:101E000003F1A40318BF03F81FCC5B45ADD1424BCF
:101E10009B78042B00F0E1822BB93F4A1388B3F57D
:101E2000F07F00F20382FFF731FE3C4896F8A015E0
:101E3000FEF7F8FB103096F8BF15FEF7F3FB0E30F7
:101E400096F8CD15FEF7EEFBB6F8DA25B6F8D835DC
:101E50001343B6F8DC2513431BB213B10123A6F8D4
:101E6000DE35D6F87C352E4A1A40002A00F0EB8287
:101E7000DA0700F15B825D0440F1DC812949D6F884
:101E800080250B400A40C6F87C35C6F8802513F43F
:101E9000004200F01982002286F8232486F83324B9
:101EA000D90440F11B8296F8EB35022B02D10123B5
:101EB00086F8EB35DFF870B05B460BF1780402E092
:101EC0000633A3420CD01A78072AF9D19978DA7828
:101ED000914202D35A79002AF2D007201DF0F4FF74
:101EE00000234FF4806086F8BC340CF00DFD002810
:101EF00000F08D820C4DA84698F8051029B398F88B
:101F0000000000B35B4618E0F06501207883050807
:101F1000BC02020038670120F8250120A06B0120D7
:101F200009600002F6DFFFFDE06B01203C6A012042
:101F30008180808006339C4207D01A788A42F9D18A
:101F40005A79002AF6D01DF0BFFF08F10608444573
:101F5000D2D1BB4B93F802B0BBF1080F00F0128254
:101F600096F88D35D6F88025A3F10103C2F3C03170
:101F7000B3FA83F386F86A165B0986F8683696F832
:101F80008E35A3F10103B3FA83F35B0986F86C364F
:101F900096F8D933032B02D9002386F8D933A949FF
:101FA000D6F87C350A400B40B17DC6F88025C6F8CE
:101FB0007C35002900F0F281B6F88036002B40F025
:101FC000F981D6F8843613F07F4F02D00023C6F88B
:101FD0008436D6F88C369C4A1A401AB140F2022355
:101FE000C6F88C3696F88836013B042B02D90123BB
:101FF00086F88836ABF1050B944BBBF1030F93F8D1
:1020000090B540F27E81BBF1000F20D00023FB6031
:102010008B4B6FF007017C60C91A03F108080C466E
:1020200004E004EB08035B4580F0248118F8010B01
:102030000028F6D009F0ACFA0028F2D083799B078B
:10204000EFD5FB6801227C68002B40F019817C4BA6
:102050009B7913B100237A4A9371B6F8963613F040
:102060000C0F03D1C3F30313022B03D94FF42063E6
:10207000A6F89636B6F8983613F00C0F03D1C3F3D2
:102080000313022B03D940F60123A6F8983696F8DD
:10209000052796F811379A4200F23D8196F80437E9
:1020A00096F810279A4204D2002386F80437A6F83F
:1020B000083796F8062796F8FA379A4202D900238D
:1020C00086F806376249FC6001F1780BBC6811F8AC
:1020D000013C4FF0030803EB4303234493F870E201
:1020E00093F871C293F872020B461A787245A8BF32
:1020F000724603F8012B5A796245A8BF62465A71AD
:102100009A788242A8BF0246B8F101089A70ECD1D1
:102110001E318B45DBD1D6F84424FC68002A00F040
:1021200053810020012102E00635AC420ED02B780D
:10213000282BF9D16B78043301FA03F31342F3D05F
:10214000063522EA03020120AC42F0D108B1C6F8FC
:102150004424404D05F108042B4613F8012B072AAF
:1021600000F29B809C42F8D1EB4688B0FF212022F0
:102170006B46184644F0B6FD3649034611F8012B6C
:1021800053F82200013040F08F808C4243F8222027
:10219000F4D1B6F88625DD46B6F884359A4202D3E6
:1021A0002D4BC6F88435FF232C4986F82C3899F935
:1021B0000430142B05D0D9F8002031EA020200F0D7
:1021C000098109F10C09D145F1D1254A5379012B37
:1021D00004D0022B04D1234B1B790BB9002353717C
:1021E0001437BD46BDE8F08F1F480AF05CFCA5E53A
:1021F0001E4A1146BA60DA0001EBC30393F8B81027
:1022000021B1D3F8BC30002B00F0FD80BB68134433
:1022100093F8B920002A3FF427AD93F89831002BAA
:102220007FF422AD182386F80C341DE54FF4F073CB
:102230001380F8E51C0740F182800D491FE600BFBE
:10224000F8250120FEDFDDFDFDFDFFFFC41E00209F
:10225000C36601200B260120AE014A0101000200E5
:10226000B42C01209C2901203C6A012078830508B8
:10227000FE9FFFFDFB6800227C68002B3FF4E7AE69
:1022800076494B7C002B7FF4E8AE4B79012B3FF471
:10229000DEAE002A7FF4DBAEDFE6EB4688B020221C
:1022A000FF21684644F01EFD05F8018B08F1010886
:1022B000B8F1080F3FF46DAF05F8018B08F1010884
:1022C000B8F1080FF0D164E796F8231400293FF421
:1022D000E7ADD90486F833243FF5E5AD1A067FF55E
:1022E000E2AD96F80C34182B06D801229A405C4BCC
:1022F0001340002B7FF4D7ADDFF878B10BF17804F1
:10230000EEE50023554A1371BBF1000F00F09980F0
:102310000123FB607CE6002296F8043786F8052747
:10232000002B3FF4C6AEA6F80827B9E64D49D6F80B
:1023300080250B400A40C6F87C35C6F880259804F5
:102340007FF5A5AD48499AE500283FF405AD474B18
:102350004FF0FF0C90F9045096F80D1503F16C0046
:1023600093F90820AA4204D10139012483F808C056
:10237000C9B20C338342F3D1002C3FF4EDAC86F8A4
:102380000D15E9E41A469B79002B3FF4E9AD537C27
:10239000012B7FF4E5AD02235374E1E534490B438F
:1023A0000A43C6F87C35B6F88036C6F88025002B7F
:1023B0003FF407AE96F87C0609F0EAF800287FF4AF
:1023C00000AEA6F88006FCE528201DF07DFDD6F8BD
:1023D0004424A6E686F82C38F7E6D6F87C351F4A62
:1023E00023F48053C6F87C35D6F8803523F4805327
:1023F000C6F88035538CB3F57A7FBFF414AD4FF433
:102400007A7353840FE5172386F80C34FEE6D6F86A
:102410007C3523F00063C6F87C35D6F8803523F090
:102420000063C6F8803565E5D6F87C25D6F880359A
:1024300022F0800223F08003C6F87C25C6F88035A0
:102440008AE45A461CE7D6F8802543F0080342F098
:102450000802C6F87C35C6F8802509E5F825012074
:1024600000410001F79FFFFDF6BFFFFD006B01205B
:1024700020061500E06B01202DE9F04FAE4E83B031
:10248000AE4B4FF0010AD6F83C28DFF8F08202F29A
:10249000DC524345C6F83C284CD29B46A84BA94D7C
:1024A0009F1CA74B5988002900F021817A18AA4265
:1024B00034BF00200120052998BF40F0010000280A
:1024C00040F01581BBF800003C46C0F30B000BE068
:1024D000118814460A44002900F00981AA4280F0BC
:1024E0000681052940F2038161888142F0D161793A
:1024F0008B07EDD123885846DBF8081094F8049038
:102500000193FEF7D7FABBF80010B9EB113F00F0CA
:10251000F6804FF0000ABBF804100BF11C0B5BF8BF
:10252000140CC1F30B013CF0A3FA5BF8042CC34577
:102530001060B6D3D6F87C35834DC6F88035FFF7EA
:1025400085FB337AA5F17801804C03EB830203EB22
:10255000C203727AC2EB021205EB830301EB420263
:10256000C6F80834C6F804241AF05EFB4FF0FF33B7
:10257000D6F80804636022F07BF81DF0F7FC05F53F
:10258000956305F5A46103E00633994200F0C1802C
:102590001A78002AF8D19D78D878854202D35879E4
:1025A0000028F1D096F8E8356421227203EB83030A
:1025B00003EB83039B00632BD8BF6423C6F8343836
:1025C000B6F8EC3501FB03F3632B40F3A7801A4602
:1025D000C6F8383800235E4C5E49C6F83C38C1F86E
:1025E0001447C6F84038C6F84438C6F84838C6F824
:1025F0004C38C6F85028A6F8543886F8563823F0D8
:10260000EBFAB6F86A38DFED546A05EE903AB6F8A0
:1026100066389FED527AF8EEE55A07EE903A9FED54
:10262000500AF8EEE77AB6F8641865EEA65AB6F8DE
:10263000583896F85A0867EE877A35EE800AC4ED66
:10264000A17AFDEEC07A17EE902A07EE901AF8EE06
:10265000E77A2032402A67EE877AC4EDA27A61D801
:10266000FEF72EFBFDEEE57A3E4981ED000A17EEFE
:10267000902A2032402A5BD8B0EE650AFEF720FB94
:10268000F1EE407A96F86828C1ED017A07EE902ABB
:102690009FED357A9FED320AF8EEE77AA7EE870ACA
:1026A000FDEEC07A17EE902A2032402A3DD8FEF780
:1026B00007FB07EE903ADFED2D6A2D4BF8EEE77A37
:1026C000C6F87C08A3EC010A86EEA77A83ED007AAF
:1026D00030F07EF917F0FCF9264B012250461B68BA
:1026E00086F85528C6F83C3803B0BDE8F08FDBF813
:1026F000081058464FF0000AFEF7DCF90BE7019B83
:10270000A11D58469A1FFDF7BFFC00287FF403AFB8
:10271000FFE6F27D003A18BF012243E70A46C6F8F9
:10272000381857E79FED140A9CE79FED130AC0E79E
:10273000DFED117AA6E700BFF065012064B8060856
:10274000004000080080000838670120AC03012029
:10275000C86B0120C41E002088C3E43A17B7D138E3
:10276000DB0FC93F5C6E012035FA8E3CC0C9FB48C7
:10277000646E01202C1D01200000000078C10608B5
:1027800038B501221C4B032805461C4C83F81C2736
:1027900020D96A1C00231A490220D2B24FF0140E2D
:1027A0005200402A28BF4022C854023301EB030CD8
:1027B0009A420CF801ECF7D8FF2D4FF0FF034FF0D1
:1027C0000E0008BF0222224482F88038BDE838405B
:1027D0000CF006BA00EB800004F5A473257205EB3B
:1027E000C00003EB8000C4F8080421F041FF20F092
:1027F000F1F820F0C3F9CCE7C41E0020F0650120F9
:10280000706E0120054B0121D3F8C42883F8C1184C
:1028100042F40012C3F8C428704700BFF0650120DD
:102820000368C3F30D032DE9F041054686B00C465D
:10283000002B41D1394A0120394E0221B242CDE963
:102840000233CDE9040120D3364B9A421CD303F561
:1028500080439A4224D3344B9A4223D903F58033E0
:102860009A4221D903F500339A421FD903F5003368
:102870009A421DD903F500339A421BD90A2105203B
:1028800008F0B2FD3CF036FF034601A902A803930D
:102890003CF070F880B14FF0FF3006B0BDE8F08139
:1028A0000B46F2E70323F0E70423EEE70523ECE70A
:1028B0000623EAE70723E8E71C4E96F8DC38012BED
:1028C00002D16FF00100E8E701232F68D4F80080FF
:1028D00086F8DC383BF0EEFFB0B9154C236923F4E1
:1028E00040732361236943F400732361236943F038
:1028F00001032361C7F80080BFF34F8F3BF0DAFF7D
:10290000236923F001032361002386F8DC380028C3
:10291000D7D12B6804332B60BFE700BF004000080D
:102920000040000800800008FFFF0008F06501205B
:10293000003C02402DE9F041594F8AB03B78B12B61
:102940006ED1FDF797FD80F00104E4B2554B04F021
:102950000104554DB3F87F32544EADF80030B54206
:1029600060D3002C00F09A801022002106A844F0C9
:10297000B9F94F4B0497DB1B05934E4B1A69002A9C
:1029800005DA4D4A5A6002F188325A601B69012308
:1029900000250222694604A88DF82430089541F0EC
:1029A00021FB022269464FF6FF703F4FFDF738FCCE
:1029B0000446B74245D30025022201A904A8ADF878
:1029C000045041F00FFB022201A92046FDF728FC2C
:1029D00040BA022202A9C043ADF8080004A841F0A1
:1029E00001FB079868B106ABC0F104022946184400
:1029F00044F078F9089818B906A904A8FFF710FF61
:102A000008909DF82430089823B12A4A136943F0AE
:102A100000431361B0FA80F040090AB0BDE8F081CC
:102A2000012493E7A9881C3555F8140CC1F30B0158
:102A30003CF01EF855F8043C1B68834218BF012483
:102A40008DE7B7F8048002A904A88DF80D50C8F3EB
:102A50000B081C3708F10603ADF8083037F81C3CAA
:102A6000C3F30B021B0BADF80A2006228DF80C30C5
:102A700041F0B8FA062202A92046FDF7D1FB044630
:102A800057F8141C424604A841F0ACFA204657F807
:102A9000141C4246FDF7C4FB04468AE70120BCE74C
:102AA000004000087883050864B8060878C1060865
:102AB00000800008003C02402301674510B51B4C14
:102AC000FFF7C4F80122D4F83C3884F8E42803F274
:102AD000DC53C4F83C38FFF72DFF10B9FFF72AFF8D
:102AE00060B1134B1B78B12B02D1FDF7C3FC78B951
:102AF0000A21052008F078FC3CF0FCFDFFF71AFFE6
:102B00000028EED10A21052008F06EFC3CF0F2FD11
:102B1000084A00230121126884F8E43884F8551823
:102B200084F8E538C4F83C2810BD00BFF0650120EA
:102B3000004000082C1D012001230B4A10B50B4C4E
:102B400082F81C37A375FFF7B9FFFFF795FC41F238
:102B50000242FF230E20A4F8802884F88238BDE8C2
:102B600010400CF03DB800BFC41E0020F0650120ED
:102B700090F88730F7EE002ADFED695A002103EE66
:102B8000903A90F88B3006EE103A90F88930F8EED3
:102B9000E33A04EE103A90F88A30B8EEC66A04EED2
:102BA000903A90F88D3063EEA57A03EE903A26EED7
:102BB000256AB8EEC44AF8EEE44AF8EEE33A26EEA7
:102BC000276A24EE254A64EEA54A63EEA53A24EE70
:102BD000064A64EEA74A63EEA73AF0B5514D0626C1
:102BE00000F1660EA5F10C0CB7EE005A06FB01F2DF
:102BF00090F88670AC180244F0EE456A15E00129A1
:102C000004F1060402F10602EED190F8883007EED6
:102C1000903A90F8903006EE903AF8EEE77AF8EEB7
:102C2000E66A27EEA55A66EEA56A237866EE867AEE
:102C300007EE103AB8EEC77A27EE277AFDEEC77A8C
:102C400017EE903A66EE847AFA2BA8BFFA2323EAAD
:102C5000E3731372637807EE103AB8EEC77A27EE83
:102C6000277AFDEEC77A17EE903AFA2BA8BFFA231F
:102C700023EAE37353725CF8213007EE903A002B9D
:102C8000F8EEE77A49DDA37807EE103A90F88C3039
:102C9000B8EE477A03EE103AB8EEC33A37EE677AE9
:102CA00023EE253A87EE272AB0EE627AA2EE037A67
:102CB00064EEA77A66EEA36A67EE857A27EE877AD6
:102CC000FDEEE77ABDEEC77A17EE103AFA2BA8BFF1
:102CD000FA2323EAE373937217EE903AFA2BA8BF14
:102CE000FA2323EAE3730EF801300131A38807EEDB
:102CF000903AF8EEE77A67EEA67AFDEEE77A17EEFD
:102D0000903AB3F57A7FA8BF4FF47A738F4223EAE3
:102D1000E3739381BFF673AFF0BDB7EE007AC7E7F8
:102D20000AD7233C0886050890F88E306BB3B0F8BC
:102D30005A308BB190F88F20642102EB8203C3EBF1
:102D40000313B3FBF1F3A0F85A30962312FB03F3FD
:102D5000B3FBF1F3A0F85C3043884BB190F88F30AF
:102D6000642203EB8303C3EB0313B3FBF2F343804F
:102D7000B0F846304BB1962290F88F3013FB02F337
:102D80006422B3FBF2F3A0F84630704790F821308C
:102D90004BB3438B83B190F82230FA22642113FBAA
:102DA00002F203EB8303B2FBF1F2B3F57A7F4283C5
:102DB000A8BF4FF47A738383838843B1FA2290F8D3
:102DC000223013FB02F36422B3FBF2F38380C38847
:102DD0004BB190F8223003EB8303B3F57A7FA8BFA1
:102DE0004FF47A73C380704770B50B4C002504F51F
:102DF000247694F8863013B12046FFF7B9FE2046BA
:102E00000135FFF791FF3046FFF7C0FF042D04F1B5
:102E1000A404EED170BD00BF38670120034BD3F886
:102E2000E80808B106F096BE704700BFF0650120C3
:102E300008B50B4605490246D1F8E80828B104490F
:102E4000FEF71CF8BDE80840E8E708BDF065012082
:102E5000BD080108024B0146D3F8E808FDF730BD74
:102E6000F065012008B504460848FFF7F3FFFFF7B7
:102E7000D5FF074B186E0BF031FE07F0A1FF012CB8
:102E800001D13CF037FCFAF7F5FD00BF6D320608C2
:102E9000F06501200048DDE7B63D06080CB4C30626
:102EA00007B500D561B905A904980191FFF7C0FFE6
:102EB000FFF7F0FF012003B05DF804EB02B07047AC
:102EC0000020F8E708B5FFF7C5FFBDE80840E1E7D7
:102ED00010B504460348FFF7BDFF2046BDE810408B
:102EE000F0E700BF793206080948002408B5FFF76B
:102EF000EFFFFFF793FF074B83F8EC48C3F8EC496B
:102F000083F8F0491FF00AFF2046FFF7ABFF00BF30
:102F10007E320608F0650120034B0146D3F8E8082D
:102F200008B106F003BE7047F06501200CB407B588
:102F300010F020000BD079B92320FFF7EDFF05A991
:102F400004980191FFF774FFFFF7A4FF012003B07D
:102F50005DF804EB02B070470020F8E70FB407B546
:102F600004A951F8040B0191FFF762FF03B05DF86B
:102F700004EB04B0704730B52B4885B0FFF76AFF0B
:102F80002A4B1B7923B92A4805B0BDE8304099E7A0
:102F9000FBF7B6FC08B92748F6E7FBF7D1FC08B900
:102FA0002548F1E7254B1B68DB6998470028F7D0D7
:102FB000FBF7BEFC02680446037D81795208407C21
:102FC000E51D0C34029020790190E08800901C48A7
:102FD000FFF7C4FF15F8010BFFF79EFFA542F9D1DB
:102FE000184C1948FFF736FF6378022B06D007D933
:102FF000032B10D11548FFF72DFF0CE01448FAE71A
:1030000004F580541348FFF725FF94F8E437022BAA
:1030100005D0032B05D005B0BDE830403AE70E4897
:10302000E9E70E48E7E700BFA53206089C29012022
:10303000AF320608BE320608CC320608281D012031
:10304000DB320608982D01200933060819330608DB
:103050001F3306082C330608323306084B330608A4
:103060000FB407B504A951F8040B0191FFF7E0FE76
:10307000FFF710FF03B05DF804EB04B070472DE9D3
:10308000F041037903F0E002402A50D004D85AB14D
:10309000202A29D0BDE8F081602A4BD0802AF9D1BE
:1030A00082794179254812E003F00703052B16D8F1
:1030B000DFE803F0101510150309D0F805102048BB
:1030C000BDE8F041CCE7D0F8052051421D48BDE8ED
:1030D000F041C5E7B0F80720B0F80510F6E7B0F901
:1030E0000720B0F90510F1E746790024164D17487E
:1030F00005EBC605FFF7AEFE012395F8A872A742BF
:1031000002D8BDE8F041C5E6D5F8A4624FEA8408CC
:1031100056F824204AB113B90D48FFF79BFE56F824
:1031200008100C48FFF71AFF00230134E7E7417944
:103130000948C5E70948BDE8F04191E7AC33060806
:103140005D33060873330608788305088A3306085A
:1031500070360608C64606089B330608C3330608C1
:103160000249034801F521610EC979E70070F01F9B
:10317000DB33060810B57521044623F0E7F8014655
:103180000948FFF76DFF1A21204623F0DFF80146BA
:103190000648FFF765FF1B21204623F0D7F80146BC
:1031A0000348BDE810405BE7EF3306080234060829
:1031B0001534060838B50C4D95F8DB0310F0FD0406
:1031C00005D10A48FFF74CFF2046FFF7D3FF95F8DB
:1031D000DB33013B012B06D80548FFF741FF0120F7
:1031E000BDE83840C6E738BDF06501202834060840
:1031F00033340608C04BC1491A68C14B2DE9F04F62
:10320000C04C93B08046C048C04DC14FDFF82893F2
:10321000B2FBF3F2FFF7A2FEB4F8F2294FF47A738F
:103220000A20B2FBF3F103FB1122B4F9F43992B294
:10323000B2FBF0F2B748FFF713FFB74AB749B848F7
:10324000FFF78CFEFFF726FEA17DB64A05EB810154
:10325000B54BB648D31AD1F87C14A288FFF700FF0B
:10326000B348FFF7F7FD94F8F619B248FFF776FE7A
:10327000B148FFF7EFFD94F8F719B048FFF76EFE7D
:10328000FFF708FEAE48FFF7E5FD00210A4694F877
:10329000F7334E1C0B4113F0010F08D012B1484612
:1032A000FFF7D8FD31463846FFF758FE0122072EBA
:1032B0003146ECD1A34E96F86A1506F5EC7306F18B
:1032C0003C02012918BF134693F8DC30032B02D0CF
:1032D0009D48FFF743FE9D4B96F86A15A3F5CE7205
:1032E000012918BF134693F8DC30012B02D198480E
:1032F000FFF734FE954B96F86A15A3F5CE720129B7
:1033000018BF13461B695B7B012B02D99148FFF75D
:1033100025FEDFF8AC92FFF7BDFD0027D4F8F839A1
:1033200009F1200A039359F8041B29B3012303FA76
:1033300007FB039B1BEA030F1CD01BF01F0F19D0C8
:10334000854B5AF82720D85D52F8202037B18348A2
:10335000CDE90412FFF77EFDDDE904128048FFF796
:10336000FDFDBBF1020F05D196F83D1711B17D4867
:10337000FFF7F4FD0137D6E7FFF78CFD94F8001A4C
:10338000D4F8FC2905EB81017748137AD1F8B814F9
:10339000527AFFF765FE75497548FFF7DFFD7549FD
:1033A0007548FFF7DBFDFFF775FD744B744819682E
:1033B0004FF47A73B1FBF3F1FFF7D0FD07A8FEF7E6
:1033C00015FB38B107A90AA840F00AFF0AA96D4801
:1033D000FFF7C4FDFFF75EFDD4F88C2A002A00F049
:1033E000F18007EE902ADFED686AB8EEE77AC6EE64
:1033F000877AFDEEE77A17EE903A644FB7F8CC0083
:1034000058B107EE900ADFED606AF8EEE77A86EED3
:10341000A77AFDEEC77A17EE900AD4F80C1A59B1C4
:1034200007EE901ADFED586AF8EEE77A86EEA77A93
:10343000FDEEC77A17EE901AB6F87867642ECDE9DC
:10344000000131465248A8BF6421FFF709FE97F8F2
:10345000CE3097F8CF2005EB8303B7F8D0104D4856
:10346000D3F8CC34FFF7FCFDB7F8E0104A4889B236
:10347000FFF7F6FD49494046FFF77DFD4848FFF755
:10348000E9FCD4F880351B0640F1CC8097F8003178
:10349000032B8CBF43484448FFF7DCFC94F8C0344E
:1034A000022B40F091804148FFF7D4FC97F800319F
:1034B000042B00F2AE803E48FFF7CCFC97F81031A9
:1034C000002B00F0AD8005EBC303D3F82415394879
:1034D000FFF744FDFFF7DEFC3748FFF7BBFC012692
:1034E000D4F8C448354F002C40F0A080FFF7D2FC40
:1034F00013B0BDE8F08F00BF341D0120463406082C
:1035000040420F00F06501204B340608788305081F
:10351000063506085E340608000001200008000099
:103520007F3406080080000800400008A334060825
:10353000D2340608E4340608EC340608EE340608F3
:10354000F6340608C41E00200F3506089C20002013
:10355000173506081C350608B80301207036060822
:10356000243506082A3506082E3506084035060893
:10357000613506086F350608753506082C1D0120D3
:103580007B3506089535060800247449E876012045
:10359000A8350608EE35060815360608C64806089A
:1035A000243606082A360608363606084636060841
:1035B000CA5F0608833606089F3606088F36060857
:1035C000FC870508134618E702200BF0BDF90646F4
:1035D00008B91E4868E72FF0E1F996F9041005EBE9
:1035E00080000131D0F8E0241948FFF7B7FC94F8C7
:1035F000C334012B04D11748FFF72CFC164853E7BE
:10360000B379164805EB8303D3F8E014FFF7A6FC63
:10361000F4E794F8C2340BB911484DE711484BE771
:10362000114954E71148FFF715FC53E794FAA4F346
:103630003846B3FA83F306FA03F205EB8303D3F8B3
:10364000581524EA0204FFF789FC4CE74C360608BB
:10365000563606086A3606086F3606083D400608E4
:1036600073360608B33206083E3406089336060859
:103670002DE9F04FDFF86C8199B098F80B30002BF2
:1036800000F093804E4800254E4EDFF85CB1FFF706
:1036900019FC2F46DFF85491DFF854A10BA9E8B2CA
:1036A00018F0CCFA9DF83430002B53D0139C54B151
:1036B00007EE904A9FED440AF8EE677A80EE270AFB
:1036C00042F024FD04460B9A29465846FFF746FC73
:1036D000109A002A6BD002FB04F04FF47A73B0FB0F
:1036E000F3F30993DDF848C0BCF1000F61D00CFB87
:1036F00004F142F21073B1FBF3F1082D98F80B308E
:1037000018BF7F18002B56D017984FF47A7E0A23E3
:10371000079015980690169805901198B0FBFEFE3C
:10372000CDF810E00998B1FBF3FE03FB1E11CDE9C3
:1037300002E10999B1FBF3F103FB1100BCFBF3F3C8
:10374000CDE9001021465046FFF78AFC0023B36202
:10375000C6E90D33013540361F2D9FD198F80B3047
:1037600003B31A4C4FF47A731948D4E94512B1FBEC
:10377000F3F3D208D4F81C11FFF772FC0A221548A3
:10378000B7FBF2F102FB1172FFF76AFC124B1B78D8
:10379000432B04D11148D4E94821FFF761FC0023F1
:1037A000C4F81C3119B0BDE8F08F0D486BE70992E1
:1037B00098E76146A1E721464846FFF751FCC5E777
:1037C000B5360608F46F01208096184BE876012084
:1037D0005C3706087C370608391D0120A03706082B
:1037E00013370608F06501201D37060862460608F3
:1037F0002C37060813B52948FFF72CFB284B93F804
:103800003534002B48D02748FFF75CFB18F098FFB1
:1038100080B1254B254893ED280A8DED010AFFF76D
:1038200019FB234B9DED010AB3F8CC303BBB21487B
:10383000FFF748FB204C2148B4F81418FFF78EFB23
:1038400094F8103813B31E48FFF73CFBB4F818186F
:103850001C48FFF783FB94F81238CBB11848FFF7E8
:1038600031FBB4F816181848FFF778FB94F81138B4
:1038700083B1134802B0BDE81040FFF723BB42F00C
:1038800045FC81B21148FFF7EBFBD3E71048DBE7BB
:103890000F48E4E70E48EDE70E48EBE7CA370608A5
:1038A000F0650120E037060840260020E7370608CB
:1038B000E876012001380608C41E002010380608EA
:1038C00030380608403806085A3806080B3806080B
:1038D00039380608F97806080EB403B503AA52F879
:1038E000041B0192FDF712FD064BD3F8E8281AB924
:1038F0000549986EFCF7E4FF02B05DF804EB03B0F5
:10390000704700BFF0650120B63D06082DE9F0477D
:1039100098460B7981460F4603F0E0041646402C8A
:1039200031D10024674DDFF8A081DFF8C09122E09B
:103930003B7903F00703013B042B04D8DFE803F0D5
:1039400006080B0E2000315D28460AE03157FBE7E0
:1039500036F81410F8E736F91410F5E756F8241085
:103960004046FFF7FBFA7B79013BA34202DD484664
:10397000FFF770FA01347B79A342D9DCBDE8F08708
:1039800056F82410E0E703F00703052B58D8DFE8CA
:1039900003F0030C141619313578602C5ED045D82D
:1039A000002C66D0202C7CD0E8E796F90050602CE3
:1039B00054D03BD8002CF5D148E03588EDE7B6F976
:1039C0000050F4E7D6F800A0202C554669D02BD83B
:1039D000002CD3D151463C48FFF7C0FAD7F8051068
:1039E0008A4518D8B8F1000FC8D03848BDE8F0476C
:1039F000FFF7B4BA202C356853D015D8002CBDD1B0
:103A000029463048FFF7AAFAD7F80510A94202DB89
:103A10004B42AB42E6DDFFF73DFA2B463A6848469B
:103A20002B49BDE8F04757E7602C17D0802CA5D173
:103A30003178284B2848002914BF31461946D5E76C
:103A4000202C2DD007D8002C98D12546B7F9054059
:103A5000B7F9076011E0602CE8D100257B7945FAC1
:103A600003F3DB07BDE8F0474CBF1C481C48FFF7D9
:103A700075BAB7F80540B7F8076029461148FFF74F
:103A80006DFAAC42C7DCAE42C5DBB8F1000F3FF4C3
:103A900075AF324621461348BDE8F047FFF75EBADE
:103AA00000257A79104B03EBC20393F8A8229542C4
:103AB000B1DAD3F8A43253F82500BDE8F047FFF798
:103AC000C9B900BF87330608703306087A3806087C
:103AD000803806085A600608C6460608D833060825
:103AE000F97806082F41060878830508EC340608A3
:103AF00013B50446084601920091FCF781FF024687
:103B00002046DDE9001302B0BDE81040FEE60EB429
:103B100003B503AA52F8041B0192FDF7F7FB054B0E
:103B20000549986EFCF7CCFE02B05DF804EB03B0DB
:103B3000704700BFF0650120B63D06080246014906
:103B4000E5E700BF9A380608154BD3F828312DE970
:103B5000F041044688B0F3B11A6804A91846D56A42
:103B60006A46A847064688B104AC6D460027DFF8D0
:103B70003C80013735F8022B34F8021B4046FFF732
:103B80006FFABE42F5DC08B0BDE8F0810549204679
:103B9000FFF7BDFFF7E7044908B0BDE8F041B6E71D
:103BA000E8760120CB380608E3380608B138060865
:103BB00013B504460846019140F082FD024670B1FB
:103BC0000D2804D10199094843F0B9F938B1074BE0
:103BD0002046074A074902B0BDE8104097E703496D
:103BE000054802B0BDE81040FFF73ABAC8EC050836
:103BF000EA380608F53806081F39060813B50446E2
:103C00000846019140F05CFD0199024668B1042824
:103C100003D1094843F093F938B1074B2046074ACE
:103C2000074902B0BDE8104071E70349054802B0FA
:103C3000BDE81040FFF714BAC0EC05082D3906089E
:103C4000F53806083D3906082DE9F04300279BB0FA
:103C5000064608460C4640F033FD05461C22394610
:103C600002A8019743F03EF825B3402D07D040232A
:103C70002A46384930461BB0BDE8F04347E70DF10E
:103C8000040804F1400902222146684643F06BF91A
:103C90000023102209A968468DF80270FDF7EEFC9A
:103CA000099B0DF10202934222D1023408F8010B64
:103CB000A145E8D100213D220AA8099143F012F85C
:103CC000002D3AD0244C257ED5B1202204F11C01D0
:103CD00001A842F0DDFF98B104F11C0109A8FDF72D
:103CE000EBFB09AB1D4A30461D49FFF710FF04E00E
:103CF0001A7830461B49FFF70AFF1BB0BDE8F08376
:103D000094F86430CBB9C5B901AD174C0FCD0FC4D1
:103D100095E80F0084E80F00144B012209A8A4F1D4
:103D2000100183F82C21FDF7C7FB1148FFF7D0F8ED
:103D300009A91048FFF794F9DFE70C4B93F82C31F1
:103D40001BB9054B1B7E002BF2D0074909A8FDF7D4
:103D5000B3FBEDE750390608F06501208E390608FF
:103D6000F5380608723906080C660120E87601204D
:103D700098390608A73906082DE9F74F394F8346C9
:103D800008460D4640F09CFCD7F87C950446B8B92F
:103D9000354D0126354F3648FFF75CF855F8041BC2
:103DA00049B106FA04F313EA090F02D03846FFF7C7
:103DB000D5F80134F2E703B0BDE8F04FFFF76AB879
:103DC00002462C492846FDF709FC78B9264C2A4DB5
:103DD0002A48FFF73FF854F8041B0029EBD00B7872
:103DE000002BF8D02846FFF7B9F8F4E72B782D2BF5
:103DF00011D10135013C4FF0010A1B4B002653F84D
:103E0000048BB8F1000F09D12A461D49584603B06A
:103E1000BDE8F04F7BE64FF0000AEEE72246414650
:103E200028460193FDF7DAFB019BC0B90123B3409B
:103E3000BAF1000F0DD029EA03031248C7F87C3508
:103E4000FFF708F841460C4803B0BDE8F04FFFF714
:103E500007B949EA03030C48C7F87C35F0E7013697
:103E6000CDE700BFF065012038890508BE39060896
:103E7000B4390608183706088F360608C23906080E
:103E8000CD390608DE390608E73906082DE9F74F6F
:103E9000814608460E461746984640F011FC0446F7
:103EA000E8B9404D4048FFF759F820460AF02AFB90
:103EB0003B68184206D020460AF036FB01462846E9
:103EC000FFF74CF80134182CEFD13B6813B9374891
:103ED000FEF7C0FF03B0BDE8F04FFEF7DBBF0246C0
:103EE00033493046FDF77AFB0546A8B92C46314DDB
:103EF0003148FEF7AFFF20460AF004FB10EA080F36
:103F000006D020460AF010FB01462846FFF726F8A7
:103F10000134192CEFD1DDE733782D2B2AD101366E
:103F2000013C012548F080734FF0000A0193504690
:103F30000AF0FAFA2246834601463046FDF74EFB68
:103F400018BB50460AF0DEFA019B03421DD09DB11A
:103F5000BAF1180F02D03B6840EA03081748C7F8C7
:103F60000080FEF777FF5946124803B0BDE8F04FD6
:103F7000FFF776B80025D5E7BAF1180F02D03D68F3
:103F800025EA00050E483D60EBE70AF1010ABAF1A7
:103F9000190FCCD132460B49484603B0BDE8F04F6B
:103FA000B5E500BF8E360608EF390608F939060870
:103FB000183706088F360608C2390608DE390608A3
:103FC000E7390608CD39060840F20223004A5DE7CA
:103FD0007C6C01206FF07F43004A57E7746C01202E
:103FE00010B5044621F0C2FD20B920460449BDE8C1
:103FF00010408CE50348BDE81040FFF731B800BF22
:10400000003A06080F3A060870B5054608461646F7
:10401000FDF7D8FB0D4B044693F89025904205D24E
:1040200001460B48FFF71CF8204670BD2EB1FF2853
:1040300003D10848FFF714F8F6E7013A0649284685
:104040004FF0FF34FFF763FDEEE700BFC41E002012
:104050001A3A06082B3A06083E3A06082DE9F04FB0
:10406000074691B082480E46824DFEF7F9FF0023C5
:1040700081494024062285F834313046012391F8E5
:104080009015C5F830D185F8354106F015FF0A20A6
:1040900007F04EF995F834310C2BDAB240F2E48097
:1040A0009DF80C50FE2D30D0FF2D0BBF15240F2492
:1040B00001260026944240F0D780611E6846C9B2AE
:1040C00034F018FB04F140030DEB030414F8413CF9
:1040D000834240F0C48006F1FF389DF80D305FFA4E
:1040E00088F8B8F1010F12D903F01F075C09613796
:1040F0006248FEF7AFFE022E6AD0013C042C65D860
:10410000DFE804F00B5E606462000226D2E79DF8EF
:104110000E701D469DF80F40EAE759486C464FF077
:10412000000ADFF8B891FEF7CDFEDFF8B4B15548CC
:10413000FEF790FE0AF1010A14F8011B4846FEF74B
:104140000DFFBAF10C0F49D1FEF7A4FE022E4FD09D
:1041500064223B464C48B5FBF2F102FB1152C9B256
:10416000D2B2FEF77DFFB8F1010F71D8474A484B34
:104170009DF810104748002914BF11461946464DB6
:10418000FEF76EFF9DF81110444B4548002914BFFF
:1041900019462946FEF764FF022E59D19DF81240B8
:1041A0004048FEF757FE4CB3FF2C37D00A223E485A
:1041B000B4FBF2F102FB1142D2B2FEF751FF20E054
:1041C0003A48ABE73A48A9E73A48A7E73A48A5E7AB
:1041D00000230DF11F008DF83F309FE7374B03FBA5
:1041E0000AF2B2F1553FA5D85846FEF733FEA1E7D3
:1041F0003A4629463248FEF733FFB7E72846FEF72E
:1042000061FE9DF813402F48FEF724FE44B1FF2CB9
:1042100021D021462C48FEF723FF04E02B48EEE78F
:104220001D48FEF74FFE0DF1130500241A4E274FCF
:10423000DFF8688015F8013F7BB1FF2B0CBF3A46D1
:104240004246214601342248FEF70AFF042CF1D1F0
:1042500011B0BDE8F08F1D48E3E73246F1E71D4994
:104260003846FFF754FCF3E71B48FEF72BFEEFE759
:10427000843A0608E8760120C41E0020953A060814
:10428000A03A0608C63A0608D83A0608643A06086C
:104290006D3A06080F3B0608743A060805480608FA
:1042A000263B06082D3B0608413B0608A73A0608B0
:1042B000AF3A0608B73A06083E340608ABAAAAAADF
:1042C000F43A0608493B060887330608783A060898
:1042D000593B0608643B0608743B0608653206082D
:1042E0005A6006082DE9F84F07460C46DFF8A4800F
:1042F000DFF88490DFF8A0A0204640F0E1F9064600
:1043000060B91D4B1D4893F80C241D4B03EB820331
:10431000D3F83816BDE8F84FFEF7A2BE0246414674
:104320002046FDF75BF960B1DFF85CB000255BF873
:10433000041BB1B9224638461249BDE8F84FFFF7D1
:10434000E6BB114C114D1248FEF784FD54F8041BD6
:1043500019B12846FEF702FEF8E7BDE8F84FFEF770
:1043600099BD324620460135FDF738F90028DED1E7
:10437000544689F80C54BFE7F06501207D3B0608E0
:1043800078830508CD390608B48905088F360608F4
:10439000C239060818370608C648060838B50D465B
:1043A0000446052219492846FDF718F968B9184B43
:1043B00093F86C2022B9012183F86D2083F86C10EA
:1043C0001448BDE83840FEF77DBD03221249284657
:1043D000FDF704F9A0B90E4D95F86C3063B195F86E
:1043E0006D304BB10D492046FFF791FB002385F856
:1043F0006C3085F86D3038BD0948FEF763FDF5E790
:1044000020460849BDE83840FFF781BB4947060808
:10441000F0650120873B0608AE4806089D3B06086C
:10442000D43B0608E83B0608F8B5174C054694F857
:104430006C307BB194F86D3063B11449FFF767FBC2
:1044400028461349FFF763FB002084F86C0084F8CA
:104450006D00F8BD0F4E96F82C7197B1207E0028A4
:10446000F7D10D4D06F59C740FCD0FC495E80F00E4
:1044700084E80F00012386F8733107F01BFA3846F1
:10448000E7E70120E5E700BFF06501209D3B060856
:10449000F73B0608E87601200C66012008B5FFF717
:1044A000C3FF50B1054B01229A75FEF707FB044884
:1044B000FEF70EFD0020FEF7D5FC08BDF0650120DB
:1044C000153C060808B5034610462AB1DB0600D5A0
:1044D00011B1FEF7FDFC002008BDF8B50D4E0546F4
:1044E00096F8643093B9F8BD25B12388C3F30B0364
:1044F0009D4204D0A288D4E9020142F07FFB1C3423
:10450000BC42F1D3002386F86430ECE7024C034F41
:10451000F6E700BFF065012064B8060878C1060818
:104520002DE9F04F164685B01A4682460191304675
:104530000021334CFFF7C6FF4FF0000906F01003CF
:1045400005460293FEF76AFC2379019A03F01803EB
:10455000934203D0002A48D1182B46D14FF00D0BBF
:10456000274B0BFB0933B3F80900FCF733FA8046FD
:104570002046FBF7FAFF0746D8E90221024401442E
:104580002046FBF7ABFF80F001012A460390C9B239
:104590003046FFF797FF0546DDE9022302B123BB52
:1045A000174A0BFB09FB52F80BB0B2060FD573B9D3
:1045B000594614480393FEF7D1FCD8F80820214649
:1045C000039B50463A44FFF7A1F9FEF763FC5946B6
:1045D0000D48FEF7C3FCD8F80C20002321463A44CE
:1045E0005046FFF793F9FEF755FC09F1010940F237
:1045F0006D230D349945A5D105B0BDE8F08F00BFFE
:10460000989D05081C3C06081D3C06080149FFF75B
:104610007EBA00BF273C060838B50C46054615494A
:104620002046FCF7B7FF30B9FEF7DEFB1248BDE8C5
:104630003840FEF747BC11492046FCF7ABFFA0B954
:104640000F4A82F8CE0182F8D60182F8720282F80F
:104650007A0282F8160382F81E0382F8BA0382F8FF
:10466000C20382F8F9030748E1E72846BDE838406D
:10467000CCE700BF363C06083C3C0608573C060821
:10468000F06501205F3C06082DE9F043064687B03F
:1046900008460C4640F014F8082844D1671E03ADC4
:1046A000073429463A46A84612F8010FFCF76CFF7A
:1046B00001F8010BA242F7D10023DFF880908DF8BA
:1046C000143017F8010FFCF75FFF05F8010BC1B2BA
:1046D0004846019142F00DFC20B10199284642F074
:1046E00008FC28B13046FFF791FF07B0BDE8F08322
:1046F000A742E6D11049404621F0C8F90E480823E8
:104700000E4910F8012B013B11F8014B02F1180280
:104710006A4402F80C4CF4D103A909488DF814300E
:10472000FEF79EFCE1E70028E8D0304607B0BDE880
:10473000F043FFF703BA00BF046A012028320608DD
:104740007B3C06082DE9F74F4FF0000B064601AA07
:1047500008462E495D4642F087FA01270446DFF8F5
:10476000BC80DFF8BC90DFF8A4A01CBBBBF1000F3D
:1047700028D1274C002D44D029462648FEF770FC4E
:1047800094F864300BB904F0FFFBFCF7B5F9002393
:1047900084F86D30FEF728FB15B12846FFF79DFE23
:1047A0009FB13046FFF740FE78B1FEF787F9002051
:1047B000FEF758FBBBF1000F0AD02046FDF702F8C8
:1047C00085B2C5B93046FFF721FF03B0BDE8F08FD1
:1047D00041462046FCF726FF80B949462046FCF7B3
:1047E00021FF0028EED05F4601AA5146002042F08A
:1047F0003BFA0446B9E74FF0000BF5E74FF0010B29
:10480000F2E70548FEF764FBBFE700BF4741060833
:10481000F06501208B3C0608AE3C0608823C060889
:104820008047060807B5009313460A460249FFF77A
:104830006EF903B05DF804FBC43C060820B10078B3
:10484000B0FA80F040097047012070472DE9F3412C
:1048500006460846FFF7F2FF0D46074670B10024F2
:1048600001A92046013439F0BDFC01463046FFF76E
:10487000EDFF122CF4D102B0BDE8F0810846FCF740
:10488000A1FFC4B2112C72D8681C3D4DFBF798FFF4
:104890008046E8B93B4B03EB440393F874118A1E3E
:1048A00051425141374B03EB440393F87421AA5C06
:1048B000002955D093F87531192040F2EE2100FB04
:1048C00003132146304802B0BDE8F041FEF7C8BBF3
:1048D0000178284642F00DFB78B1032C2B49A0EB60
:1048E000050394BF0022012202EB42020A4452FA5D
:1048F00083F393F8A876032F04D1304602B0BDE8C5
:10490000F04183E64046FBF75BFF08B3022FF4D18A
:10491000FCF758FF40F6CA0280B21A4B904203EBF4
:104920004403A8BF104640F2EE229042B8BF1046A2
:104930001922A0F2EE20B0FBF2F083F87501BB1E45
:10494000594259410F4B03EB440383F87471A9E7B3
:10495000022FF4D1304602B0BDE8F041FFF7EEB8C7
:1049600021460B4802B0BDE8F041FEF779BB1123A8
:104970003A460849304602B0BDE8F04152E700BF70
:1049800054010608E8760120DD3C06087883050816
:10499000ED3C0608FA3C06082DE9F04F024691B0BE
:1049A00008460B46FFF74AFF044628B1104611B0EF
:1049B000BDE8F04FFFF7C2B84FF0FF32274626465A
:1049C000DFF8E082DFF8E092DFF8E0A2CDE908202E
:1049D000A24A126E92F83810CDE90E02CDE90C1001
:1049E000CDE90A0007AA9E49184642F03DF905465E
:1049F00004944DB9089A0C9FBA4262D19948FEF7C7
:104A00002FFB11B0BDE8F08F062F12D8DFE807F0BA
:104A1000041E2328454C510051462846FCF702FE4F
:104A200078B14FF48060012409F08EFF90F90430D2
:104A3000089307AA8A490020013742F015F9054674
:104A4000D7E72846FCF7BEFE0890F2E72846FCF7B9
:104A5000B9FE0990EDE72846FCF7FBFD0A90E8E770
:104A600028463FF02DFE4146024605902846FCF7B9
:104A7000B5FD18B3059A49462846FCF7AFFD064632
:104A80000028D6D02846FCF79DFE04280646D0D93B
:104A900001467548FEF7E4FAB3E72846FCF792FEB4
:104AA00000230C900F93C4E72846FCF78BFE0D9073
:104AB000BFE72846FCF7CDFD0E90BAE7012304932B
:104AC000B7E7DFF8EC8151B2434613F9010B884296
:104AD00008D00135092DF8D1002101316348FEF7D6
:104AE000BFFA8EE701216248FEF7BAFA00237AB2D4
:104AF00018F9011B8A4200F00C810133092BF7D110
:104B00003A460121E9E7A7F11402534253410593C4
:104B100008AD002303F10108EB68A3BB95F900B0D1
:104B2000584609F0DDFED5F804A020B1D0F8009079
:104B3000B9F1000F5ED1BAF1000F19D14FF4614302
:104B40004FF0010A6B60AB680BB90323AB60002325
:104B5000D5F804905846029319462A7ACDE9009276
:104B60001A4609F042FFE86028B94146414891E7FA
:104B70004FF0000AE7E74A464146BAF1000F37D046
:104B80003D48FEF7EBF9B8F1020F05F110054FF0C3
:104B90000103BFD1059BDDF83C800B9D53B1374825
:104BA000FEF790F9D8F800301B6A1BB12A46344949
:104BB00040469847049B002B4ED03249324B142F6D
:104BC00018BF19463148FEF74BFA142F09D1049B40
:104BD00003B936B12B68DB691BB132462C49284634
:104BE0009847002C66D100224146284639F0AEFA9B
:104BF0002848C6E7C5F80C90BAF1000F25D0414609
:104C000025485246FEF7AAF95146484602F082FF6F
:104C1000D5F808A0BAF1000F0FD099F804209245FA
:104C20000BD0534641461D48FEF798F9D9F800309D
:104C30005FFA8AF148469B699847D9F82C30002BD7
:104C4000A1D00023C9F82C309DE7D9F808204146AF
:104C50001348FEF783F9DBE70B49B3E7F065012062
:104C600047410608383D0608203D06087C3E0608F8
:104C7000513D06085D3D0608793D0608303E0608B0
:104C8000157B0108023D0608C6480608593E06087D
:104C9000E50801089D3D0608B93D06080B3E0608DB
:104CA000E63D06081A3D0608FB3906080F3D0608D2
:104CB000268A05081C4F0026DFF874904FF0030A7F
:104CC00005F0DEFE052006F033FB99F89035B3427F
:104CD00089D917F801BBBBF1000F15D0584606F073
:104CE00057FC044680B1584605F0E8FD08B1A0F82D
:104CF00006A001210490F5F74FFFA379049813F063
:104D0000010F03D0F5F7D0F90136DEE7F5F7C6F964
:104D1000FAE73A4602210548FEF7A2F9099B002B63
:104D20003FF4F1AE0023F2E600260120513D0608D3
:104D3000C41E002010B5044608460B46FFF77EFD52
:104D400028B9032208491846FCF748FC28B9074847
:104D5000FEF7BEF80120FEF785F820460449BDE8BD
:104D60001040FEF7D4BE00BF8E3E0608923E0608F5
:104D7000E83B06082DE9F74F05460846FFF75EFDBC
:104D80000B46044618B9334A92F8987127B9284659
:104D900003B0BDE8F04F39E42646DFF8C880DFF8FD
:104DA000C89001AADFF8C4A018462B4941F05CFF67
:104DB00010B905F073FE08E056B9012201462846F5
:104DC000FFF722F9421C04461BD103B0BDE8F08F67
:104DD000FCF7F8FC2F28834636D80FB105F050FEBB
:104DE000BBF1060F14D01D4901235FFA8BF291F835
:104DF0009015E0B206F060F8002759464846FEF7E5
:104E00002FF901AA14490020013641F02DFFCFE708
:104E1000DAF880351B0113D5FF2C0FD0E1B22846FC
:104E2000FFF71CF9E8E701372846FFF717F90B4BA6
:104E3000F9B293F890258A42F5D8DDE70027F6E726
:104E40000748FEF73FF8D7E72F2241462846FEF7EE
:104E50005EFED6E7E876012047410608C41E002022
:104E6000003A0608C53E0608B43E0608F065012073
:104E70002DE9F04F064685B008460B46FFF7DEFCED
:104E8000044628B1304605B0BDE8F04FFEF756BEE7
:104E900003AA30491846274641F0E6FEA0460546DB
:104EA000DFF8C090DFF8C0A0DFF8C0B05DB92A4BD2
:104EB0003A46A1B2186E3AF0F9F968BB2749304674
:104EC000FEF725FE28E0B8F1000F06D0B8F1010F7B
:104ED00025D03046FEF732FE1EE028463FF0F0FBBC
:104EE0004946024601902846FCF778FB50B3019AE8
:104EF00051462846FCF772FB30B3019A59462846C2
:104F0000FCF76CFB10B3019A28461549FCF766FBC9
:104F1000F0B13046FFF77AFB05B0BDE8F08FBB1E5D
:104F2000294630465A425A41FFF76EF8421C044661
:104F3000F2D003AA0749002008F1010841F094FECD
:104F40000546B3E74746F4E70127F2E70227F0E713
:104F50000327EEE747410608F0650120F13E060809
:104F6000EE3E0608E53E0608E83E0608EB3E06086B
:104F70002DE9F74380460846FFF760FC0B460546DF
:104F800028B14046FEF7DAFD03B0BDE8F08301AA80
:104F90002D4918462F4641F067FE2E460446DFF89D
:104FA000A8907CB9022DECD1A7F57A73B3F57A7F7E
:104FB00021D94FF4FA634FF47A7224494046FFF73F
:104FC00031FCE1E74DB1012D10D001AA4946002086
:104FD000013541F049FE0446E3E7012221464046FF
:104FE000FFF712F8431C0646EFD1CDE72046FCF749
:104FF000E9FB0746E9E7164DB8B2D5F830385B68EB
:105000009847FF2EBCEEC00A0CD1F8EE407A95F816
:105010009025104BA24213DC10EE101A0E48FEF73A
:105020001FF8B1E70D4BF8EE407A10EE102A31462A
:1050300003EB86030A48C3ED677AFEF711F8A3E78E
:105040000134E3EC017AE5E747410608FF3F060833
:10505000C41E0020847801201C3F0608E876012049
:105060000F3F0608F8B507460846FFF7E7FBC8B14B
:105070001F4B5E6901363046344609F055FA054645
:10508000F0B90134192CA8BF0024204609F04CFACD
:105090000546A8B9B442F4D138461649BDE8F840EF
:1050A000FEF735BD0846FCF78DFB044609F03CFAD7
:1050B000054628B921461048BDE8F840FDF7D0BFA5
:1050C0000B4B5C6109F056FD2A4621460B48FDF763
:1050D000C7FF182C09D80A480C2101FB040090F8DE
:1050E000B806BDE8F84009F07BBD0020F9E700BF35
:1050F000AC0301202B3F06083F3F0608553F06083A
:105100007883050838B50446114D0846FFF796FB2D
:1051100068B1104B93F900104B1C06D10E4B197A55
:105120000E48BDE83840FDF79BBFC9B2F8E7084616
:10513000FCF748FB032804D8C0B2FDF721FB294641
:10514000E3E7204603220649BDE83840FEF7DFBC0E
:10515000C6480608AC030120F06501206E3F060832
:105160007E3F060838B50446114D0846FFF766FB3A
:1051700068B1104B93F901104B1C06D10E4B597AB4
:105180000E48BDE83840FDF76BBFC9B2F8E70846E6
:10519000FCF718FB032804D8C0B217F039FE2946E3
:1051A000E3E7204603220649BDE83840FEF7AFBCDE
:1051B000C6480608AC030120F06501206A3F0608D6
:1051C000793F0608444B2DE9F74FDFF824A1054647
:1051D0001A7A88468AF800205A7A93F864308AF856
:1051E00001200BB903F0D0FE00263C4CFBF784FCF9
:1051F000B1460D23394A4146734352F803B058462D
:10520000FCF710FA002841D0B9F1000F01D0FDF7EA
:1052100041FE59463248FDF7A1FE002221462846AC
:10522000FEF766FCFDF736FE237903F01803082B22
:1052300045D0102B48D02046FDF721FF274A0D23EB
:1052400003FB0623B3F80900FBF7C4FB0746D8B1FC
:105250002046FBF78AF90090D7E902210244014475
:105260002046FBF73BF978B9594601901D48FDF7F8
:1052700075FE019AB96828461346009A0A442146E9
:10528000FEF744FBFDF706FE09F10109013640F285
:105290006D230D349E42ACD10020FFF71EF9FF2391
:1052A0008AF800308AF80130B9F1000F11D1424676
:1052B0000D49284603B0BDE8F04FFEF728BC0B4966
:1052C0002846FFF71FFFB6E708492846FFF74AFFC1
:1052D000B1E703B0BDE8F08FF0650120989D0508A7
:1052E000213C0608993F0608CD390608C64806083D
:1052F000AC0301202DE9F74F074608460E463FF064
:10530000DFF9044620B1012825D132782A2A22D19A
:10531000B24E00254FF00D0BDFF8E092B24640F29E
:105320006D28AF48FDF7CEFD0BFB05F34846013570
:105330005AF80310FDF712FE221E3146384618BFF8
:1053400001220D36FEF7D4FBFDF7A4FD4545EBD158
:1053500003B0BDE8F08F3D21304641F0CAFD002882
:1053600000F0368101460A4611F8014D202CFAD092
:10537000921B0130814610F8011B2029FAD05FFAF8
:1053800082FA4FF00008DFF854B20D23524630463F
:1053900003FB08F10BEB01045BF801100091FCF733
:1053A0001DF90546002857D1009908463FF088F9B5
:1053B000824551D1267906F0E001402900F0CB80EA
:1053C0000ED8002956D0202900F09D803846854906
:1053D000FEF79DFB204603B0BDE8F04FFDF74FBE42
:1053E000602900F091808029F0D148463FF068F9AB
:1053F000E3790546A679DB070CD52046FBF700FBD1
:105400000378014633B12A46484641F098FD00280A
:1054100040F0D880002D00F0D580AE42C0F0D280A0
:105420000D23204603FB08B393F805A0FBF7E8FA29
:105430003246002141F056FCAA452CD82A466A493A
:10544000484641F07CFD30B32046FBF7D9FA2A46A6
:10545000494641F0D3FB1EE008F1010840F26D23FC
:10546000984592D132466149384603B0BDE8F04FC5
:10547000FEF74DBB06F00703042B1CD10B460A2296
:105480004846FCF7FBF8D4F80530014683429DD32B
:105490002046FBF7CBFA0D23554803FB08F85BF8D1
:1054A0000810FDF75BFD00222146384603B0BDE839
:1054B000F04FFEF71DBB052B0FD101230A224846F2
:1054C000FCF7DCF8D4F8053001468342FFF67EAFE6
:1054D0005B4283423FF77AAFDAE74846FCF772F95E
:1054E000B4F80550B4F8071016F0050FAAB28BB245
:1054F00001D02AB20BB29042FFF668AF98423FF754
:1055000065AF0146C4E765793A4A002602EBC50556
:10551000B246334695F8A8220092009AB24202D9C8
:10552000BAF1000F03D0002B3FF450AFB3E7D5F82A
:10553000A41251F8260060B149460193FCF72AF8FD
:10554000019B30B94FF0010A31462046FBF76EFA55
:1055500053460136E1E706F007066379013E009302
:10556000009BAB4297DD4846814610F8013B202B5B
:10557000FAD02046FBF744FA8246042E04D8DFE82E
:1055800006F0031010161F004846FCF71BF90AF836
:10559000050048462C2141F0ACFC013500F1010921
:1055A000DEE74846FCF70EF92AF81500F1E700237C
:1055B0000A2200214846FCF761F84AF82500E8E78E
:1055C0000123F5E732460C493846FEF7A0FAFDE61E
:1055D0003146384603B0BDE8F04FF3E5989D050825
:1055E000A93F0608F73F06085A600608CD390608A5
:1055F000EC3F060878830508BC3F0608213C0608F6
:105600002DE9F04F914689B00C461A46002180469C
:105610004D46FEF757FF00270646DFF8E0B0B9F128
:10562000000F69D029460622204641F031FB0028B0
:105630003246404613BF012100214FF0010A4FF0CE
:10564000000AFEF73FFF0646287813F05DFC07903E
:1056500010B3687913F058FC079B4FF461714FF059
:10566000190C5B79EA780793AB781CFB021295F86A
:1056700001E01CFB0313297900B14079CDF804E067
:10568000CDE90232079B5A46CDE9041000935146FA
:105690003B464046FDF74AFC207813F035FC079066
:1056A00010B3607913F030FC079B4FF461714FF039
:1056B000190C5B79E2780793A3781CFB021294F82B
:1056C00001E01CFB0313217900B14079CDF804E01F
:1056D000CDE90232079B5A46CDE9041000935146AA
:1056E0003B464046FDF7DAFB013706340635142FFA
:1056F00095D109B0BDE8F08FCA46CDE70540060850
:105700002DE9F041064686B008460F46FFF796F8A9
:10571000054638B100235C4901201A4606B0BDE8B1
:10572000F0416DE70846FCF74DF81328044600F3F6
:10573000A28006268DF81750544D4643781CFBF77F
:105740003FF8074670B1FCF73DF8C0B213F0F0FB2C
:1057500040B1AB19027983F8F0259DF81730013379
:105760008DF817303846FBF72BF8074668B1FCF781
:1057700029F80D2809D8062303FB045383F8F10503
:105780009DF8173001338DF81730DFF8FC80B11C1D
:105790000DF1170238464144FCF718F8FBF710F8F2
:1057A000074668B1FCF70EF8012809D8062303FB69
:1057B000045383F8F4059DF8173001338DF8173042
:1057C0003846FAF7FDFF80B1FBF7FCFFC0B213F0DB
:1057D000AFFB50B10623027903FB045383F8F52590
:1057E0009DF8173001338DF817309DF817200623E8
:1057F000042A2FD103FB04530022A3F8F4251AF046
:10580000B5FB06234FF4617603FB045595F8F005CC
:1058100013F07AFB95F8F32595F8F2751923804675
:1058200095F8F50513FB076713FB026613F06CFB95
:105830004379214698F80520039395F8F4351448E8
:105840000097CDE9016395F8F135FDF709FC06B045
:10585000BDE8F081052A05D103FB0453002283F83B
:10586000F525CCE7062ACAD0002308EB060248F843
:1058700006309380C3E713232A460649304606B014
:10588000BDE8F041FEF7CEBFE06B0120F0650120DE
:10589000054006081E4006082DE9F04F174689B05E
:1058A0001A460C46002181463D46FEF70BFE3A4E55
:1058B00007F16C038046DFF8E8B0079394F9041011
:1058C0000023364A92F90800884260D001330C3236
:1058D000092BF7D10C35079B0C349D42EED109B052
:1058E000BDE8F08F29460C22204641F0D1F900286E
:1058F0004246484613BF012100214FF0010A4FF0F4
:10590000000AFEF7DFFDEA7995F90430804606EBE0
:10591000820251464846D2F8E02404922A7A06EBE5
:105920008202D2F8E0240392AA7906EB8202D2F82E
:10593000E02402926A7906EB8202D2F8E024019216
:105940002A6800925A46FDF7F1FAE279514694F935
:105950000430484606EB8202D2F8E0240492227A10
:1059600006EB8202D2F8E0240392A27906EB8202CF
:10597000D2F8E0240292627906EB8202D2F8E024A7
:105980000192226800925A46FDF788FAA2E7002F9A
:10599000A8D1BA46D9E700BF78830508006B01207B
:1059A000244006082DE9F04707468AB00846FEF76E
:1059B00045FF044638B10023544901201A460AB075
:1059C000BDE8F04768E70DF11C0807904E1CC8E9D8
:1059D00001000846FBF7F6FE4C4B40B21A4693F91D
:1059E0000410814200F08A8001340C33092CF6D176
:1059F000002425463046FAF7E3FE064638B1013565
:105A000000230A22EDB21946FBF738FE07904FF04B
:105A10000009DFF800A13046FAF7D2FE064640B38F
:105A2000FBF7D0FE3A49002251F804CBD3B26045CF
:105A300003D00132102AF7D100230AEB8302D2F8F7
:105A4000E024904215D1B9F1020F1FD0B9F1030F34
:105A500021D05A1EB9F1010FD2B212D00B2A03D8AD
:105A60008DF821300135EDB209F10109B9F1040FCA
:105A7000D1D1052D15D838460AB0BDE8F047FEF75C
:105A80005DB8042AF0D88DF82230EBE7052BEBD86F
:105A90008DF82430E6E79A1E0D2AE5D88DF82330DC
:105AA000E0E798E807001B4B84E807009DF82320F7
:105AB000002103EB82020846D2F8E02404929DF80C
:105AC000242003EB8202D2F8E02403929DF82220E6
:105AD00003EB8202D2F8E02402929DF8212003EB2E
:105AE00082030D4AD3F8E0340193079B00939DF99C
:105AF0002030FDF7D3F90AB0BDE8F0870C2301256B
:105B00008DF8200003FB042474E700BF3C6A0120E9
:105B10005888050878830508244006082DE9F04FC9
:105B20008BB00C460021074608921A46FEF7CAFCC5
:105B30000026089D4FF019094FF46178DFF8A4B0F2
:105B40000990089B002B49D029460A22204641F0A3
:105B50009FF80028099A384613BF012100214FF011
:105B6000010A4FF0000AFEF7ADFC2A89099033467E
:105B700006925146EA88384605922A790492EA78D4
:105B80000392AA7819FB028202926A7819FB0282B8
:105B900001922A7800925A46FDF7C8F922893346C5
:105BA0000136514606923846E2880A350592227936
:105BB0000492E2780392A27819FB02820292627840
:105BC00019FB0282019214F80A2B00925A46FDF743
:105BD00065F91E2EB5D10BB0BDE8F08FDDF820A021
:105BE000DCE700BF414006082DE9F04380468BB05A
:105BF00008460F46FEF722FE044638B100236549E9
:105C000001201A460BB0BDE8F04387E70846FBF7D2
:105C1000D9FD1D28054600F3B3800A268DF82740DC
:105C20004643781CFAF7CCFD044630B1FBF7CAFDB9
:105C30009DF8273001338DF827302046564CFAF76F
:105C4000BFFD074668B1FBF7BDFD0D2809D80A2343
:105C500003FB054383F8BC019DF8273001338DF821
:105C60002730DFF83091711C0DF127023846494486
:105C7000FBF7ACFDFAF7A4FD074668B1FBF7A2FD00
:105C8000222809D80A2303FB054383F8BF019DF8A6
:105C9000273001338DF827303846FAF791FD074653
:105CA00068B1FBF78FFD0D2809D80A2303FB0543D4
:105CB00083F8C0019DF8273001338DF827309DF817
:105CC0002730062B0CD0002309EB0602404649F88A
:105CD000063053601381FDF731FF0BB0BDE8F08350
:105CE0000A260023384606FB0546A6F8C231A6F868
:105CF000C431FAF765FD074640B1FBF763FD9DF837
:105D00002730A6F8C20101338DF827303846FAF75C
:105D100057FD58B1FBF756FD0A2303FB0543A3F8D3
:105D2000C4019DF8273001338DF827301B4B4FF00D
:105D3000FF324FF461705A600A2202FB0542B2F84A
:105D4000C4310693B2F8C231059392F8C03104937E
:105D500092F8BF310393192392F8BE1113FB01018E
:105D6000029192F8BD1113FB010300210193084633
:105D700092F8BC310A4A00932B46FDF78FF8ACE746
:105D80001D232246074940460BB0BDE8F043FEF70D
:105D900049BD00BFA4780120E8760120AC030120B2
:105DA000414006081E4006082DE9F04F8046914606
:105DB0001F460C4616464FF0000BDFF820A12DEDD4
:105DC000088B95B094ED008AB5EE408AF1EE10FA9A
:105DD0007DD0D4ED019A94ED029AD4ED038AB9F105
:105DE000000F49D0D6ED00BA96ED01BAB4EE6B8A39
:105DF000D6ED02AA96ED03AAF1EE10FA6CD1F4EEFC
:105E00004B9AF1EE10FA67D1B4EE6A9AF1EE10FAFD
:105E100062D1F4EE4A8AF1EE10FA0CBF01210021A2
:105E20003A460D46404681F00101FEF74BFBB0EECD
:105E30006B0A074611A8FAF7CFFCB0EE4B0A0790A1
:105E40000EA8FAF7C9FCB0EE6A0A06900BA8FAF79A
:105E5000C3FCB0EE4A0A059008A8FAF7BDFC059904
:105E6000069A079B039040460291294601925246AA
:105E700000935B46FDF75AF8B0EE480A11A8FAF70E
:105E8000ABFCB0EE690A05460EA8FAF7A5FCB0EE29
:105E9000490A06900BA8FAF79FFCB0EE680A059035
:105EA00008A8FAF799FC069B059A00210390404642
:105EB0000292524610341036CDE900535B460BF186
:105EC000010BFCF7EBFFBBF1080F7FF47BAF15B0C4
:105ED000BDEC088BBDE8F08F0021A1E76440060807
:105EE0002DE9F74F07460D46DFF8A8A1DFF8A8B166
:105EF0002846FEF7A3FC064638B100235D49012081
:105F00001A4603B0BDE8F04F4EE705225146284639
:105F1000FBF764FBA0B9584B0022C3F8E822C3F892
:105F2000F822C3F80823C3F81823C3F82823C3F8BA
:105F30003823C3F84823C3F8582303B0BDE8F08FD3
:105F400004224E492846FBF749FB04462846002C0C
:105F500044D1FAF735FC80460028EED03EF0B0FB85
:105F6000474BC2B253F8049BB9F1000F07D12A4640
:105F70004449384603B0BDE8F04FFDF7C8BD494677
:105F800040460134CDE90023FBF728FB0646DDE956
:105F900000230028E6D1374A034600211546013385
:105FA00042F8101B082BFAD10BEBC404D4F8BCC088
:105FB000BCF1000F03D094F8B8E0764505DB494604
:105FC0003148324DFDF74CF892E70CEB061305EB28
:105FD000061401360FCB84E80F00EEE7FBF7F2FB67
:105FE000072804463DD82846FAF7EAFB064658B388
:105FF000FAF786F9204B012503EB041383EDBA0A67
:106000003046FAF7DDFB064638B1FAF779F91A4B54
:10601000013503EB041383EDBB0A3046FAF7D0FBDE
:10602000064638B1FAF76CF9134B013503EB04134C
:1060300083EDBC0A3046FAF7C3FB38B9384603B0E3
:10604000BDE8F04FFDF77ABD0546D9E7FAF758F9F4
:106050000948032D00EB041484EDBD0A3FF44DAF55
:10606000ECE7072332460A49384603B0BDE8F04F53
:10607000FEF7D8BBD0790120E876012078400608E9
:10608000B4890508CD3906087D400608C6480608CB
:106090001E4006081A3D0608788305082DE9F74FCB
:1060A00092460C461A46002181465646FEF70AFAE9
:1060B00000258046DFF864B0BAF1000F2CD03146DD
:1060C0000422204640F0E4FD00284246484613BF23
:1060D0000121002101270027FEF7F4F9738880468B
:1060E0005A46019339463AF82530484600932B46E4
:1060F000FCF71CFF63885A4639464846019304362C
:1061000034F8043B00932B460135FCF7C7FE042D01
:10611000D2D103B0BDE8F08F5746EBE787400608C1
:106120002DE9F34105460846FEF788FB0C46074675
:1061300038B10023334901201A4602B0BDE8F041CE
:10614000ACE731492046FBF725FA034668B92D4AEA
:106150004FF47A704FF4FA610133108051800432A9
:10616000042BF9D102B0BDE8F0812046FBF72AFBF1
:106170000328064641D82046FAF722FB074670B1AD
:10618000FBF720FB4FF0010804463846FAF718FBEE
:1061900048B9284602B0BDE8F041FDF7CFBC40F257
:1061A000EE248046F1E7FBF70DFBB8F1000FF0D0CD
:1061B000A4F2EE2240F2DC539A4203D8A0F2EE227F
:1061C0009A420AD940F6CA0340F2EE220F49284605
:1061D00002B0BDE8F041FEF725BB0D4B00210D4A92
:1061E00003EB8603A3F86843A3F86A033346CDE9BB
:1061F00000400846FCF752FEB4E703233A4606493E
:10620000E5E700BF507A01201A3D060898400608CD
:10621000E876012087400608FA3C06082DE9F04F91
:106220008FB08946174600211A4606460024FEF71D
:1062300049F90DF1240B0546DFF86CA059F824301C
:10624000594602A8029337F031FF57B357F824306C
:106250003046029A039393422A4613BF012100213C
:106260004FF001084FF00008FEF72CF904A905468D
:1062700003A837F01BFF04A923465246009130467D
:106280004146FCF753FE2346013452464146304610
:10629000CDF800B0FCF702FE202CCFD10FB0BDE846
:1062A000F08FB846EFE700BFA6400608F0B50746F6
:1062B00089B008460E46FEF7C1FA054638B10023FC
:1062C000194901201A4609B0BDE8F040A6E7084682
:1062D000FBF778FA1F2804461DD83046FAF770FA03
:1062E000014620462CF0DEFC78B103AE0E48314664
:1062F00000EB840037F0DAFE23460C4A2946284694
:106300000096FCF7CBFD09B0F0BD384609B0BDE8FA
:10631000F040FEF77BB91F232A460549384609B0ED
:10632000BDE8F040FEF77EBA607A0120A64006087C
:106330001E4006082DE9F04F924685B00C461A46DD
:10634000002181465546FEF7BDF800268046DFF85D
:106350006CB0BAF1000F2FD029460422204640F03D
:1063600097FC00284246484613BF0121002101271F
:106370000027FEF7A7F8EB7880465A460293394685
:10638000AB78484601932B8800933346FCF7CEFD4B
:10639000E3785A463946484602930435A378019378
:1063A00034F8043B009333460136FCF777FD102E9A
:1063B000CFD105B0BDE8F08F5746E9E7B0400608F9
:1063C000F0B5074685B008460E46FEF737FA054693
:1063D00038B100231C4901201A4605B0BDE8F04041
:1063E000A8E70846FBF7EEF90F28044623DC304601
:1063F000FAF7E6F9014620462CF0CCFBA8B104F1EF
:106400002002124B2946284603EB820393F87B2394
:10641000029293F87A230192B3F878330C4A0093EE
:106420002346FCF73BFD05B0F0BD384605B0BDE89E
:10643000F040FEF7EBB80F232A460649384605B070
:10644000BDE8F040FEF7EEB9E07A0120E8760120E1
:10645000B04006081E4006082DE9F04F87B01446EC
:106460001A46054603910021FEF72CF84FF000086C
:106470000646DFF820B106234FF0000903FB08F7BA
:10648000C037039BDB5D0493002C7FD0E35D28467F
:10649000049A05939A42324613BF012100214FF01E
:1064A000010A4FF0000AFEF70DF8059B06465A4612
:1064B00051462846CDE900934346FCF737FD049B3F
:1064C0005A46514628460137CDE9009309F10109A2
:1064D0004346FCF7E3FCB9F1060FD2D108F10108FD
:1064E000B8F1060FC7D1E427DFF8A8B0039BA7F1E6
:1064F000E40913F807A0002C4AD0E35D3246284691
:106500009A45049313BF012100214FF001084FF079
:106510000008FDF7D7FF049B06465A464146284629
:10652000CDE900930623FCF701FD01370623194A44
:1065300041462846CDE9009AFCF7B0FCEF2FD5D1B3
:10654000039B93F8EF70ACB194F8EF803246284685
:10655000474513BF0121002101240024FDF7B2FFAC
:1065600000230C4A2146009328460723CDF80480D7
:10657000FCF7DCFC0023074A21462846009307234A
:106580000197FCF78BFC07B0BDE8F08FA24696E7B9
:10659000A046CAE7C2400608F0B5054687B00846DF
:1065A0000B46FEF74BF9044638B100231C49012085
:1065B0001A4607B0BDE8F0404EE703AE194F02AAF5
:1065C0001849184640F050FBB8B1032C04D12846B6
:1065D000FDF7B4FA07B0F0BDFBF7F4F802AA46F8ED
:1065E000040B39460020013440F03EFBECE7324614
:1065F00021460D48FCF734FDECE7032CE7D1059B61
:10660000DDE903461A4601933146E0B22CF00CFB5B
:10661000019B0028EBD12846FDF7F8FFDAE700BF21
:10662000607A012047410608C24006082DE9F04F74
:106630000F46164689B04FF00009B8463446DFF8D9
:106640003CB11A4600210546FDF73CFF0790002E9D
:106650007CD021460C22404640F01AFB0028079AC5
:10666000284613BF012100214FF0010A4FF0000A14
:10667000FDF728FF94F90B2007904B4604925146F2
:1066800094F90A2028460392B4F908200292B4F93A
:1066900006200192B4F9042000925A46FCF746FC09
:1066A00098F90B204B4609F10109514604922846FE
:1066B00098F90A200C3408F10C08039238F9042CDC
:1066C000029238F9062C019238F9082C00925A46A9
:1066D000FCF7E4FBB9F1080FB9D10024DFF8A09072
:1066E0000C2303FB04FA9EB34FF00008012356F875
:1066F0000A2003FA08FB57F80A3053403BEA030329
:1067000014BF0121002112EA0B0F08D023464A468C
:106710002846CDF800800791FCF708FC079957F848
:106720000A301BEA030F06D023464A462846CDF816
:106730000080FCF7B3FB08F10108B8F10E0FD5D1CA
:106740000134082CCCD109B0BDE8F08FB246A7E7E0
:10675000B046012357F80A2003FA08F3134207D082
:1067600023464A4601212846CDF80080FCF796FBD7
:1067700008F10108B8F10E0FEBD1E1E7D6400608A9
:10678000EE400608F0B506468BB008460D46FEF70B
:1067900055F8044620B300233F4901201A460BB0A8
:1067A000BDE8F04042E72D2B03D0A3F13002092AC7
:1067B0004BD8052C05DD30460BB0BDE8F040FDF7A9
:1067C000BDB92846FAF7FEFF0AAB621C03EB44048E
:1067D00024F80C0C15F8013F303B092BFAD914466C
:1067E0002B78002BDFD1062CE5D1BDF81C20BDF99C
:1067F0001C30072ADFD8BDF91E10A1F5FA7292B23B
:10680000B2F5FA6F1AD8BDF92040A4F5FA7292B227
:10681000B2F5FA6F12D8BDF92270B9420EDCBC4253
:106820000CDBA1420ADCBDF924C00CF1640292B277
:10683000C82A03D8BDF92650112D11DD174930465D
:106840000BB0BDE8F040FDF762B9202B02D1013555
:106850002246C4E730460BB0BDE8F040FDF7D6BE97
:106860000C200F4A6DB200FB0322A2F86C14A2F8B0
:106870006E44A2F8707482F872C482F87354009166
:106880000021084A0846CDE903C5CDE90147FCF7D8
:1068900005FB0BB0F0BD00BF507B01200341060893
:1068A000E8760120D64006082DE9F04F89468DB0E4
:1068B000164600211A4607460024FDF703FEDFF8BE
:1068C000DCA00546C4EBC40309EB030259F803003E
:1068D000918840F3074892790890ADF824108DF81C
:1068E0002620B8F1000F53D0002E54D0F218F058E3
:1068F0009188937907220A9008A8ADF82C100AA96C
:106900008DF82E3040F0C4F900282A46384613BFCF
:10691000012100214FF0010B4FF0000BFDF7D2FDDC
:106920009DF82E3005465246069359469DF92D3066
:10693000384605939DF92C3004939DF82B30039332
:106940009DF92A3002939DF8293001939DF8283053
:1069500000932346FCF7EAFA9DF826305246594642
:10696000384606939DF9253005939DF9243004930C
:106970009DF82330CDE902839DF8213001939DF8E5
:106980002030009323460134FCF788FA102C99D16B
:106990000DB0BDE8F08FB346DEE700BF1941060831
:1069A0002DE9F04F06468DB00D469C4FDFF8A082D2
:1069B000DFF8A09228463DF083FE034630B9024638
:1069C000974901200DB0BDE8F04F6DE7052239462B
:1069D0002846FAF703FE0446C8B9924D01467022D4
:1069E00005F5996040F07EF9C5F86844C5F874442F
:1069F000C5F88044C5F88C44C5F89844C5F8A4444B
:106A0000C5F8B044C5F8BC440DB0BDE8F08F042211
:106A100041462846FAF7E2FD044638BB2846F9F716
:106A2000CFFE82460028EFD03DF04AFEDFF828B2C4
:106A300002465BF8041B39B92A467B4930460DB043
:106A4000BDE8F04FFDF763B85046CDE90012FAF704
:106A5000C5FD019A40B92046744D1DF02BFF0099E9
:106A60004846FCF7FDFAA5E70134E2E70722704942
:106A70002846FAF7B3FD074600287AD12021284698
:106A800040F037FA044670BB6A4D6B48FCF766FA73
:106A9000214601342846FCF761FA0E2CF8D1002477
:106AA000DFF8B891654FFCF7F5F9DFF8B4810C26F3
:106AB0000025DFF8B0A1214666434846FCF74EFAB0
:106AC0000123F2595E48AB400135134214BF4146E1
:106AD0005146FCF743FA0E2DF2D10134FCF7DAF9F6
:106AE000082CE4D190E704AC564D03AA554940F078
:106AF000BBF8002848D0022F11D1049A072A07D8E2
:106B000005990D2904D80378722B13D06E2B22D04F
:106B1000082300224C493046FDF784FE74E7FAF75B
:106B200051FE03AA44F8040B29460020013740F027
:106B30009BF8DEE70C203B4B00FB0233012000FA00
:106B400001F1D3F868040843C3F8680438493046B3
:106B5000FFF726FF58E7334B0C2000FB02330122DE
:106B600002FA01F1D3F8682422EA0102C3F868248A
:106B7000ECE72846002404AD324F03AA314940F027
:106B800073F8A8B1082C03D13046FCF7D7FF3BE7D8
:106B9000FAF718FE03AA45F8040B39460020013421
:106BA00040F062F8EDE729493046FCF7B0FF2BE7EB
:106BB000082CE9D1049B0F2BF5D8DDF814E0BEF1C9
:106BC000070FF0D8DDF818C0BCF10D0FEBD8079F08
:106BD00007F16402C82AE6D8089DFF2DE3D809987A
:106BE0006428E0D80A996429DDD88842DBDA0B9C56
:106BF000032CD8D8C3EBC3020A4B134483F8CD143B
:106C000083F8C8E4094983F8C9C483F8CA7483F8CF
:106C1000CB5483F8CC0483F8CE4498E71A3D060899
:106C2000B07B0120E8760120CD390608C648060869
:106C3000364106083E410608C7460608507B01203B
:106C40004341060847410608494106080341060832
:106C5000784006087D400608B48905088733060891
:106C6000014106082B4906082DE9F04F89B000269E
:106C70000C46002107921A460746B246FDF722FC51
:106C80004FF01909079D4FF46178DFF894B0069032
:106C9000079B3BB32946062220463FF0F9FF002818
:106CA000069A384613BF012100214FF0010A4FF028
:106CB000000AFDF707FC6A790690334619FB028249
:106CC0005146384605922A7919FB02820492EA78E5
:106CD0000392AA7802926A7801922A7800925A4620
:106CE000FCF724F9627933460136514619FB0282DA
:106CF000384606350592227919FB02820492E27821
:106D00000392A27802926278019214F8062B009204
:106D10005A46FCF7C3F80A2EBAD109B0BDE8F08F85
:106D20004F4106082DE9F04F074689B008468B46CB
:106D3000FDF784FD044638B10023544901201A466A
:106D400009B0BDE8F04F8FE7514B084693F810A704
:106D500093F8119793F8FA87FAF734FD0928054656
:106D600000F38B8006268DF81F404A4C46430BF1FA
:106D70000100F9F725FD834658B1FAF723FD0D28E8
:106D800007D8A31983F838059DF81F3001338DF813
:106D90001F305846F9F714FD834668B1FAF712FD23
:106DA000824509D3062303FB054383F839059DF883
:106DB0001F3001338DF81F305846F9F701FD824628
:106DC00068B1FAF7FFFC484509D8062303FB0543E1
:106DD00083F83A059DF81F3001338DF81F30504677
:106DE000F9F7EEFC814668B1FAF7ECFC804509D36F
:106DF000062303FB054383F83B059DF81F30013351
:106E00008DF81F30DFF88480311D0DF11F024846D8
:106E10004144FAF7DBFC9DF81F20062A0BD0002323
:106E200008EB0602384648F806309380FCF786FEE9
:106E300009B0BDE8F08F02FB05424FF461701923E1
:106E400092F83D1513FB0101059192F83C1513FBD7
:106E5000010300210493084692F83B35039392F80E
:106E60003A35029392F83935019392F838350A4A47
:106E700000932B46FCF712F8DAE70923224607496C
:106E8000384609B0BDE8F04FFDF7CCBC207C0120AE
:106E9000F0650120E87601204F4106081E400608F3
:106EA0002DE9F04F144689B00F461A4600210646D8
:106EB000FDF708FB0546002C00F0D58022783B78D2
:106EC0009A42024630460DBF4FF001084FF00008CD
:106ED00001210021FDF7F6FA23780546994A41463B
:106EE0003046FCF723F83B784146964A3046FBF79C
:106EF000D5FF002C00F0B980627830467B789A424A
:106F00002A460DBF4FF001084FF000080121002173
:106F1000FDF7D8FA637805468B4A41463046FCF7C0
:106F200005F87B784146884A3046FBF7B7FF07F102
:106F3000CA0304F1CA0B4FF0020904934FF0000A90
:106F4000822305933B78534500F39180002C00F099
:106F5000F28097F8EA30304694F8EA209A422A46BE
:106F60000DBF4FF001084FF0000801210021FDF78F
:106F7000A9FA94F8EA300546744A41463046FBF7D0
:106F8000D5FF97F8EA304146704A304607F1EC09E0
:106F9000FBF784FF002C00F0D08004F1EC034A469C
:106FA00004F1FC014FF001089A4633F802CB32F8A5
:106FB000020B844518BF4FF000088B42F5D188F0D2
:106FC00001012A463046C9B2FDF77CFA0821054680
:106FD0005046FAF751FA5E4A034641463046FBF7FF
:106FE000A5FF97F8EA104846FAF746FA584A0346CA
:106FF00041463046FBF752FF002C00F0A0804FF0D6
:10700000FC094FF0010807EB090104EB0900FAF74E
:10701000C1FA09F10409002818BF4FF00008B9F5BA
:107020008E7FF0D188F001012A463046C9B2FDF7C3
:1070300049FA082104F1FC00F9F762FC454A0346CD
:1070400041463046FBF772FF97F8EA1007F1FC0063
:10705000F9F756FC3F4A03464146304609B0BDE8C1
:10706000F04FFBF71BBFA0463DE7A04659E7059B45
:107070003B440693002C5CD0059B0698234419469C
:107080000793FAF787FA049B1A789BF800309A4224
:107090004CD1B0FA80F84FEA58184B4609F110026B
:1070A000F85AE15A0233884218BF4FF00008934261
:1070B000F6D188F001012A463046C9B2FDF702FA3E
:1070C000627804EB090105469BF81800FAF7A6F967
:1070D00002909BF8003041461F4A30460193079BBF
:1070E00000930AF10103FBF721FF049B07EB090161
:1070F0007A780AF1010A187E0BF1010B0793FAF76F
:107100008DF9079B4146049A09F110090290304617
:107110001B7801320193069B0492009353460E4A5A
:10712000FBF7BCFE059B093305930BE74FF0000806
:10713000B3E7A046D9E7A04623E7A04651E7A0461B
:1071400082E700BF684106087A410608A8410608A0
:10715000C0410608D74106088F4106082DE9F04FC7
:107160008FB004460846B04902AA3FF07DFD0646AE
:1071700040B903460246AD494120FFF791FE0FB0EA
:10718000BDE8F08FAA49FAF705FA074620BB02AA24
:10719000A5493FF069FDFAF715FB0828054606D911
:1071A00008233A46A3492046FDF73CFBE7E7A24CFB
:1071B00094F81037834202DC84F81057DFE7064664
:1071C00004F5E2673146384625F036FD013694F87D
:1071D0001037B342F6DCEFE798493046FAF7DAF9B0
:1071E0000546E0B902AA90493FF03EFDFAF7EAFAF7
:1071F0000828064603D908232A469149D3E78E4C2E
:1072000094F81137834202DC84F81167B7E7284607
:107210000135314636F022FF082DF8D1F4E78949CF
:107220003046FAF7B7F9074600BB02AA7E493FF09D
:107230001BFD0028A3D0FAF7C5FA0828054603D994
:1072400008233A468049AEE77B4C94F8FA378342EC
:1072500009DD014604F5E26025F038FD294604F514
:10726000E26025F041FD84F8FA5788E77749304617
:10727000FAF790F9054618BB06AE6F4BDFF8A891F8
:107280000146B0461022304693F8FA773FF02AFDC7
:10729000BD4202AA80F20E81494600203FF0E4FC84
:1072A00010B93A466A490EE1FAF78CFA013528F826
:1072B000020BEDE7674C96E80F0084E80F005EE7ED
:1072C00065493046FAF766F9054600283BD15A4B26
:1072D0000DF11808074693F8FA9746464F4502AA5B
:1072E00051494FF0000080F2F2803FF0BDFC0146B2
:1072F00010B94A465949E6E0B2464FF0000B032266
:1073000030463FF030FE30463DF0DAF9584502D8BD
:1073100001370436E2E79AF800000BF1010BFAF7A7
:1073200033F90AF8010BEEE74A464D49CBE04146F6
:1073300020460135043408F10408032225F066FCD8
:10734000AF42F4D11BE747493046FAF723F9054627
:10735000002840F0AC80384F02AA334997F81087D4
:107360003FF082FC00283FF40AAFFAF72BFA461EE2
:1073700001D4B04503DC434601223B4913E72A49C7
:1073800002AA00203FF070FC014600283FF4F7AE4F
:107390004FF000080DF10C09082203A88DF81480A5
:1073A000CDE903883FF0DFFD03A83DF089F94045B2
:1073B0001CD802AA1C4900203FF056FC00283FF4CC
:1073C000DEAE90F800A04FF0000897F81197DFF8B4
:1073D000A8B04D4502AA14494FF000007EDA3FF0F4
:1073E00043FC024658B94A4620496CE099F800002F
:1073F00008F10108FAF7C8F809F8010BD4E7002DE5
:1074000040D11378303B092B3CD919490192FAF746
:10741000C1F8019A90B310465946FAF7BBF8019AA1
:10742000002838D013494EE047410608006D01207E
:10743000EE410608F4410608F0650120FF41060808
:107440000842060816420608224206083442060888
:1074500023430608EC6D01205E42060843430608FC
:107460006A420608884206088D42060863430608F9
:107470004F320608A0420608994206084FF001085C
:107480004FF0FF3510460192FAF79CF90028019A57
:1074900003DA214917E0A846F2E70EAB03EB4503F8
:1074A000013523F8200C94E74A461C490BE032468C
:1074B0001B4908E01B4900203FF0D6FB00283FF4A1
:1074C000F9AE3A4618492046FCF721FB57E63FF053
:1074D000CBFB00287FF428AF144C31E73FF0C4FB0E
:1074E0000028E1D106EBC600114C082203A9823026
:1074F0003744204425F08AFB5046FAF745F887F8D0
:10750000DA0704EB061006A96A0002303FF076FBAA
:1075100087F8F28733E600BFD5420608EA4206083C
:107520000D4306084741060840420608FC6D01204D
:10753000006D01202DE9F04F0F46914689B00021E2
:1075400087EA09099846139A06460025FCF7BAFF10
:107550006FEA09030446DFF880900693284606F098
:10756000D1FF129B184230D0069BDFF870B0034069
:1075700014BF4FF0010A4FF0000A049310EA07030A
:10758000284614BF4A465A460593079206F0CCFF98
:107590004346079A5146039000903046FBF7C6FCDD
:1075A000049B22463046B3FA83F14909FCF78AFF6F
:1075B000039B059A0446009351464346002A14BF94
:1075C0005A464A463046FBF769FC0135182DC5D1AD
:1075D00009B0BDE8F08F00BF724006088843060876
:1075E00037B50446084601913DF06AF80199054611
:1075F00002462046F9F7F2FF70B9625D1046F9F7CE
:10760000ADFF00B932B901352C442046013403786E
:10761000202BFAD003B030BD0020FBE70329F0B5E2
:10762000054685B00C46164614D80B4F3970FBF74B
:1076300031FC0A492846FDF765FD2246084901A8A4
:10764000F9F792FE01AB324608212846FCF768FFA5
:10765000FF233B7005B0F0BDAC030120C64806080F
:107660006E3F06080329F0B5054685B00C46164660
:1076700014D80B4F7970FBF70DFC0A492846FDF72B
:1076800071FD224608496846F9F76EFE6B463246A0
:1076900010212846FCF744FFFF237B7005B0F0BDA6
:1076A000AC030120C64806086A3F060810B5114B16
:1076B00086B0114904460493104B11480393114BB3
:1076C000114A0293114B0193114B0093114BFBF79D
:1076D00045FCFBF7DFFB10491048FBF7C1FC3CB150
:1076E0000F4A1049104806B0BDE81040FBF7B8BC7F
:1076F00006B010BDCF43060899430608D4430608D8
:10770000A4430608DE4306088F430608E74306083D
:107710006F350608FF650120F3430608FB430608A2
:10772000C8EC0508C0EC05080C4406080120BDE7BC
:107730002DE9F04F3E4C87B00A4600210646FCF783
:10774000C1FE05903B4A2378608802EB8303D3F89F
:10775000FCA8F9F73FF98368C1680493364B93F8A6
:107760006420002A4BD0DDF8108004910027217995
:107770006279049B07FB012213F80290B8F1000F15
:107780003FD018F802504D45059A304607F10107E1
:1077900013BF012100214FF0010B4FF0000BFCF74C
:1077A00091FE05907DB305F00F022D095346594611
:1077B000403502923046214ACDE90075FBF7B6FB11
:1077C000B9F1000F2AD009F00F024FEA19195346F8
:1077D0005946029209F140023046CDE90072174A3B
:1077E000FBF75CFBA279012A38BF0122BA42BEDC5A
:1077F0000834134BA342A5D107B0BDE8F08F9046E3
:10780000B4E74546BFE7B8F1000FD9D053460D4A5B
:10781000594630460097FBF789FBD1E77306E1D460
:107820005346084A594630460097FBF737FBD9E7DD
:107830005C8B050878830508F0650120394406084B
:10784000748C05084F44060838B50C4B0C4603EB06
:10785000C0050B4895F8E42703EB8203D3F8FC1826
:10786000FBF77CFB95F8EA3733B1611C0548C9B2D8
:10787000BDE83840FBF772BB38BD00BF7883050810
:10788000C64606088633060873B50E4611490546F6
:10789000F9F780FE18B93070012002B070BD2C7865
:1078A000602C8CBF613C413C072C10D80135012372
:1078B0000A2201A92846F9F7E1FE019B9D4206D064
:1078C0000F2804D8013440EA04143470E4E700209F
:1078D000E3E700BFA344060802460846531C05D14F
:1078E000044B1A681B790A600B7170470249F9F75B
:1078F0003BBD00BFA344060887330608224BB0F502
:10790000FA6F1A680346A8BF4FF4FA63B3F57A7F9B
:10791000B8BF4FF47A73D20416D540F2DC529042CD
:1079200015D040F2DB5207EE903A9042F8EE677ABB
:107930001FD8DFED166A9FED167A77EEE67A9FED97
:10794000150AA7EE870A7047B0F57A7F02D89FED37
:10795000120A704707EE903ADFED106A9FED107A39
:10796000F8EE677A9FED0F0A77EEE67AA7EE870AC0
:107970007047DFED0D6A9FED0D7A77EEE67A9FEDA9
:107980000C0AA7EE870A7047706B012000007A444A
:10799000D62000C000E082440000000000407A448D
:1079A000661000400000404200A0BB44D6200040CA
:1079B0000000834410B584464FEA810E102312F470
:1079C000004F4FEA420214BF0E240724013B92B23B
:1079D000CCF80040F444F2D100EB81128C01035149
:1079E000122042F8213010BD10B584464FEA810EB6
:1079F0000424130B013C4FEA021203EB430392B23F
:107A000003F11803CCF80030F444F2D100EB011379
:107A10000A018450062043F8214010BD704700BF82
:107A2000704700BF034B00EB400003EBC000407CFD
:107A3000704700BFF40600202DE9FF471E46C368CB
:107A4000044689469246BDF83070DDF834804BB369
:107A5000CBB20D2B24D81A4AD556BAF1FF3F23D00A
:107A600023683146174A3846CDE9005AC047524686
:107A70005FFA89F12079F2F731FB024600B1028802
:107A8000D3B2314638460393C2F30323120B029359
:107A90002368CDE900520C4AC04704B0BDE8F08726
:107AA0000025DAE74D1CD8E77B06F6D4236831467B
:107AB000064A3846C4460C9504B0BDE8F047604716
:107AC000A4EC0508684406087544060899440608AD
:107AD00000231E211D22017042708370C370704705
:107AE000704700BF00207047704700BF00207047FC
:107AF00001207047704700BF704700BF704700BF4C
:107B0000704700BF9FED010A704700BF00000000F2
:107B10000020704703681B691847094B002230B5E5
:107B200093F9004001325D7804330119062ACD72C1
:107B300013F8025C055513F8014C8C75F0D130BD7B
:107B400024BD0508002383700370C3704370704721
:107B5000D0F8FC304BB1D0F88C31D0F814211B6830
:107B60005B689A4205D3D01A7047D0E907239A423E
:107B7000F9D2C0681044C01A704700BFD0E909129A
:107B800091420ED38A1AD0F80011036981B1D0F85E
:107B90008811013B096849680A4493420BD9981A35
:107BA0007047036919448A1AD0F800110029EED1F0
:107BB000013B981A70470020704700BFD0F8003191
:107BC00013B190F8A4017047D0E90903181AB0FA6C
:107BD00080F04009704700BFD0F8FC20034610B485
:107BE00072B1D0F81421C1685C69881A013A205C2E
:107BF00008BF0A465DF8044BC0B2C3F814217047B1
:107C0000006A5C69411C205CDC68C0B2A14238BFDC
:107C10000A465DF8044B1A62704700BFD0F8A831DD
:107C200003B11847704700BFF8B590F8BD31012B7C
:107C30001CD0002A164619DD05460F460269436A24
:107C4000D41AA8693946B4421844A8BF344622461B
:107C5000361B3EF0D3FF686A2A6927440444002E8D
:107C6000B4FBF2F302FB13436B62E9DCF8BD00BF27
:107C70000023084901E0152B09D003EB430201332F
:107C800011F802C00A448445F5D11046704700201F
:107C9000704700BFD823012008B3B1FA81F35B0914
:107CA000E9B14FF0100C10B50E4C4FF0010E22460A
:107CB00004E001334E2B10D092F804C0604502F16D
:107CC0001C02F6D10EF1010C71455FFA8CFEF0D169
:107CD000C3EBC30304EB830010BD002010BD0020E4
:107CE000704700BF887A05082DE9F0411E4688B02C
:107CF000030990460E9F00F00F04403349B30793E9
:107D0000FFF7CAFFC2790546079B41463046CDE9D9
:107D10000042144AB847C8B12868F2F775FBA97940
:107D20006A7911F0020FDFF84CC04FEA92020E4957
:107D3000ED7908BF61460132079B0094CDE901024D
:107D4000CDE90315094A00213046B84708B0BDE81F
:107D5000F081074A41463046BC460E9408B0BDE863
:107D6000F0416047A8440608D9330608BA4406081B
:107D7000DC440608C648060870B5094C236873B190
:107D80000546002606E099681A681E732160904730
:107D9000236823B15A681846AA1A002AF3DA70BD7C
:107DA000508E01202DE9F041154686B088461946CF
:107DB0006A1CBDF830600D9F23D0030900F00F044A
:107DC000174A30464033CDE900450593B847A8B17E
:107DD0002A4698F80510D8F80000F2F7C7F968B1FC
:107DE000028801783046059B0391C2F30321120BF0
:107DF00002910021CDE900420A4AB84706B0BDE829
:107E0000F0817306FAD4030900F00F00064ABC465D
:107E10000C904033304606B0BDE8F041604700BFEB
:107E2000EE44060800450608294506082DE9F04FEE
:107E3000704D0A460021824605F1800B2DED028B24
:107E40008BB0FCF73FFB814600266B4B1C78AB7A6E
:107E5000B34200F391801035AB45F5D140F21620C6
:107E6000F8F7B8FDD0E902530CB12C461D460DF1D0
:107E7000100B00271522002158463EF033FF2E78C4
:107E8000002E41D069783046FFF706FF95F90230A1
:107E900008EE100A5A1C029353425341002C00F082
:107EA000A580002214F802C0A018B44540F09A80C2
:107EB00090F90280029A424540F0928042788A42CC
:107EC00008BF0123012203F001030BF807204A46F3
:107ED00083F0010150460393FCF7F4FA039B8146BB
:107EE0004CB1464A18EE101A3046CDE900A242467F
:107EF000FFF758FF039B424A18EE101A3046CDE9AF
:107F000000A2029AFFF74EFF01370335152FB6D1B5
:107F10006CB304F13F06394FDFF8E4801BF8013BF6
:107F200002930BBB2078F8B194F9022001321BD0E8
:107F30006178FFF7B1FE05464A4601215046FCF73D
:107F4000C1FA94F90220029B294681462078CDE9A6
:107F500000A7FFF727FF2078029B4FF0FF3229464A
:107F6000CDE900A8FFF71EFF0334B442D6D10BB011
:107F7000BDEC028BBDE8F08FE888F8F72BFDD0E967
:107F800002230CB114461A46297A6B7A06FB013398
:107F900012F903800CB3E756B8454A4650460DBF68
:107FA00001230023012100210293FCF78BFA029B9D
:107FB000814644B1114A31462846CDE900A23A46ED
:107FC000FFF73AFD029B0E4A314628460136CDE9BD
:107FD00000A24246FFF730FD37E74FF0FF37DBE7FF
:107FE00000236FE703323F2A7FF45CAF4FF0FF3886
:107FF0006DE700BF00040120546601202D2F010809
:108000009D2E01082DE9F04F07468BB040F2162057
:108010000391F8F7DFFC039A044600213846FCF789
:1080200051FA3F4A0646D4E9025314780CB12C4663
:108030001D461522002104A83EF054FE05F13F0321
:10804000039395F80090B9F1000F30D095F801A096
:10805000002C63D0224600231178494557D128339C
:1080600092F8018001226B4403F8182CD045324667
:10807000384613BF012100214FF0010B4FF0000BD8
:10808000FCF720FA064654B1B8F1000F07D0254B93
:108090005A464146484600933B46FFF725FE224B91
:1080A0005A465146484600933B46FFF71DFE0335AE
:1080B000039B9D42C5D13CB3651C0DF110084034B3
:1080C000DFF86090DFF860A018F8013BCBB915F835
:1080D000013CB3B116B13046FAF7FAFE29783B46B7
:1080E00015F8010C0022CDF800900026FFF7FCFDEA
:1080F000002215F8010C3B461146CDF800A0FFF711
:10810000F3FD0335A542DFD10BB0BDE8F08F01339D
:108110000332152BA0D14FF00008A7E7A046A5E732
:10812000546601202D2F01089D2E010810B5013144
:108130001446FFF7B1FD28B9064B1A681B79226077
:10814000237110BDC27920460349BDE81040F9F7FC
:108150000BB900BFA3440608B544060808B5294B6F
:108160001B68DB041ED5B5EE400AF1EE10FA26D0EE
:10817000DFED257AB4EEE70AF1EE10FA1FD49FED99
:10818000237AB4EEC70AF1EE10FA2AD870EE677AB5
:108190009FED1F7A9FED1F0AA7EE870A3DF0B6FFFD
:1081A00080B208BDDFED187AB4EEE70AF1EE10FAFE
:1081B0000BDA9FED190A3DF0A9FF80B208BD9FEDD3
:1081C000170A3DF0A3FF80B208BD70EE677A9FEDFD
:1081D000147A9FED140AA7EE870A3DF097FF80B24C
:1081E00008BDDFED117ADFED116A70EE677A9FED61
:1081F000107AA7EEA67AB0EE470A3DF087FF80B26C
:1082000008BD00BF706B01200000404200E08244C6
:1082100066BEFFBE0060BB4400007A440080BB44E1
:1082200038DFFF3E00407A440000834466BEFF3ED4
:1082300000A0BB446D4B1B782DE9F04F87B0002B9D
:1082400000F0CE806A4D4FF000086A48A968FAF73E
:1082500007FF69686848FAF703FF684B6848DFF86A
:10826000D8A1D3E90031C91A664B1A68B1FBF2F202
:10827000FAF7F6FEFAF70EFE6348FAF723FE6348B4
:10828000FAF720FE624B5FFA88F41B78A34221D8EC
:10829000604C0025604FFAF7FDFD2646013556F883
:1082A000041B3846FAF75AFE162DF7D101255A4E0F
:1082B000FAF7F0FD23466168013530461B68043447
:1082C000C91AFAF74BFE162DF4D107B0BDE8F04FEE
:1082D000FAF7E0BD514B14264FF03C0B671C03EB43
:1082E000840306FB045693ED000A3DF00FFF96F859
:1082F0001EE081B2B6F80E901EF0010F80B214BFDE
:1083000052222D221EF0020F0490504614BF542317
:108310002D231EF0040F07EE903A14BF56232D2391
:108320001EF0080F009317EE903A14BF4FF0430C65
:108330004FF02D0C1EF0800FCDF804C014BF4FF08D
:10834000530E4FF02D0EB1FBFBF10591642101FBA3
:1083500009F1CDE902E13946FAF700FEB37FDB0708
:108360003AD55C232E4A6343D118D05891ED010AC7
:1083700070B1B8EE400ADFED2B7A20EE270A07EE47
:10838000900AF8EE677A80EE270A3DF0BFFE00B251
:10839000642290FBF2F102FB11022348FAF7DEFDA2
:1083A0001421224808F1010801FB075701FB04547E
:1083B000F988628A0491218B02F0030392080391E9
:1083C000E18A0291A18B0191A18A009119214B436D
:1083D000218AFAF745FE55E71548FAF73BFDDFE736
:1083E000144807B0BDE8F04FFAF76CBD80010020DB
:1083F000B40C00203D4506084D4506088C160020AB
:1084000064450608B81D012091450608ED4506089B
:1084100054240020600D00209D4606087C55002055
:10842000BC0D002000401C46664606087B46060838
:1084300072460608A1460608494606082DE9F84F87
:1084400006460C461E4D36274FF00008DFF87890A0
:10845000DFF878A02046FCF7F1F9D5F800B048B96C
:1084600021465846F9F7DEF820B921466868F9F741
:10847000D9F880B15846FAF7EDFC696811B1504659
:10848000FAF76CFDA96811B14846FAF767FD4FF09D
:108490000108FAF7FFFC013F05F11005DAD120468B
:1084A000FCF7CCF948B9B8F1000F06D122463046A6
:1084B0000449BDE8F84FFBF72ABBBDE8F88F00BFC1
:1084C0003CBD0508C9460608C3460608BD46060861
:1084D00070B504680546236A1B6943B1236AD0F866
:1084E00094001B69984701282AD002280DD0236ADE
:1084F000DA699AB9586958B399692162BDE8704040
:10850000C3E905223EF088BD2362236ADA69143389
:10851000002AF9D1236ADA69002AEBD0216A1433E0
:1085200094F824200E7B2362F6B2DAB996B9284675
:10853000F1F72CFD28460121BDE87040F1F7A6BCFB
:10854000236A01462846143B2362F1F79FFCCEE7DD
:10855000206270BDAB68002BE9D09A8819681204BC
:108560008A61E4E700212846F1F790FC002384F8B3
:108570002430002EDBD0EDE738B58569002D3DD0E5
:108580002C68236A1B7B5BBB20463CF03BF8236ACC
:108590005B680BB3236A5A68236A22F01F025B6888
:1085A000216A886803F01F0100F11F03194421F0BC
:1085B0001F01BFF34F8F00290ADD02F12003114490
:1085C0000F488B42C0F85C221A4603F12003F8D111
:1085D000BFF34F8FBFF36F8F2846BDE8384077E772
:1085E000AB68002BD0D01A6820469B8893613CF082
:1085F00009F8236A5B68002BCCD1EDE738BD00BFDA
:1086000000ED00E038B5846904B938BD2568284616
:108610003BF0F8FF2B6A1B7B1BB92046BDE83840B6
:1086200056E7A368002BF8D01A6820469B88936110
:10863000BDE838404CE700BF8160F4F78FBD00BF54
:108640000171F4F78BBD00BF38B5D0F8A8310446EE
:108650000D460BB19847B8B1636AA269D554636AF5
:1086600021690133D4F800218B4228BF00236362C3
:1086700022B12046BDE83840F4F722BFD4F82021CB
:10868000136843F08003136038BD00BF90F8BD212C
:10869000012A0AD0D0F800210AB1F4F711BFD0F8AE
:1086A0002021136843F0800313607047AF4B1B68B1
:1086B00093B35B692DE9F04786B0984748B3AC4D5A
:1086C000D5F8CC36002B01DDF7F7CCFAA94C63784E
:1086D000022B22D0032B1CD195F8E83713B1A64802
:1086E000F7F736FB95F8D43613B1A448F7F730FB0B
:1086F00095F8183713B1A248F7F72AFB95F85C37BD
:108700003BB1A04806B0BDE8F047F7F721BB032313
:10871000637006B0BDE8F0877047A37804F10408E1
:1087200004F1080704F5BD56072BF2D801A252F850
:1087300023F000BFCD870108F9880108F7870108F9
:10874000C187010855870108778801088B880108CF
:108750000F87010823784FF0010A207D032B0CBFFF
:108760004FF080094FF48079002800F0B080012894
:10877000FAD1D5F8403800215A024FF0FF33B3FB4D
:10878000F2F362689A18D5F8383803F1020341EB26
:1087900001009342814139464FF0020038BF1A462A
:1087A000F6F756FA032800F25B8101A353F820F094
:1087B00013870108A388010813870108A38801080B
:1087C00095F8A037002BA4D06F489BE7002305A99C
:1087D000092218460391F6F7E1F8012899D1059B83
:1087E00093F8FE21552A00F0D5800222012385F856
:1087F000E42763708DE7654803213023052200904C
:10880000A170614862493BF035FD82E70623A37001
:108810002369652B39D92278653B032A0CBF6FF099
:108820007F026FF0FF0203EA02030CBF80224FF4C5
:10883000807201339A42236127D2E268D5F8381852
:1088400098180231884207D395F8E41711B901212D
:1088500085F8E41701216170C5F8C427C4E9012037
:10886000D5F8402802FB03F35B02C5F8A837C5F82A
:10887000AC370523A370A26841460120F6F77EFAC3
:10888000012840F0A5800623A37000213046F6F7AA
:108890002BFB012840F09C80A3780133DBB2A3704E
:1088A00042E7D4E901C32269A3EB0C01914288BFDE
:1088B000C4E903C10328A9D00133B3FBF9F209FBD2
:1088C00012320AB14B449B1A002063602075D5F820
:1088D000382841460232F6F7BBF9032800F2C0807F
:1088E00001A353F820F000BF138701086189010834
:1088F000138701080D88010805A900230922D5F86E
:108900002C08F6F74BF801287FF403AF0022059BF3
:108910002270B3F80B20B2F5007F1BD11A7C022A1B
:1089200018D193F8FE21552A14D193F8FF21AA2AD1
:1089300010D1B3F80EC0D5F82C686644C5F830687D
:108940005F7B7A1EC5F840787F2A03D87A4237EADF
:10895000020245D00322012385F8E4276370D8E69C
:10896000636884F814A00133A360FDE6281D01208C
:10897000983D0120982D0120804501206C44012064
:10898000B0440120F444012038450120698A0008E0
:10899000984C060893F8FF21AA2A7FF426AF03F526
:1089A000DF72039903F5FF73906840B11679A6F161
:1089B0000B0706F0F706012F05D9062E03D010325B
:1089C0009342F1D111E70123C5F82C08A37094E775
:1089D00002287FF49EAE012385F8E437637098E6A1
:1089E0007A02013AC5F84828D88A00B9586AC5F809
:1089F0003408B3F81120520102F2FF125212C5F8E6
:108A00005028B3F8131001B9196A94440CEB400CC8
:108A10004000A1EB0C01B1FBF7F140F6F477C5F88B
:108A20003818B94219D94FF6F477B94211D9032150
:108A30002170DB6A3244C5F84C3895F81038104480
:108A4000C5F83C080BB9F7F78FFFA3780133A37083
:108A50005FE6022323700023ECE70123237079E70C
:108A6000207D81E62DE9F84FAD4C80462379DB0768
:108A70002DED028B6BD5AB4B6579AB4E1F88012D6D
:108A800056D0022D35D0002D3ED094ED068AF37BD2
:108A900033B1B38923B1A54B1B78002B40F0CB80B9
:108AA000A279337A632B06D8022D00F0DD80217C79
:108AB000002940F0ED8095429D4BB0EE487ADFED05
:108AC0009D6A38BF1546B27B1D70D4E90A31E36256
:108AD0005B1A07FB03F307EE903AF8EEE77AA7EE8E
:108AE000A67A84ED067A002A5FD1BDEC028BBDE840
:108AF000F88F6389BB42C8D28F4B012594ED068A5B
:108B00001B686571E361C2E7A389BB4219D38A4B35
:108B1000E1691A68F37D521A03EB830303EB8303C5
:108B2000B2EB830FB1DB012594ED068A6571AEE7E8
:108B3000E389BB4280F086802389BB4201D20025B5
:108B400065717D4B94ED068A1B68E3619FE765794B
:108B5000DFF8D091EB1E012B32D9B9F80800C0F331
:108B60000B003CF0D9FA092840F3A7806E4EB9F803
:108B70000070F3889F4203D33288BA42BFF47FAFBC
:108B8000B7EB430F3FF77BAF0323DFED6C7A674A08
:108B90006371B0EE678AA3710023C4ED067A137087
:108BA00023816381A381E3817EE0012D7ED0022DAC
:108BB0009BD10720BDEC028BBDE8F84F06F010B842
:108BC000594EB9F80070F3889F4202D33288BA42F6
:108BD00002D2B7EB430F63DDB9F80800C0F30B0016
:108BE0003CF09AFA092873DD0022357D6271A2718A
:108BF000002D70D04D4B1D702B46154699B2B28892
:108C0000738812FB01F213FB01F3717C92B29BB2E9
:108C10008A422281638140F2B980521A92B28B4219
:108C2000A28140F2B1805B1A9BB2E381642363743A
:108C30000023636123E713F035FA002841D10222B3
:108C4000A2712EE73C4BE1691A68337E521A03EB9E
:108C5000830303EB8303B2EB830FFFF616AF02250A
:108C600094ED068A657112E7207C88B90121C4F869
:108C7000148080462174C3F16403314908FB03F377
:108C800081FB0301DB17A3EBA1536433637412E789
:108C900060692C49A8EB00088845ECDB63740AE79F
:108CA000032D7AD194ED068A0325F0E6BDEC028B04
:108CB0000820BDE8F84F05F093BFB9F800701A4ED0
:108CC000DDE6337C83422CBF01220022A271E8E65C
:108CD000032DE7D0D9E632881B4BDFF850A01B6884
:108CE000B7FBF2F2013293F96C10082A28BF082270
:108CF000D3B28AF80030002980D091423FF47EAF91
:108D0000124991F800E00EF1010101F003018E45D6
:108D10003FF474AF4FF0FF3C4FF0A40B22E000BFD4
:108D2000508E0120B8770120746B0120B7770120A5
:108D3000B6770120ACC527372C1D012000000000AC
:108D40006BCA5F6B80969800F8690120F865012076
:108D500018B93CEA2C0C28BF8C46013101F0030104
:108D60008E4515D012480BFB010090F96C00824231
:108D7000EED18C465FFA8CF0F9F702FD9AF80030DC
:108D8000B9F80070657939E700234EE7002246E71D
:108D9000BCF1FF3F3FF432AFECE7B9F80800C0F395
:108DA0000B003CF0B9F909283FF7E1AE6DE600BFD2
:108DB000386701202DE9F047694CA36820469847A1
:108DC000002869D0B4F90E3004F14805A17D06EE03
:108DD000903AB4F91030092907EE103AB4F912307C
:108DE000F8EEE66A07EE903AB8EEC77A4FF0010364
:108DF000F8EEE77AC4ED126A84F8543084ED137A01
:108E0000C4ED147A4AD0574F28461CF051FFBB8D51
:108E1000002B4CD1544B1B685B0770D4BB6AD4ED5C
:108E2000127AB3F90220D4ED135A06EE102AB3F9E0
:108E30000420B3F9003007EE102AB8EEC66A00EE3F
:108E4000103AD4ED146AB8EEC77A484DB8EEC00AAD
:108E50003B8835EEC66A464E36EEC77A05F10808FD
:108E600037EEC00A84ED136A84ED147A84ED120A99
:108E700053B9A84506F10C0605ED010A0CD03B8854
:108E8000B5EC010A002BF4D030460C363EF0A8F8C1
:108E9000A84505ED010AF2D1BDE8F087314F04F194
:108EA000200128461CF0C8FEBB8D002BB2D0D7F89D
:108EB00028C02846DFED2F6A00252F49ACF10202B9
:108EC0000CF10406B3F5C87F1CD0D1ED007AB8EEE2
:108ED000E77AD0ED007AE0EC016A77EE877AFDEE72
:108EE000E77AE1EC017A22F8025FB242EAD1012B83
:108EF0000CD0013BBB851C4B1B685B078ED534F047
:108F0000C5FF8BE7B0EE667A0D60E2E71B48DFF83D
:108F100074E0816BB4F80C80C831194E8EFB01A946
:108F2000C917D0E90C20C1EBE911C832C830A1EB58
:108F30000801ACF804108EFB0281D217C2EBE112DB
:108F4000ACF800208EFB002EC017C0EBEE10ACF882
:108F50000200B581F5817381F9F7EEFDBB8DC8E79D
:108F6000E4250020B0250020706B01203026002071
:108F7000B425002000000000808E0120508E0120CA
:108F8000C46B01201F85EB5138B5074C074DAC422F
:108F900003D3074B01221A7038BDA288D4E902100E
:108FA0003DF02CFE1C34F2E764B8060878C10608D0
:108FB000546601202DE9F04F0C4695B00546344922
:108FC00020461746FEF70CFB064600284FD13149D4
:108FD0002046FEF705FB064600284AD12E492046CA
:108FE000FEF7FEFA0646002845D12C492046FEF73A
:108FF000F7FA0646002840D120462949FEF7F0FA44
:109000000028064612BF0824264601240FB144F06A
:10901000100424493046FEF7E3FA80B344F02004FC
:10902000214B1B780BB9FFF7AFFFF7F765FD14F085
:10903000090F00F047831D48F9F74AFF0020FEF7AB
:1090400035FB14F4807306933CD11948F9F740FFBF
:109050001848F9F737FF04F01803182B05D1164804
:10906000F9F736FF1548F9F72DFF01232BE001240E
:10907000CCE70224CAE70424C8E78124C6E71049E4
:109080003046FEF7ADFA0028CAD044F48074C7E732
:10909000FC460608034706080B4706081147060862
:1090A0001A470608A53C060854660120234706080F
:1090B0002B470608434706084F4706087747060828
:1090C0001E47060800230593F9F7E4FEBC4904F0A7
:1090D0001008BC48F9F7C4FFBB49BC48F9F7C0FF0A
:1090E00004F48473082B07D1B9492846FAF738F8F5
:1090F000B7492846FAF7A8FD14F0800308930CD16D
:10910000B44B204613F83C2F002AB34A06BF012176
:1091100013460021B14AF9F7C1FEB1492046FEF7D6
:1091200007FBB0492046FEF76DFFAF492046FEF72A
:109130007DFEAE4BD3F800B0AD4B1B680493B8F185
:10914000000F40F0FD814646AA48F9F7C1FEAA4B40
:109150004FF00009DFF864A307930393049B6BEAC5
:1091600003030A93039B53F8047B0393002F40F0FF
:10917000E981049BDFF848A363EA0B030993079B8B
:1091800053F8042B03920793002A40F005829B4B6F
:1091900020469B4A9B49FCF77FFB089B002B40F035
:1091A000A382DFF820A32046DFF81CB39AF8002042
:1091B0009BF80030DFF814939A42934A13BF0121C1
:1091C000002101270027FBF77DF99BF80030394685
:1091D0000646013B8D4A204659F82330F9F7A6FE92
:1091E0009AF8003039468A4F013B884A204659F8A0
:1091F0002330F9F753FED7ED007A864A2046F5EE84
:10920000407AF1EE10FA0CBF01210021F9F746FE79
:1092100033463A4680492046FCF7C6FD7F4B804ADC
:1092200020468049FDF702FAB8F1000F05D07E4BC9
:1092300093F90230002B00F0DF817C48F9F748FEFB
:109240007B48F9F73FFE0023774A20467949FDF72E
:109250002BFB794B6FF07F42784F794E204601937C
:1092600000923A683168FEF765F940F20222754BC8
:10927000204600920193BA68B168FEF75BF9B8F135
:10928000000F40F0BB817048F9F722FE42466F485C
:1092900008266F490127DFF838C210F8013B11F8A2
:1092A000019B03F1500EEE440EF8209C1CF801EBDC
:1092B0000EF1500AEA440AF8109C2FB1A3EB0E0EEF
:1092C000DEF1000747EB0E07013EE6D187F0010112
:1092D00020468DF83860FBF7F5F810AB5D4A39464B
:1092E00020468DF84860F9F721FE0CAB594A394603
:1092F0002046F9F7D3FD584B584A20465849FCF709
:109300008DFF584B584A20465849FDF713F8584BE3
:10931000524A20465249FDF79FF8564B564A20467E
:109320005649FCF76DF9564B564A20465649FCF70C
:10933000F5FB564B564A20465649FCF7AFFE564BB6
:10934000564A20465649FDF7ABFD564B564A204635
:109350005649FDF789FCB8F1000F40F0518154489F
:10936000F9F7B6FD534F4FF0000BDFF86881414627
:10937000022238463DF08CFC002897F800A02046D9
:1093800014BF01210021039A0CBF4FF001094FF0D7
:109390000009FBF797F8BAF1020F039040F0338110
:1093A00098F801204FF0190A40F2EE234946204672
:1093B0001AFB0232404B019298F800208CE000BF6B
:1093C000874706081F390608954706083D390608ED
:1093D000C6480608508E01205A6006089A470608BB
:1093E000A7470608B147060818350608A08C0120D3
:1093F0006C6B0120DD46060838890508CE47060853
:109400003C6A01204C880120EB460608D547060837
:10941000D0790120DE470608DC8A01204941060890
:10942000507B012024810120B07B0120E546060805
:10943000ED470608B0800120FA470608746C012049
:10944000288D012001480608F1460608E089012020
:10945000283206087B3C0608EB390608607A0120B2
:10946000888101200D480608E07A01200882012049
:109470000848060813480608E06B0120888401208C
:1094800017480608A4780120908201202048060889
:10949000507A01207C82012028480608006D0120B6
:1094A000C088012031480608207C0120A08B0120C3
:1094B000F5460608C083012054010608B747060890
:1094C000C3470608D08D0120FC690120B489050836
:1094D000046A01205C7801209A5C5B460092864A0F
:1094E000F9F724FD7A7840F2EE21844B20461AFBEE
:1094F0000212494601923A789A5C5B4600927E4A93
:10950000F9F7CCFC0BF1010B023708F10208BBF1B3
:10951000120F7FF42CAF7A4B224600212846FAF72F
:10952000FFFF230700F18580764E224628463178DA
:10953000FEF774F8224671782846FEF793F8B7E0F4
:10954000714E04E63B7823B301230A9A204603FABE
:1095500009F31A400B930CBF0121002109923246F6
:10956000FAF7B0FF049B0646204663EA0B020B9B0A
:109570001A423B46524614BF01210021F9F7D6FC9E
:1095800009993B4652460039204618BF0121F9F798
:1095900085FC09F10109E5E5039B1B7853B34FF006
:1095A0000109049B09FA07F913EA090F0BD06BEACA
:1095B00003035246204613EA090F039B14BF0121FF
:1095C0000021F9F7B3FC1BEA090F13D0099B3246BF
:1095D000204613EA09090CBF01210021FAF772FFA6
:1095E000B9F100010646039B524618BF01212046EF
:1095F000F9F754FC0137C2E5444B25E6444A46E6F8
:10960000444B0393AEE698F8002049463B4B204676
:109610009A5C5B460092404AF9F788FC3A78374BEF
:10962000494620469A5C5B4600923B4AF9F736FC75
:1096300068E70027F9B2013722462846FDF7EEFF1A
:10964000042FF7D12F4FDFF8F4803B7888F80030F3
:10965000069B33B93148F9F73BFC31492846FBF703
:1096600051FDFF2388F80030F1B20136224628462A
:10967000FDF7F8FF042EF7D17B782A4C2370069B68
:10968000A3B92948F9F724FC25492846FBF76AFDC8
:109690002648F9F71DFC2648F9F7DCFBFF23237069
:1096A000002015B0BDE8F04FFAF717BFFF23237075
:1096B000059B002BF4D01F48F9F70AFC1E48F9F768
:1096C00001FCEDE7A10706D50E4B22462846197886
:1096D000FDF7A4FFE4E76207E2D50A4B22462846DD
:1096E0005978FDF7BFFFDBE7054B224618212846D6
:1096F000FAF716FFDCE700BFDD3C06085401060858
:10970000FC460608188E0120DD460608E5460608D8
:10971000F1460608F5460608ED3C060835480608F9
:10972000C6480608AD030120584806087F480608C9
:109730008247060892480608A8480608AC0301209C
:10974000002237E4012235E4224B30B583B09A7908
:1097500001906AB393F82630DFED1F6A07EE903A66
:109760001E4B1F4CF8EEE77A1D7886EEA77A84ED43
:10977000187ADDB11B4BDDED017AB3F86A30F8EEF3
:10978000670ADFED197A00EE103A60EEA70AB8EE2C
:10979000400AF7F7F5F904F12003002103EBC502B5
:1097A0001960083303ED010A9A42F9D103B030BDC4
:1097B0000E4A12681201F9D593F82630DFED066AD9
:1097C00007EE903A064BF8EEE77A86EEA77A83ED3D
:1097D000187AEBE7F8250120555555405424002010
:1097E0007C550020508E0120BD378635706B0120DE
:1097F000A54B1B78002B00F0B2802DE9F04FA34D54
:1098000083B095F80491B9F1010F02D003B0BDE81F
:10981000F08F9F4B9F4C1B6893F83470002F6ED0D5
:109820009D4B0022DFED9D6AA64694ED187A904686
:1098300093F800B040F6FF7A67EE266A9FED986ACB
:109840002B46984E019200941CE000F47061B1F533
:10985000006F00F0B38000F29380B1F5806F00F0EC
:10986000DB80B1F5C06F7BD1C0B24CF0080C9882A0
:1098700083F81EC0013214330EF1040E0236D2B248
:10988000BA422AD093F81EC09889BCF1010FDCD1EE
:10989000504500F0D080C0F30801400A01FA00F002
:1098A00081B2002900F0BF807F4C80B2BBF12D0F48
:1098B00004EB5101B1FBF0F000F0D7804FF6FF71DF
:1098C0008842D7D007EE900A0199F8EEE77A014472
:1098D00080B2019167EEA67AB3E0009CB8F1000F68
:1098E0000DD0DDED017AB8EE677A07EE908AF8EEDA
:1098F000677A27EE267AC7EE276AC4ED196ADFF881
:10990000B4A16A4A9AF80030A26613B3684E0027E1
:10991000DFF8788106F14C09B8F80E30304694ED46
:10992000180A013707EE903A08F114080836F8EEE5
:10993000E77A27EE800A3DF04BFB9AF80030D4ED31
:109940001A7ABB42A9EC010A87FEC00A84ED1A0A02
:10995000E2DC022385F8043103B0BDE8F08F7047E4
:10996000B1F5007F31D14CF0020CC1B283F81EC0BA
:1099700093F81FC019828C45BFF47CAFD87779E784
:10998000B1F5406F13D0B1F5606F06D1C0B26CF085
:109990007F0C988383F81EC06CE7B1F5206F14D15B
:1099A000C0B24CF0200C188383F81EC062E7C0B22E
:1099B0004CF0400C588383F81EC05BE7C0B24CF0FB
:1099C000100CD88283F81EC054E7504546D0C0F32F
:1099D0000801400A01FA00F081B221B3324C80B292
:1099E000BBF12D0F04EB5101B1FBF0F049D04FF664
:1099F000FF7188423FF43EAF07EE900A0199F8EEFE
:109A0000E77A014480B2019167EEA67A4CF0010C2E
:109A1000D88183F81EC017E0C0B24CF0040C588205
